:020000040800F2
:10000000F8BF01201D010208FB0E0508E90E0508D6
:10001000FD0E0508090F0508150F05080000000072
:10002000000000000000000000000000210F050893
:10003000230F050800000000D51105080D0200205F
:1000400001000208250F0508310F0508390F0508C2
:100050000576050801000208C5690508CB69050891
:10006000D1690508D7690508DD69050891300508DB
:10007000A1300508B1300508C1300508D1300508A8
:10008000E1300508F130050801000208495605086D
:100090001D5605082D5605083D560508E369050857
:1000A0004D0F0508530F0508650F05086B0F050870
:1000B000710F0508770F05087D0F0508F53605084F
:1000C000113705082D3705084937050801000208D2
:1000D00001000208390300203F03002045030020EF
:1000E000076A05082B0F050801000208A90F05087B
:1000F000AF0F0508C70F0508C10F05080131050836
:100100000100020801000208850F0508010002082D
:100110002D030020330300209D0F0508A30F0508C1
:100120001131050821310508313105084131050833
:100130005131050800000000000000008956050844
:100140005D5605086D5605087D5605080100020834
:100150006131050871310508813105084B03002024
:10016000653705088137050801000208010002080B
:10017000010002080100020801000208000000005E
:100180000000000001000208000000000000000064
:100190000100020800000000000000000100020849
:1001A0000000000000000000000000000100020844
:1001B0000100020801000208010002080100020813
:1001C000010002080248002343643C3000F048B9B3
:1001D000B4040020054B43F82010054B01221A609F
:1001E000044B4FF080525A60704700BF740B0020E0
:1001F000780B002000ED00E010F4FF7F02BF024BFF
:100200000422C3F8002E704700E100E00D4B10B54A
:100210001C6801341C604FF0E02304F001021B69EC
:10022000094B53F822300BB120469847074B1B6807
:10023000A34205D1BDE8104005490020FFF7CABF21
:1002400010BD00BF240A00207C0B0020200A0020E3
:10025000C9B4040838B5334B03EB8003D3F88C41A1
:10026000002C37D06368196889B28A06E18341D5CA
:10027000608A00283AD0A28A92B20132B2FBF0F52D
:1002800000FB1522E08A92B290422FD01968E183D8
:100290005968A3890B40A17AE9B1234909689942B9
:1002A00019D1FFF78FFFA38BDD0631D40125637AC7
:1002B000A28B5B0742BFE38B23F01003E383E38B46
:1002C0001A4202D0206A00F0C3F8637A35B323F0F3
:1002D0000403637238BDE17AA0690129A18A89B259
:1002E0000CBF20F811304354A282DCE7DA6822F018
:1002F0002002DA60C80642BFDA6822F01002DA6033
:100300000A0742BFDA6822F02002DA600025CEE751
:100310006268D36843F01003D360C7E743F0040377
:10032000D7E700BFB4040020A80400200420FFF792
:1003300091BF0520FFF78EBF0120FFF78BBF022082
:10034000FFF788BF0320FFF785BF0620FFF782BFB6
:10035000114B70B500220446DA6100F071F80F4DC0
:100360000646EB68DA030CD4EB68DB0744BF0123D5
:10037000EB60E86810F4F97007D000F075F8012020
:1003800003E0611CEDD00CB9032070BD00F058F8FB
:10039000801BA042E5D9F7E7280A0020003C024074
:1003A0002DE9F843DFF8948098F81830012B0546C2
:1003B0000F463FD001234CF2503088F81830FFF739
:1003C000C7FF0446A0B94FF0FF333B602B68012BF9
:1003D00014D1287C00F050F84CF25030FFF7B8FFF1
:1003E000154A136923F004030446136100F034F83E
:1003F000002388F818302046BDE8F883AE68DFF89F
:100400003890D5E902231344B342EFD9297C304612
:1004100000F02EF84CF25030FFF79AFFD9F8103068
:1004200023F0FA03C9F8103010B13E600446DDE74E
:100430000136E6E70224DEE7003C0240280A0020FD
:10044000014B1868704700BF240A0020000000001C
:100450005FF800F021AF04085FF800F0910505088F
:100460005FF800F0B1E202085FF800F0D50305087C
:100470005FF800F0490505085FF800F0250505085C
:020000040802F0
:10000000FEE700000F49D1F8883043F47003C1F8CF
:1000100088300D4B1A68002042F001021A60986087
:100020001A6822F0847222F480321A60074A5A60F9
:100030001A6822F480221A60D8604FF000638B6047
:10004000704700BF00ED00E000380240103000248F
:1000500010B5002494B02C22214609A803942AF05C
:1000600055FB2A4B00941A6C42F080521A641B6CA8
:1000700003F080530093009B254B01941A6842F4CF
:1000800040421A601B680A9403F440430193012222
:10009000019B04944FF4A023CDE9072310234FF4D0
:1000A00080000F220B930223CDE90D3002924FF016
:1000B000080E4FF4A87211930723CDE90FE21293B3
:1000C0004FF4A0524FF4805307A8CDE905232EF03A
:1000D000CFFA10B10F4830F0C9FB109B0F9A3021B6
:1000E000DB00B3FBF2F3B3FBF1F201FB1232003A97
:1000F0001199B3FBF1F118BF012202A831F034F9D4
:1001000008B10548E7E714B010BD00BF0038024051
:1001100000700040289105083A9105080446DFF870
:100120002CD00B490B4A0C4B03E051F8040B42F85E
:10013000040B9A42F9D300200849094A01E041F82A
:10014000040B9142FBD3204630F0E4BCF8BF012001
:100150003CC8060880040020B4040020B404002039
:100160000410002040F8044B40F8045B40F8046B96
:1001700040F8047B40F8048B40F8049B40F804AB43
:1001800040F804BB40F804CB40F804DB68467047F5
:10019000024B5A690260586100207047B404002085
:1001A000024B5A6912685A61704700BFB4040020BC
:1001B000024B9A69C0E9002198617047B40400209D
:1001C000044A93691968916110B15A68184610473A
:1001D000704700BFB404002038B5054D0446AB6934
:1001E0000BB1A34200D338BD0120FFF7E9FFF6E7CA
:1001F000B4040020C460056146618761C0F81C80BA
:10020000C0F82090C0F824A0C0F828B0C0F82CD0C6
:1002100080ED0C8B80ED0E9B80ED10ABC0F808E0FC
:10022000FFF7B6BF124D6C6908B50CB930F05EFC33
:1002300060602046FFF7D0FF23686B612046C468EA
:10024000056946698769D0F81C80D0F82090D0F8FD
:1002500024A0D0F828B0D0F82CD090ED0C8B90EDE5
:100260000E9B90ED10ABD0F808E00120704700BF66
:10027000B404002010B50021044600F0F9FA18B9C2
:1002800014B120460DF0DEFD10BD002100F0F0BAE3
:1002900010B50121044600F0EBFA18B914B120465C
:1002A0000DF0D0FD10BDFFF7E5BF10B501220C46E3
:1002B00000F002FC18B914B120460DF0C3FD10BDCA
:1002C00000F0FABB00F0BABB2DE9F0432B4C864698
:1002D00000254FF0030CD4F8AC02002101310EEBE5
:1002E00001039A0803F00303825C5B0042FA03F304
:1002F00003F00303022BF1D0D4F8B802090100EB9C
:100300000E108E0889B300EB860603681A0729D100
:10031000D4F8B8125A1AC2F3011E99424FEA921742
:100320004FEA4E0E4FEA12121CD8D4F8BC12994272
:1003300018D9D4F8AC8218F8071041FA0EF303F07C
:1003400003030CFA0EF9012B41EA09010AD104EB6F
:10035000450E3F2D08F807109ABF0135AEF8CC22A4
:10036000C4F8C8320430B042CFD12DB1013D04EB06
:100370004503B3F8CCE2AEE7BDE8F083B404002057
:1003800030B51C4CD4E9AD53C01AC109C0F3021EEC
:100390006B5C012202FA0EF223EA02036B54D4F8DA
:1003A000C02283094FEA101CB2EB901FD4F8AC02B4
:1003B00088BFC4F8C032C15C4FEA9C0E0CF0030346
:1003C00003255B0005FA03F321EA030100F80E1090
:1003D0000CF1010CD4F8AC024FEA9C0E0CF00303B4
:1003E00010F80E105A0041FA02F202F00302022A3B
:1003F000E7D030BDB404002021F00F0138B50B1A4E
:10040000134A144C013BDB00A2FB03235B0A9A0056
:10041000C4E9AB030546C4F8BC120732A1EB831153
:1004200001331D4403EBD202C4F8B8120021C4F812
:10043000B4522AF06BF9002301214FF0FF32C4E9D6
:10044000B033C4E9D4322381A4F84C1338BD00BFC3
:10045000F32C23FAB4040020024A138902331381D7
:10046000704700BFB4040020024A1389023B138185
:10047000704700BFB4040020024B1889003818BF31
:1004800001207047B4040020F8B51C4D2B890022D0
:1004900043F00103C5F8C8222B81C5F8502305F1AC
:1004A000080405F5007654F8043F1A071AD1D5F868
:1004B000B822981AC0F3011193424FEA901C4FEAF8
:1004C00041014FEA10100DD3D5F8BC22934209D256
:1004D000D5F8AC7217F80C2042FA01F303F00303CD
:1004E000012B02D0B442DED1F8BD03238B401A4366
:1004F00007F80C20FFF7E8FEF4E700BFB404002083
:1005000081B3F8B5184E0F46051F002455F8043F77
:100510001A071AD1D6F8B822981AC0F3011C9A42C9
:100520004FEA90114FEA4C0C4FEA10100DD8D6F854
:10053000BC229A4209D9D6F8ACE21EF8012042FA50
:100540000CF303F00303012B03D00134A742DDD1E8
:10055000F8BD032303FA0CF31A430EF80120FFF74A
:10056000B3FEF2E7704700BFB40400202DE9F0436A
:10057000614ED6F8C832D6F8AC1283B0C3B1D6F803
:10058000B03200259800C6F8C85288B10024A308EC
:1005900004F00302CB5C5200134103F00303032B6E
:1005A0001FD001348442F2D3D6F8C832002BEAD1EE
:1005B000D6F8C4324FF000094FEAD3080127D6F825
:1005C000B43213F809504FEAC9043DB304F00303F1
:1005D000E8074FEA94024FEA430314D46D0801344C
:1005E000F4E72046FFF770FED6F8B032D6F8AC122A
:1005F0000134B4EB830F4FEA8300C8D3D6F8C83276
:10060000002BC0D1D4E78A5C42FA03F303F0030362
:10061000012B09D06D0804F10104D7D1C84509F1B7
:10062000010326D09946CAE7D6F8B8C223016A4624
:100630005CF8033040F265310CEB04105BB10CF058
:1006400091FD009B3BB10DF041FEDDE900010DF095
:1006500015FE0DF051FED6F8B402E30804F00701D0
:10066000C25C07FA01F122EA0102C254D6F8AC12C8
:10067000D0E70027BE463A46032402250FE00128B2
:1006800006D104FA03F32CEA03030B704FF0010EBA
:10069000D6F8C43201329A421FD8D6F8AC1290086C
:1006A00002F0030311F800C05B004CFA03F000F005
:1006B0000300022801EB920119D00328DFD105FACB
:1006C00003F32CEA030C81F800C0D6F8C4321746B5
:1006D00001329A424FF0000EDFD93389002223F015
:1006E0000103C6E9B027338103B0BDE8F083BEF152
:1006F000000FEAD0C5E700BFB4040020044B1A89FC
:10070000002142F00102C3F8C8121A81FFF72EBF80
:10071000B4040020554BD3E9AE122DE9F043521A30
:100720000024D3E9AB61C0E90144C0E90344C0E956
:10073000054402604FEA810C22462146A146A646A6
:100740002746254616F809304FEA4E0E43FA0EF3B7
:1007500003F00303012B02F1010255D0022B24D038
:1007600033BB01379445876004F101046DD04FEA33
:10077000920902F0030E16F809804FEA4E0148FA7A
:1007800001F818F002013BD108F0030894452DD080
:10079000B8F1010F04D1C3689C4288BFC460002433
:1007A0004FEA920902F0030ECCE7013545600131B2
:1007B000944541D04FEA920902F0030E16F8093031
:1007C0004FEA4E0843FA08F303F003089B0718D4D6
:1007D00001292CD0022903D143690133436102214D
:1007E00083698B42D2D294458161D1D1C3689C4246
:1007F00000D9C4602D013F01C0E90157BDE8F08375
:10080000194694459ED1F5E701359445456025D0BC
:100810004FEA920902F0030E16F809804FEA4E01E2
:1008200048FA01F818F0020FEAD108F0030803694A
:10083000013303610121D3E701299846F7D002294A
:10084000CAD083699942CED8D0E7C368A342D0D337
:100850002D013F01C0E90157BDE8F0830269013273
:1008600002618269002AC1D18361BFE7B40400201C
:100870002DE9F84300F10F0636093FD06E4C23896D
:10088000E3BBB4F84C230D46E2BBD4F8C002D4F865
:10089000B072B84232D24FF0010ED4F8ACC2013877
:1008A000013F604467440021CCF1010818E04A1C74
:1008B000964255D913F00C0F42D18A1C964240F251
:1008C000AA8013F0300F41D10132964240F2A88045
:1008D0003F2B2ED8511C8E4240F2A780B8420AD03E
:1008E00008EB000910F8013F9A07E0D013F00C0F55
:1008F00021D10122E2E7BEF1000F0FD000231846FC
:10090000BDE8F883D4E9D412914226D2D4F8C002CB
:10091000D4F8B072874288BF9E46BED835F0BEFB81
:10092000D4F8C002D4F8B072B8424FF0010EB4D37C
:10093000E4E70021D2E713F0300F0CD10122C4E725
:1009400003F03002B2FA82F25209C1E73F2B8CBFAA
:1009500000210121C2E70022BAE735F09FFB94E7AE
:100960004FEA8909A9EB0201012A01F1010704D12B
:1009700009F101039B08C4F8C032D4F8C4324B45D6
:1009800038BF4B46B808C4F8C43207F0030E1CF851
:1009900000804FEA4E0E0123023103FA0EF343EAC0
:1009A000080389450CF8003012D34FF0020E880876
:1009B000D4F8ACC201F003031CF800805B000EFA0F
:1009C00003F3013143EA080389450CF80030EED205
:1009D000D4F85033D4F8B8823344C4F8503308EB19
:1009E000071312011846002129F090FEEA074FEA8A
:1009F0000716034683D50022D4F8B40248F806202F
:100A0000F9080122445C07F00707BA402243425428
:100A10001846BDE8F8834FEA890909F10109A1E701
:100A20004FEA890909F102099CE74FEA890909F1AE
:100A300003090A4696E700BFB4040020034B1A8955
:100A4000012A02D808B1FFF79BBC7047B40400200C
:100A5000034610F00F001CD1164AD2F8B812994282
:100A600016D810B4D2F8BC429C420ED95B1AD2F808
:100A7000AC429A09C3F30111A25C49000A4102F099
:100A80000302012A4FEA131305D05DF8044B7047A7
:100A900070470020704701301A18910802F00302D5
:100AA000615C520041FA02F202F00302022AF2D023
:100AB0000001EAE7B40400202DE9F84F0F4606468E
:100AC000002800F0CA80734D2C89002900F0918025
:100AD000002C40F09280D5F8B802D5F8B0C2301A98
:100AE000030903F1010E0F31BEEB8C0F4FEA111118
:100AF0004FEA8C0A80F0B780D5F8AC92A4464FF04C
:100B000001084FEA9E040EF0030B19F804404FEA67
:100B10004B0B44FA0BF404F00304022C2BD02CB939
:100B20000CF1010C0CEB08048C4226D341455CD03F
:100B300065D3C4448C4525D2002A5ED0C209D5F8BD
:100B4000B412895C03F007031941384601F0010132
:100B5000FFF78EFE044600284FD04FEA08123146B8
:100B600029F090FD2B89012B02D83046FFF708FCB5
:100B70002046BDE8F88F08F101080EF1010EF2459C
:100B8000BFD1D3E75C1843449C421FD9980803F0B7
:100B9000030219F8007052004FF0020C01330CFAF6
:100BA00002F23A439C4209F800200FD99808D5F880
:100BB000AC7203F0030217F800E052000CFA02F2E4
:100BC000013342EA0E029C423A54EFD1D5F8C432C6
:100BD000A1EB08029C4238BF1C46120106EB08102C
:100BE0000021C5F8C44229F091FD34462046BDE8F5
:100BF000F88F012C01D8FFF7C3FB0024B8E75C187D
:100C0000A00804F0030719F800E07F004FF0030C80
:100C1000A8EB01010CFA07F72EEA0707012909F8EA
:100C2000007004F1010410D003EB080EA708D5F8FA
:100C3000AC3204F00302D95D52000CFA02F2013426
:100C400021EA02027445DA55F0D1D5F8C032834268
:100C5000CBD9C5F8C0023446C8E701463846BDE8DE
:100C6000F84FFFF705BE0129BFD029B14FF00108A9
:100C7000002A7FF463AFC0E7D5F8AC42800903F0E7
:100C8000030359000322235C8A4023EA020323540E
:100C9000DBE700BFB404002010B58AB0044603A807
:100CA000FFF738FDDDE90430039A0090074920463C
:100CB00000F09EFFDDE9083206980549CDE90020E5
:100CC000079A204600F094FF0AB010BD54E10508D1
:100CD00078E105082DE9F843DFF858914749D9F83C
:100CE000B822074600F084FFD9F8B01289006DD011
:100CF000DFF84481002515F03F0633D005F00306E8
:100D00007600D9F8AC22AB08D35C334103F003037F
:100D1000022B63D0032B5FD0012B4AD1D9F8B82224
:100D20002B01D25842455BD0354B9A425AD0354BB5
:100D30009A425BD0344B9A4256D0344B9A4253D0AD
:100D4000334B9A4254D0334B9A4251D0324B9A4251
:100D500052D0324B9A424DD0314B9A4214BF682246
:100D60004D2227E0A9421ED9D9F8AC022C4602E058
:100D700001348C4208D0A20804F00303825C5B00BB
:100D800042FA03F39B07F3D0621B7F2A0BD9254954
:100D90009209384600F02CFFD9F8B03224F03F0514
:100DA000B5EB830F12D220492A01384600F020FF0C
:100DB000A7E72E221D49384600F01AFFD9F8B032B5
:100DC0000135B5EB830F4FEA830194D338461849B8
:100DD000BDE8F84300F053BB6D22EBE73D22E9E7A5
:100DE0005422E7E74C22E5E75322E3E74422E1E718
:100DF0004122DFE74222DDE74622DBE7C0E10508CA
:100E0000D8200608C0180608B02906088029060858
:100E1000E815060874150608681D0608041E06086D
:100E200044220608DCE10508F8E1050800E20508AF
:100E3000BCE10508B4040020F82A0608064A034667
:100E4000506A1A684168C1F31E018A4202D3521ADD
:100E50001A6070470068F5E7B4040020014441F2CD
:100E60000553884204D398B2012838BF0120704747
:100E700010F8012B03EB43135340F2E7034B044AF2
:100E80005A620022C3F80422704700BFB404002055
:100E9000E85906082DE9F04781460F46002943D05E
:100EA000FFF7DCFF214B5C6A82460CB9204637E035
:100EB00094F90730E668002B06F1FF364FF0000585
:100EC00016DB013604F11808B54215D32468ECE7A7
:100ED00005EB06084FEA580808F106033A4654F8AD
:100EE0002310484629F076FC0028CCBF45464646EC
:100EF000731B012BECD8E4E7236933F815309A45CE
:100F000010D163695B5D9F420CD158F825003A46C9
:100F1000494629F027FC28B96068C0F31E00284420
:100F2000BDE8F0870135CFE70120F9E7B4040020E0
:100F30002DE9F84380460F46FFF7ACFF002840F04C
:100F40009280FF2F03D9494949480CF06FF9494D68
:100F5000D5F804327E1CABB1D5E9821232448A4204
:100F60002CD9024631441846FFF7AAF9D5F80432C5
:100F70000446E0B90246D5F80C121846FFF7A0F96E
:100F8000C5F80442802E344638BF80242046FFF73F
:100F90007CF90346C5F80402B8BB3046FFF775F983
:100FA0000346C5F8040278BB30460CF04BFFD5F879
:100FB00008223244C5F80822002BE3D0D5F80C22D1
:100FC0009C1832444146C5F80C2220463A464FF060
:100FD000000829F057FB04F8078039462046FFF740
:100FE0003DFF8146686AD0E90262B2422BD37600A7
:100FF0000A2E38BF0A26C6EBC6001830FFF745F99F
:1010000048B9C5F80402CFE734460022C5F80842C3
:10101000C5F80C22D2E700F1180202EB8602696AD9
:10102000026102EB460242614A680160C968C0F889
:101030000C80C2F31E020A44416862F31E01C0E93B
:101040000116424668620169436921F812909F5473
:10105000911D6B6A43F82140D96858680131C0F38B
:101060001E00D9601044BDE8F88300BF4E9105080A
:101070005C1A0608B404002010B5044629F084FB6D
:1010800001462046BDE81040FFF752BF07B501906A
:1010900001A8FFF7D3FE019A036933F8120003B0E9
:1010A0005DF804FB07B5019001A8FFF7C7FE019B9F
:1010B0004269D05C03B05DF804FB07B5019001A85C
:1010C000FFF7BCFE019B063350F8230003B05DF828
:1010D00004FB13B5019001A80C46FFF7AFFE019B7E
:1010E0004269D25C2260063350F8230002B010BD82
:1010F0002DE9F8431D46002303600B6013602B604D
:10110000164BDFF85C905C6A07468846164664B961
:101110002B68326813442B60BDE8F883336812F8FB
:10112000010B0133034433600DE04C45F0D03B68C4
:1011300001333B60E268D8F800301344C8F800304F
:101140006269E368D1188A42E8D32046FFF780FC41
:101150002B68246803442B60D9E700BFB404002047
:10116000E8590608F8B50B4B0B4F5C6A0CB1BC4252
:1011700000D1F8BDE36804F1180505EB8306B5421C
:1011800001D32468F2E755F8042B0449044800F021
:101190002FFDF4E7B4040020E85906085391050830
:1011A000C808060830B50023202511F8012F0AB918
:1011B000027030BD120600F1010420D513B12023C6
:1011C000037020460B78124A03F07F036BB9013A93
:1011D00012F8013F13F0800F044600F101000BD01C
:1011E00003F07F0323700123DFE712F9014B002C8A
:1011F000FBDA013BDBB2E9E700F8013CE8E7012B51
:1012000004BF057020460B7800F8013B0223CCE7B1
:101210005A91050838B54368194403689942054650
:1012200010D9037B1BB1084800210BF0FFFF01F12F
:10123000100424F00704083480682146FFF735F8CD
:101240002C60A86038BD00BF5C1A060870B5044663
:101250000E4611461546FFF7DDFFD4E901302A4658
:101260001844314629F03EFA63682B44636070BD30
:1012700038B50129044638BF012100250846216000
:101280006560FEF7F7FF2573A06038BD38B50546E9
:101290000C460131FFF7ECFF6C6038BD0023C0E95C
:1012A00001320123016003737047000038B5144612
:1012B0000546FFF7DDFF024B2560636038BD00BFC8
:1012C0004D120208037B10B5044613B98068FEF77F
:1012D000F9FF0023A36010BD38B505461020FEF7C6
:1012E000C9FF29460446FFF7C3FF204638BD10B5A5
:1012F000044648B1037B13B98068FEF7E3FF20463C
:10130000BDE81040FEF7DEBF10BD000038B5037B1E
:1013100004460D461BB1074800210BF087FF01680A
:1013200080682944FEF7C1FF2368A0601D44256042
:10133000184438BD5C1A060838B504460D46FFF758
:1013400069FFD4E901301D446560184438BDD0E917
:1013500000239A4210B5044602D10121FFF7D6FFBF
:10136000D4E901320021D154A06810BD10B50C465B
:101370000121FFF7E1FF047010BD7F29F8B50C468D
:10138000CEB204D80121FFF7D7FF0670F8BD06F0F2
:101390003F06B1F5006FC1F3871546F0800607D20E
:1013A0000221FFF7C9FF65F03F0505704670EDE7C4
:1013B00005F03F05B1F5803FC1F3073745F08005E3
:1013C00008D20321FFF7B8FF67F01F0707704570C9
:1013D0008670DBE70421FFF7AFFFA40C07F03F079F
:1013E00064F00F0467F07F07047047708570C67063
:1013F000CCE738B5054608460C4629F0C5F9214624
:1014000002462846BDE83840FFF720BFF8B54768D8
:10141000B942044628BF39460D4611461646FFF725
:10142000F9FEA368A81959197A1B184429F05AF92A
:101430006368A068334463602844F8BD43688B4206
:101440002CBF591A00214160704738B50446154633
:1014500062688A42084603D929448A4201D86060FA
:1014600038BDA368521A1844194429F03BF963683F
:101470005B1B6360F4E7084611462AF0CFB870B5ED
:10148000054608460E4629F07FF9044620B102467B
:101490006B68286831469847204670BD2DE9F74FA4
:1014A0008A469DF8301091460D9A11F0DF0F0746DD
:1014B000A2EB090552D0302954D1C3F347210029AA
:1014C00054D05F290CBF0526042692FBF6F106FBDB
:1014D00011210CBF2A482B4809B901350132711E70
:1014E00092FBF6F406FB14228A1A00EB020813F0B2
:1014F00020023ED005EBD573A5EB63045D10002DF3
:101500003BDDAB465E4532467B683868A8BF5A462D
:10151000414601929847019AABEB020BBBF1000FD9
:10152000F0DCB9F1000F05D07B6838684A465146B7
:1015300098474D44002C0DDD2544A642B146A8BF76
:10154000A1467B6838684A464146A4EB090498479F
:10155000002CF2DC284603B0BDE8F08FDFF82880CD
:101560001026C4E70DF130080126C0E7DFF81C8023
:10157000F6E713F00104C2D02C460025D1E700BFE6
:10158000DC080608E1080608E7080608D00806088F
:101590002DE9F04F93B09246CA07DDE91E761C9CF8
:1015A0009DF87490059380460D460BD48B0703D1AC
:1015B00009687C4B994205D028460DF0F1FC4500A6
:1015C00045F0010514F0210306D1B9F1300F03D124
:1015D000B742B8BF37461E46284610F00AFF00281B
:1015E0000DF1280B1CDBA00716D52B238DF8283016
:1015F0000DF1290322079DF814101FD5BAF1020F2F
:1016000010D118464FF0300C00F802CB01F1010C5C
:1016100083F801C0034611E0610701D52023E5E707
:101620005B46E7E7BAF1080F5BD13020187020065F
:1016300045BF01F10E0058700133023300200EAA9D
:101640001870012EA3EB0B030B924FF010020693C0
:10165000C4F34723C8BF1443CDE90C2014F0100293
:10166000CDE902138DF82700059245D0CDE900A001
:101670002B460DAA0CA90BA810F07EFD03782D2B8C
:10168000824606D18DF827300D9B013B00F1010AFF
:101690000D93012E7ADD0D9D059BB542B8BF3546F1
:1016A0002BB19DF8273003B10135069B1D4424F072
:1016B0000103AF42079371DD14F00109A7EB0505A3
:1016C0006DD120230195009337494B464A46404649
:1016D000FFF7E4FE4D460446059B4FF03009C3B9C1
:1016E00036E0BAF1100FA9D118464FF0300C00F8CF
:1016F00002CB01F1170C8BE70AABCDE900A30DAAD1
:101700002B460CA90BA810F037FD8246C1E7002537
:101710002C469DF8273053B100230122CDE9003239
:101720000DF127014046FFF7B9FE013F0444069B37
:101730005BB100230122CDE900325946069A4046AA
:10174000FFF7ACFE069B0444FF1A012ED8BF3E46AD
:10175000CDE90096079B0D9A51464046FFF79EFE45
:1017600004444DB12023009300230F4901951A46EC
:101770004046FFF793FE04440B980EAB984201D00D
:10178000FEF7A0FD204613B0BDE8F08F059B07943F
:10179000002BBCD11D461C463E46D9E7002500243F
:1017A0009AE700BFC01F06082CD805082DE9F043B2
:1017B00007469007984658BFC2F380038DB05ABFC2
:1017C0005B01DBB22B23164600930A46159BDDF81E
:1017D0005090212103A80AF071FCF20504461FD5A0
:1017E0002E2103A829F016F8D0B9652103A829F005
:1017F00011F8A8B96E2103A829F00CF880B9631C70
:1018000004F130026A4430336B442E2102F8241C68
:101810000234302203F8242CA3186B4403F8240C60
:1018200073060ED504F13002631C0DEB0204252271
:1018300004F8242C03F130026A44002102F8241C2D
:101840001C4616F010051DD09DF80C302F2B4FF0C4
:10185000000319D8012203A9CDE900323846FFF769
:101860001DFE09F1FF390546013C0DF10D01CDE9E1
:101870000089334622463846FFF710FE28440DB053
:10188000BDE8F08303A9F2E703A91D46EFE70000D6
:101890002DE9F04F81468BB014464FF000080B46FF
:1018A0001D4613F8012B0AB1252AF9D1A94208D205
:1018B0006E1AD9F80430D9F8000032469847B0447F
:1018C00029460B78002B00F08B8120234A1C0393C0
:1018D0000027134613F8016B3EB12D2E25D01ED8DC
:1018E000202E29D02B2E24D00026154612F8013B9D
:1018F000A3F13001092922D92E2B4CD16B782A2B48
:1019000023D00023154612F8011BA1F1300009284D
:101910001ED80A2000FB031BABF13003F2E7302E88
:10192000E2D147F01007039601E047F001071A469D
:10193000CFE747F00207FAE747F00407F7E70A2185
:1019400001FB0633A3F13006CFE754F8043B023520
:1019500023EAE37B2B786C2B08BF013595F800A0B8
:10196000BAF1000F00F03C81BAF1780F09D8BAF152
:10197000570F13D8BAF1470F5AD8BAF1440F00F2F3
:101980001D81D9F80430D9F8000001222946984772
:1019900008F1010885E04FF0FF3BDBE7AAF15803AF
:1019A000202BEED801A252F823F000BF371A02080C
:1019B000831902088319020883190208831902088F
:1019C000831902088319020883190208831902087F
:1019D00083190208891A0208B31A0208371A020882
:1019E000BD1B0208BD1B0208BD1B020883190208AB
:1019F000831902088319020883190208831902084F
:101A0000831902088319020883190208371A020889
:101A1000C91A020883190208F11A02088319020878
:101A2000371A02088319020883190208371A0208B4
:101A3000BAF1500FA5D154F8040B0AF0DF03502B74
:101A4000014667D1BAF1640F6AD1002880F29D8007
:101A50002D238DF8173041420A2251230DF1280A17
:101A60000A3B0DF1180BB1FBF2FC02FB1C1009281C
:101A70008CBFC01830300AF8010DDA458E46614639
:101A80005DD07245EFD95AE054F8043B019653B14A
:101A9000039B5549009304223B464846FFF7FEFC52
:101AA0008044691CFBE6039B009350493B4605229A
:101AB000F3E754F8043B8DF81830039B009301962C
:101AC0003B46012206A9E8E706A954F8040BFFF7F4
:101AD00000FBBBF1FF3F014604D0069B9B4538BF8E
:101AE000CDF818B0039B0093069A01963B46D4E7C5
:101AF00054F804AB504628F047FEBBF1FF3F0246C6
:101B000002D0584528BF5A46039B009301963B4696
:101B10005146C2E7BAF1640F97D0BAF1750F2ED0D3
:101B20002AF00F0300220F3B8DF81720DBB21022A2
:101B3000002893D130238DF827300DF1270A17F0B4
:101B4000100B9DF817302DD0002B35D0039B009340
:101B5000012201923B460DF117014846FFF79EFC1A
:101B6000013E8346039B00930AAA01963B46A2EBE3
:101B70000A0251464846FFF791FC584490E700237B
:101B80008DF817300A226123D2E7BB0705D52B2336
:101B90008DF817300A225123CAE7C7F380035B018F
:101BA000DBB2F5E7002BDDD006AA9245DAD90AF8B8
:101BB000013C0AF1FF3AD5E79B46D3E7073424F00E
:101BC0000704F4E8020137F07BF8CDE9006B00EE82
:101BD000100A039B3A4651464846FFF7E7FD5FE788
:101BE00040460BB0BDE8F08FA8BA0508ADBA0508AD
:101BF0000EB403B503AA52F8041B0192FFF748FE86
:101C000002B05DF804EB03B070470346007893F927
:101C10000020002A0ADA00F07F004022104206D19C
:101C200013F8012F02F0C001802904D0704720EA88
:101C300002005208F2E702F03F0242EA8010EFE7AA
:101C4000431C18460133027802F0C002802AF8D003
:101C5000704703460020994200D8704711F8012DC3
:101C600002F0C002802A18BF0130F4E703460144A5
:101C7000002099421A4600D87047127802F0C0023C
:101C8000802A03F1010318BF0130F2E77F289DBFCE
:101C9000024B185CC0F3400000207047F7080608AC
:101CA0007F289DBF024B185CC0F3C0000020704726
:101CB000F70806087F289DBF024B185CC0F3800020
:101CC00000207047F70806087F289DBF024B185C6C
:101CD000C0F3801000207047F70806087F2809D855
:101CE000064B1B5C13F00C0F06D1A0F15F035842AA
:101CF000584170470020704701207047F7080608D8
:101D00007F289DBF024B185CC0F300100020704775
:101D1000F70806087F289DBF024B185CC0F34010EF
:101D200000207047F708060808B50246FFF7E8FFED
:101D300002EB401008BD08B50246FFF7EBFF40423A
:101D400020F01F00104408BD3038092884BF20F05F
:101D500020000738704710B502460144E5240020F2
:101D6000914203D8B0FA80F0400917E012F8013B25
:101D700030B103F0C003802B11D10138C0B2EFE7BE
:101D8000BF2B09D9F72B09D8DB0803F0060344FA67
:101D900003F303F00300E3E71B06E1D510BD0020C9
:101DA000FCE7023981420B4603D31A880239002A24
:101DB000F8D00233181A40107047B2EB131F70B5F9
:101DC00004464FEA131019D901EB4001101A03F031
:101DD0000F0302462646012A0CBF0D880D68013A02
:101DE00025FA03F526F8025B01F10201F3D104EBB9
:101DF000400434F8023C03B9013870BD0020FCE710
:101E0000F0B5059C0025121B2E46AC420FD101EB0C
:101E10004403174600EB4404411A9FB904EB420304
:101E200016B124F812600233181A4010F0BD31F8D0
:101E3000157033F815C067443E4420F81560360C21
:101E40000135E2E71D8835445D522E0C013F023317
:101E5000E3E7F0B4049F00260D463446D11BB74299
:101E60000BD105EB47030A4600EB4707451B7AB940
:101E700007EB4101F0BCFFF794BF35F816C033F80B
:101E800016206444A41A20F8164024140136E6E70C
:101E90001E8834445C53013A24140233E7E72DE9E9
:101EA000F043079CDDF828E0DDE9087602391546A5
:101EB00084464FF6FF78A4EB020955B900EB4201C6
:101EC0001FB1012320F812300231BDE8F043FFF7C3
:101ED00068BF31F8024F013D4444264405EB090434
:101EE000A5422ABF33F8024B4FF6FF7444447444B2
:101EF00086EA040E17FA8EF72CF8027B4FEA144E8E
:101F0000360C3F0CD9E738B502290446806838BF43
:101F100002210D4618B12368B1EB930F07D9690070
:101F2000FEF7C3F92368A06065F39F03236038BD03
:101F300038B504460C20FEF79DF923682278054643
:101F400002F00102C3F39D0023F0030313432B604F
:101F500063686B604000FEF78DF9A8602268A16895
:101F6000C2F39D02520028F08DFB284638BD9942ED
:101F700010B511D313D800EB410002EB410209B9AF
:101F8000084610BD30F8023D32F8024D1B1B002BF5
:101F900002DB04D10139F2E74FF0FF30F1E7012015
:101FA000EFE710B5044638B18068FEF78BF920469C
:101FB000BDE81040FEF786B910BD70B505460C4669
:101FC0000221FFF7A0FF002C2B78B4BF01220022D2
:101FD00062F30003AA682B70B4BF6142214601235B
:101FE00088B2090C14461E4622F8020B03F10103C5
:101FF000F6D16E60208070BD0023C0E9003383609D
:10200000704728B103789B0702D48068FEF75AB95D
:10201000704738B504460D464968FFF774FF2A78C3
:102020002378A06862F3000323706A686260A9687D
:102030005200BDE8384028F025BB0A4629B901788E
:10204000426062F3000101707047FFF7B6BF08B548
:10205000FFF7D2FFBDE80840FFF7EFBF920042F064
:10206000020210B402600022C0E901215DF8044BB5
:102070001946FFF7E2BFF8B59DF8187014461D46E3
:1020800004210646FFF73FFF22462B4627B1002DCD
:102090000CDA624265EB4503317867F30001317079
:1020A0000021716052EA030102D1F8BD0027F3E775
:1020B000D6E901104C1C746020F81120120C42EA81
:1020C00003421B0CEEE72DE9F3418DED010A019D62
:1020D0000378EA0F62F300030370C5F30F4313F4B0
:1020E000FF4380460BD198F8003023F0010388F8B5
:1020F00000300023C8F8043002B0BDE8F081B3F529
:10210000FF4FF0D0C5F3C754A4F17F06002EEADBE1
:1021100005D1012102B0BDE8F041FFF74EBF162EF8
:10212000C5F31605A4F16F07D8BFC6F1170645F42D
:1021300000054FEA2717D5BFF540963C0026093623
:10214000D4BF344624113946C8BF06F00F06FFF746
:10215000DAFEC8F804702CB1D8F80800620000213B
:1021600028F0D4FA4EB1D8F8083005FA06F223F870
:102170001420C6F11006F5400134A742BCD0D8F8AF
:10218000083023F814502D0CF6E72DE9F8430446E7
:102190008F18C2F35B020D46511C9846089EFFF74C
:1021A000B2FE237868F300032370AC4600221FFAC6
:1021B00086FEBC456046626002D3401BBDE8F883E2
:1021C0000178A1F13003092B0CF1010C05D9A1F123
:1021D0004103192B12D8A1F13703B342EDD2A06805
:1021E00090468146B8F1000F0FD100EB420113B1C8
:1021F00020F812300231091A4A10DAE7A1F161031E
:10220000192BDAD8A1F15703E7E7B9F800100EFB54
:10221000013329F8023B08F1FF381B0CE2E7F8B55F
:10222000044615461E46C1B1531E1E444FF0FF37EB
:10223000E9000F3109092046FFF765FE23780021E8
:1022400023F00103237061600B4645B9A06800EBE1
:102250004101FFF7A6FD6060F8BD0127E8E7002215
:102260000F2B08DC307898400243013D92B203F115
:1022700008033E44F4D1A068013100EB41006160E5
:10228000103B20F8022CE0E738B505780B7805F014
:10229000010203F001030446981A08D1D1E9013282
:1022A000D4E90110FFF763FEEB0748BF404238BD99
:1022B000884210B5044601D0FFF7ABFE237823F027
:1022C0000103237010BD884210B5044601D0FFF70A
:1022D000A0FE63683BB12378C3F3000282F00102E1
:1022E00062F30003237010BD88421FB5044601D07D
:1022F000FFF78FFE626862B901212046FFF703FEF7
:10230000A268012313806360237843F001032370E4
:1023100010E02378D9070FD523F0010323700123A0
:102320000093A168ADF80E3008460DF10E03FFF7DB
:1023300090FD606004B010BD511C2046FFF7E3FD26
:1023400001230093D4E90121ADF80E3008460DF1C8
:102350000E03FFF755FD6060D6E74B682DE9F047A7
:1023600005460E46144603B12AB931462846BDE853
:10237000F047FFF74EBE02F10F014FEA111803EBD1
:102380001111FFF7C0FDD6E9012308EB0207A96888
:1023900007F1004014F00F0400F1FF3008BF1024D3
:1023A0004FEA400901EB400003EB42031146864629
:1023B0004FF0000CC4F1100409BB6FF001035A4345
:1023C00083182CFA04FCC8F1010820F802C003EBC2
:1023D00048034FEA48021846524228F097F909F19B
:1023E000020903464B4417B133F8022D9AB16F60CE
:1023F00032782B7862F300032B70BDE8F08733F856
:1024000002AD4AEA0C0C2CFA04FA2EF802A94FEAA3
:102410000C4C0139D0E7013FE5E72DE9FF410D46BE
:1024200049680646144601B132B92946304604B01F
:10243000BDE8F041FFF7EDBDFFF765FDB768D5F8E2
:1024400008806A68234641463846FFF7B6FC70604C
:102450002978337861F300033370DB0702460AD52D
:1024600000236968ADF80E302009994201D08342FB
:1024700004D181420AD804B0BDE8F08138F8135085
:102480009DB101238142ADF80E3012D904F00F0442
:10249000012338F8101003FA04F4013C214206D15C
:1024A000BDF80E30002BE6D003E00133DDE7ADF8D8
:1024B0000E30012312B93B807360DCE7009339468C
:1024C0000DF10E033846FFF79BFC7060D3E72DE952
:1024D000F3410D465768D1F804803B461446064642
:1024E0009268A8684146FFF742FD01301EBF2346AF
:1024F0002C461D4623782A7883EA020318BF4746F4
:10250000DB0719D4791C3046FFF7FDFC6B6800939C
:10251000D4E90121AB68B068FFF772FC70602378E2
:10252000327800280CBF002303F0010363F300029C
:10253000327002B0BDE8F08139463046FFF7E3FC67
:102540006B680093D4E90121AB68B068FFF781FCA8
:10255000E4E72DE9F3410F464E68D2F804801446B3
:102560004346314692680546B868FFF700FD0130E2
:102570001EBF23463C461F4623783A7883EA02036F
:1025800016BFB04601260026DB0719D508F1010168
:102590002846FFF7B8FC7B680093D4E90121BB68AB
:1025A000A868FFF72DFC686018B1207800F00100E2
:1025B00070402B7860F300032B7002B0BDE8F0810F
:1025C00041462846FFF79FFC7B680093D4E9012130
:1025D000BB68A868FFF73DFCE5E74B682DE9F04FC5
:1025E0000C4651688B42154621BF254619461346B5
:1025F0001C462B78DB0785B0064622D4237813F0DF
:1026000001071ED1FFF77FFCD4E9011CB068AD685B
:102610003B4699420CD100EB4101FFF7C2FB00237E
:102620007060327863F30002327005B0BDE8F08F5D
:1026300035F813203CF81340224020F813200133D2
:10264000E7E701313046FFF75EFC2F782378D5F8B5
:1026500004C0B068A26887EA0301C94301F0010E13
:1026600041F3000189B207F0010947F30007029125
:10267000B9B20191A968A1F10208616803F0010AE9
:1026800043F300039BB2A1EB0C0100936746834622
:1026900003918FB900EB4C01BEF1000F03D0012371
:1026A00020F81C300231FFF77CFB706022782B7819
:1026B000C2F300021340B4E738F8021F019B5940EF
:1026C000039B013F8944D9198F4225BF32F8021B71
:1026D000009B009959408A44029B09EA0A0159402B
:1026E0001EFA81F12BF8021B4FEA1A4A4FEA1949E8
:1026F0004FEA114ECDE72DE9F84F4B680D46516872
:102700008B42144621BF2C46194613461D4623789A
:10271000DB07064631D42B7813F001072DD1FFF7E4
:10272000F2FBD5E9012EA0686468D6F808C0A41AA7
:102730003B469A4213D10CEB4203214600EB420286
:10274000ACEB0000A1B903EB4403A3EB0C0358105E
:102750003378706061F300033370BDE8F88F30F8B0
:1027600013103EF8135029432CF813100133E0E7FF
:102770001588155201390232E4E701313046FFF77E
:10278000C2FB27782B786168B068A468D5E901E2BC
:1027900003F0010947F3000543F3000307F00108C4
:1027A000ADB29BB2A4F1020C0F4683464FF0010A72
:1027B000AEEB010E2FB900EB4101FFF7F2FA012158
:1027C000C6E73CF8024F013F6C40A0440EEB070403
:1027D000A7422ABF32F8024B1C465C40A14448EA9B
:1027E0000904E4431AFA84F42BF8024B4FEA19491E
:1027F0004FEA18484FEA144ADCE74B68F0B50D463B
:1028000051688B4224BF19461346144624BF2C46F8
:102810001D4627782B785F4017F0010785B00646E4
:1028200036D1FFF770FBD4E901212478B06814F0A9
:102830000104D5E9015324D1521BA54212D101EB69
:102840004503144600EB4505411AACB905EB4201BE
:10285000FFF7A7FA00273378706067F3000333703F
:1028600005B0F0BD31F8147033F814C087EA0C07D6
:1028700020F814700134E0E71F885F52013C0233F6
:10288000E3E7CDE90277CDE90057FFF708FBE1E781
:102890000131FFF738FB2B78DB4303F0010303938F
:1028A0002378DB4303F001030127029301976B6850
:1028B0000093D4E90121AB68B068FFF7F0FACAE7EA
:1028C0002DE9F04F4B6885B004460E4615460BB116
:1028D000536843B9237823F0010323700023636016
:1028E00005B0BDE8F08F81422DD1FFF721FBA54255
:1028F000064607462ED06B68716820461944FFF7DC
:1029000002FB2268A068C2F39D025200002127F05A
:10291000FDFEB368D4F808E0D6F804900193AB68E4
:10292000029300226B6803930EEB4908F4461146AC
:10293000039B934233D0DDF804B0CDF80090ACF1A6
:10294000020000231AE0824206D1FFF7F1FA0546A1
:102950000746D0E70546CEE70027CCE730F802AFC0
:1029600053441946029B3BF802AB33F8123003FB89
:102970000A130099038001391B0C0091009900296A
:10298000ECD14146881C13B1A8F800300146A1EBF8
:102990000E0149100CF1020C01328046C8E761605B
:1029A0002A78337853402278384663F30002227045
:1029B00005B0BDE8F04FFFF7F4BA4B6870B50546B7
:1029C000144613B11378DA0706D52B7823F00103E8
:1029D0002B7000236B6070BD636823B9BDE8704045
:1029E0000121FFF7EABA0846FFF7A2FA0646204699
:1029F000FFF79EFA012104462846FFF7DEFA6368D6
:102A000083B1A3681B88DB0704D5324629462846D4
:102A1000FFF756FFD4E9012101230846FFF7CDF95E
:102A2000606038B93046FFF7BCFA2046BDE8704018
:102A3000FFF7B7BA324631463046FFF741FFDEE7CF
:102A40002DE9F04F0C4651688FB093460131054691
:102A50000393FFF758FADBF80420A868013252000C
:102A6000002127F053FE2B78002623F001032B7062
:102A70006E60DBF8041020460131FFF744FA594636
:102A80002046FFF7C6FA039BD4F80890D4F80480D8
:102A9000D3E901370293AB6804933A46029B41465F
:102AA0004846FFF764FA002833D1049A6060012396
:102AB00013806B6023786268002A0CBF002103F04A
:102AC000010161F30003039923709BF8003009783A
:102AD0004B40DB0740F1FD806B682978003B18BF55
:102AE000012363F300012970002A00F0F2800BA893
:102AF0004FF0FF31FFF7ABFA0BAA29462846FFF744
:102B0000E6FC039A214620460FB0BDE8F04FFFF7E0
:102B1000DEBC013001D16E60CCE7029B03F10042C4
:102B2000013A4FEA420A37F8121033460E0403F115
:102B300001004ED59BB209EB48014FF0000C08F1A3
:102B40000100C3F1100629F818C00191606002313C
:102B5000CE4605968E4540D337F812209A4005920E
:102B6000029A012A09D907EB0A02C3F1100132F8CF
:102B7000022CCA40059911430591029A801A686097
:102B8000049A00F10040013802EB400207920AF17A
:102B900002020992BA1E0892D4F804A0029A524581
:102BA00029D30AF1004A0AF1FF3A09EB4A0A002246
:102BB000C3F11000D14573D96FF000416B682BB1A0
:102BC00004985A1830F81220002A73D06FF0004190
:102BD00075E0490089B20346A8E7BEF8008008FA0C
:102BE00003F64CEA060C059E2EF802CB28FA06F8EE
:102BF0001FFA88FCAEE7019A0198118832F8022C7E
:102C000042EA01420599B2FBF1F20999411A069193
:102C10000899069F00200E4686460199B9420DD8B4
:102C200009880844A8BB079921F80229019A07914D
:102C3000023A01920AF1FF326260ADE736F8021FF4
:102C4000B7F80080994041EA1E4E1FFA8EF15143B9
:102C500018FA80F81FFA81FC090CA8EB0C0CC1EBE8
:102C6000204127F802CB01EB2C40D6E738F8021FB1
:102C7000994041EA1E4EBCF80010394411FA8EF119
:102C80002CF8021B0F0C01996145EFD83844013A2A
:102C9000C8E70027DDF82080DDF818C0BE46F2E75F
:102CA000BAF8001041FA03F6324381402AF80229AB
:102CB0008AB27FE7013B6B6080E7013B636063683A
:102CC000002B3FF4F7AE5A1839F81220002AF4D03E
:102CD000F0E60FB0BDE8F08FF0B51F464B6885B049
:102CE00004460D4616464BB11378DA0706D47B68C6
:102CF000012B0BD1BB681B88012B07D1237823F054
:102D0000010323700023636005B0F0BD012120465C
:102D1000FFF753F97368002BF6D02846FFF708F940
:102D200005463046FFF704F90023CDE90133064696
:102D300003937368B3B1B3681B88DB070AD52A46CF
:102D400021462046FFF7BCFD3B462246214601A80E
:102D5000FFF776FED6E9012101230846FFF72DF89B
:102D6000706058B901A8FFF74CF92846FFF719F928
:102D7000304605B0BDE8F040FFF713B92A462946B2
:102D80002846FFF79DFD3B462A46294601A8FFF746
:102D900057FECEE710B5D0E90121034601EB420210
:102DA0000020914204D31B78DB0748BF404210BD8E
:102DB00032F8024D44EA0040F3E730B5D0E901248F
:102DC000002304EB4202944206D30278D20748BFA4
:102DD0005B420B60012030BDB3F5004F04D232F8E6
:102DE000025D45EA0343EEE70020F4E7037813F0C1
:102DF000010310B510D1D0E9012404EB4202944242
:102E000002D30B60012010BDB3F5803F04D232F82D
:102E1000020D40EA0343F2E70020F4E72DE9F74F03
:102E2000DDF830C0019206460F4609B30CEB0300F3
:102E3000D6E90189012400211A46A2468E46B8F13E
:102E4000000F17D10199002945D0002A43D1002B4A
:102E500041D0002F3BD09CF800302CB13478DB43BC
:102E600084EAD31404F00104204603B0BDE8F08FD7
:102E70006046DDE739F8025B0EF1100E45EA0141CC
:102E8000BEF1070F02DC08F1FF38D8E796F800B072
:102E90008DB21BF0010F1FBFED435AFA85FA1FFADE
:102EA0008AF5CAF3072A42B91CB1EDB2B5FA85F426
:102EB0006409AEF1080E090AE2E7EDB227B100F8A5
:102EC000015C0138013AF4E700F8015BFAE763447A
:102ED00013F8013CC1E7337813F0010F14BFFF2151
:102EE0000021002F18BF604627F010FCBCE700004F
:102EF000D0E901329FED0C0A9FED0C7A02EB4303FF
:102F00009A4205D30378DB0748BFB1EE400A704709
:102F100033F8021D07EE901AF8EEE77AE0EE077A32
:102F2000B0EE670AECE700BF000000000000804739
:102F30002DE9F74F0A2944689DF830A00D9E1546EB
:102F400014BF04220322804689460092A4B98DB1A1
:102F5000013D324615F8011F134641B930221A705F
:102F6000002203F8012F981B03B0BDE8F08F02F890
:102F7000011BEFE73346F1E7640020460193FDF7BC
:102F800079F9D8F808102246074627F07BFB019B09
:102F90003046B34607EB040C3A3BACF10204002187
:102FA000A742A6461DD9303139295C4688BFC918C9
:102FB00004F8011B39468C458E461DD83846FDF76E
:102FC00081F965BB98F80030DB0744BF2D2304F876
:102FD000013B3346621E9A4233D800232370A01B64
:102FE000C2E7BEF800E04EEA014EBEFBF9F124F85C
:102FF000021909FB11E1D3E7BEF800200231002AD3
:10300000D9D0BAF1000F08D0009A211A914204D108
:103010000BF102048BF801A02046A346BDE7284629
:1030200027F0B2FB29185A460B46AB4204D88D4212
:1030300088BF00200444C5E713F8017D02F8017F32
:10304000F3E71978107803F8010B02F80119C2E7C9
:10305000D0E9023293423DBF5A1C826018784FF08B
:10306000FF3070470368013B033310B5044602D8B4
:103070004068FDF727F92046BDE81040FDF722B96A
:10308000F8B5054610200C461F461646FDF7F2F827
:10309000054B8460C0E900743444C4606B60034B2A
:1030A0002860AB60F8BD00BF5130020865300208EF
:1030B00002690A2AF8B504461BD18369013383618A
:1030C0000123E361237D2361637D237500260A27A5
:1030D000256EB5B16B1CA26D2366555D626D934282
:1030E00001D366652666237D0D2B14D0BDB16575B1
:1030F000F8BDC369092A04BF073323F0070301336E
:10310000DFE7D4E901039847431CECD0012838BF1E
:1031100001200546E7E70A2D2775D9D0E6E7237D8C
:10312000002BE4D00A2B18BF0A25E0E70169272904
:10313000024601D0222912D1012024E0137D272B41
:10314000FAD0222BF8D0722914D1662B16D1507DDB
:103150002728F1D0A0F12203584258417047A1F12D
:103160006200132804D8084B034113F00100E5D096
:1031700000207047662904D1722B00E0622B02D137
:10318000E5E76229F8D07047EEFFF6FF38B5044650
:103190000D462069D0B10A2806D10DB1636AB3B1DA
:1031A0002046FFF785FFF4E7FEF770FD0028F7D112
:1031B0002369232B08D12046FFF77AFF2369002BD0
:1031C000E7D00A2BF7D1E4E75C2B02D00025284694
:1031D00038BD237D0A2BF9D12046FFF769FFDFE7D1
:1031E0002DE9F04F0023044685B001214364FFF729
:1031F000CDFF276AA3696363002FE369A36307DA3E
:10320000072384F83C300137276205B0BDE8F08F12
:1032100004D0062384F83C30013FF5E7002835D080
:1032200039462046FFF7B2FF052384F83C30D4E945
:103230000B3003F10042013AE56930F81220013DFC
:103240009542E2D009D8013B30F81320954218D3BB
:10325000DBD0022384F83C30D7E7A16A8B4207D346
:1032600008314900FDF721F8A36A20630833A362FF
:10327000E36A5A1CE26220F81350236A0133236286
:10328000C3E7226AE362013A2262DCE7256915B9E5
:1032900084F83C50B9E72046FFF748FF064600286F
:1032A00000F00C8284F83C702369722B6CD008D833
:1032B000622B0CD0662B71D0B9460025A8460B2393
:1032C0000EE0753BD3F1000949EB0309F5E7237DD7
:1032D000722B4FF0000569D0A8464FF001090C236E
:1032E00094F83C20002A6AD184F83C30B9F1000FF0
:1032F00008D02046FFF7DCFEB9F1020F02D12046CC
:10330000FFF7D6FE2369222B0CBF2223272320465A
:103310000193FFF7CDFE2369019A934240F0868026
:10332000237D934240F082802046FFF7C1FE204675
:10333000FFF7BEFE4FF0030935B1A36E23B9A649CE
:1033400004F16400FEF755F804F140034FF0000B60
:1033500002932169002900F0A881B9F1010F02D17F
:103360000A2900F0A281CB4563D3594604F14000FD
:10337000FEF764F801212046FFF708FF2046FFF71B
:10338000D5FE002890D11CE0237D622B0DD0662B4A
:1033900010D00025B0464FF0010990E7237D722B35
:1033A000354608D04FF00008F5E70025B0464FF04D
:1033B000020994E73546B0464FF002097FE79A428A
:1033C00094D0A36E002B3FF420AF292104F16400B8
:1033D000FDF7CCFF236E04F15006002B40F06B810B
:1033E00003213046FDF7A8FF23690370237D437056
:1033F000637D8370D4E91A57216E2A463046FEF762
:1034000005F82A46394627F03DF90023A366236EC6
:10341000A26D581C2066D15C2161991C2166105C4C
:10342000207503332366535C6375EEE64FF00109A4
:1034300082E7019B8B4209D1029819460BF1010BDF
:10344000FDF79BFF2046FFF733FE82E7002D60D19A
:103450005C2940F0278120460391FFF729FED4F82C
:1034600010A00399B8F1000F6CD00298FDF785FF0A
:10347000D346D2E004F1640B28215846FDF776FFCD
:10348000D4F868A00022216979B172BB3A290CD026
:103490007D290AD0212928D1207D7238012829D8F8
:1034A000607D3A2801D07D2824D1D4E91A218818DA
:1034B00010F8010C3D2809D1A2EB0A02514404F195
:1034C0004000FDF7C3FEA26E013AA266924508BF16
:1034D0000423584608BF84F83C302921FDF746FFF5
:1034E0002C215846FDF742FF24E021F020005B2804
:1034F0000AD10132C9B258460392FDF737FF204680
:10350000FFF7D6FD039ABEE75D2808BF02F1FF3240
:10351000F0E77B299CD120460391FFF7C9FD236981
:103520007B2BA7D104F140000399FDF71FFF204634
:10353000FFF7BEFD7B2104F14000FDF717FF4FF0C0
:10354000000B06E7BAF1780F09D8BAF15B0F0AD879
:10355000BAF1220F53D029D8BAF10A0F23D05C2137
:1035600004F1400082E7AAF15C021C2A73D8DFE86C
:1035700002F046727272728A2A7272723A727272B1
:1035800072727272307272720F722D3D37725C00FD
:103590004FF00D0B94F83C300B2B77D1594604F1CA
:1035A0004000FDF7EAFE4FF0000B4BE7BAF1550F74
:1035B0001CD0D4D8BAF1270F21D0BAF14E0F4AD17E
:1035C00006480AF021FE4FF0080BE3E74FF0090B25
:1035D000E0E74FF00A0BDDE7F8BA050801BB050884
:1035E0004FF00B0BD6E74FF00C0BD3E794F83C20D1
:1035F0000C2A06D15C2104F14000FDF7BEFED34643
:10360000C8E7BAF1750F14BF4FF0080A4FF0040A6B
:103610004FF0000BBAF1010A0AD2BBF5881FB9D3EB
:103620004FF0010384F83C30BDE74FF0020AEFE7AA
:103630002046FFF73DFD226903921046FEF744FB4A
:10364000002800F05081039A1046FEF77DFB4FEAF8
:103650000B1B8344DEE7AAF1300BBBF1070F3FF6EB
:103660007EAF4FF0030A06E02046FFF721FD2269F6
:10367000303A02EBCB0B227D303A072ACDD8BAF193
:10368000010AF1D1C9E74FF0070B83E7BBF1FF0F48
:10369000C6D80C2BC4D15FFA8BF104F14000FDF7C2
:1036A00065FE80E70298C9B2F9E7CB453CBF03232A
:1036B00084F83C3059E6033B23669BE62846FEF738
:1036C000EFFA2169D8B95F2919D07F2917D80846A0
:1036D000FEF7F0FA002855D123692E2B4DD0844DEA
:1036E00000262F781FB12369BB4240F0A4802046FA
:1036F000FFF7DEFC002F40F0A6800123AAE5082397
:1037000084F83C3004F14005C9B22846FDF72EFE8E
:103710002046FFF7CDFC2069D8B92846FDF717FEF3
:10372000744F0646002557F8041B304627F03AF838
:1037300000281CD10E35EDB2112D84F83C507FF4D9
:1037400064AD6D4BD3F81032002B14BF0E23102341
:1037500080E5FEF7A5FA40B920695F2805D07F28EB
:1037600003D8FEF7A7FA0028D7D0217CCDE7FFF6D3
:103770004CAD0135242DD6D147E5207DFEF79AFAD0
:103780000028ACD021692E292AD10A2384F83C30A4
:10379000002504F140063046FDF7EFFD2046FFF717
:1037A00087FC0A27206900283FF42FAD55BB20F085
:1037B0002003452B26D16521304684F83C70FDF767
:1037C000DCFD2046FFF774FC21692B2901D02D294F
:1037D000E8D13046FDF7D1FD2046FFF769FCE1E76F
:1037E0000923302984F83C30D2D1237D43F02003D3
:1037F000623BDBB2162BCBD8404DDD4015F0010506
:10380000C7D1C5E7FEF74CFA28B121692E290DD1A1
:1038100084F83C70DDE72069FEF74CFA0028F4D10B
:1038200023692E2BF1D05F2BD6D0EEE421F02003BC
:103830004A2BCED1ECE7652F01D0632F00D10135A3
:10384000013601354DE7212F08D123693D2B7FF447
:1038500054AF2046FFF72CFC3923FBE42E2F0FD169
:1038600023692E2B02D1237D2E2B01D05C23F1E482
:103870002046FFF71DFC2046FFF71AFC0D23E9E464
:103880000335334615F8027C632F18D0652F16D008
:103890001B4AD35C84F83C30543BDBB2052B3FF62B
:1038A000B4AC012202FA03F313F02A0F18D113F07B
:1038B000150F3FF4AAAC636A13446362A5E415F8DC
:1038C000012C2169914206F1010607D12046FFF73C
:1038D000EFFB3346652FDBD00235D3E7632FFAE7E2
:1038E000636A013BE9E7012384F83C30834651E6F3
:1038F000B3BA050878090608B40400200120400086
:10390000080A06087FB5064601AD742085E80E005A
:10391000FCF7B0FC0446034695E8070043F8046B47
:1039200083E8070001236FF001020025C4E9063295
:103930000A22C4E90A23C4E908551420FCF79AFCBA
:103940002021206304F14000FDF792FC294604F198
:103950005000FDF78DFC294604F164002566FDF753
:1039600087FC236B20461D802561A582FFF7A0FB05
:103970002046FFF79DFB2046FFF79AFB2046FFF706
:103980002FFCA36B012B06D094F83C30052B1CBFF9
:10399000062384F83C30204604B070BD30B585B0B5
:1039A00001AC05462046FFF76BFB94E80E00284665
:1039B000FFF7A8FF05B030BD30B585B001AD0446B6
:1039C0000146284621F0A4FA95E80E002046FFF7AC
:1039D00099FF05B030BD10B50446B0B1C36840686A
:1039E000984704F14000FDF76DFC04F15000FDF72D
:1039F00069FC04F16400FDF765FC206BFCF762FCD8
:103A00002046BDE81040FCF75DBC10BDD0E9043293
:103A1000013B036152F823007047036942695B1A56
:103A2000013B52F823007047F8B5446A06460D463C
:103A3000B4B1D4E900030B44834222D908310022F7
:103A400001442046FCF73CFC0246B8B961682046B8
:103A50000831FCF735FC63682360336A63603462C5
:103A6000802D2F4638BF802707F10800FCF702FCA5
:103A70000023076043600446706202E023682B4421
:103A8000236060680544656008342044F8BD38B59B
:103A90000D460C211446FFF7C7FF4FF49D72C0E995
:103AA0000124056038BD38B5D0E903329A42044696
:103AB0000D4608D3103399004069FCF7F6FBE36824
:103AC00060611033E360D4E90432591C216142F88B
:103AD000235038BDF8B504461D46D0E900038342A3
:103AE0000F46164608D31030C100A068FCF7DDFB76
:103AF0002368A06010332360D4E90103421C626094
:103B000053F8301067F3170143F8301003EBC0028D
:103B1000D6705560F8BD10B48469CAB20023616BD9
:103B20005DF8044BFFF7D6BFF0B593B00446684686
:103B30000E4617461D46FCF75DFB10B1002013B082
:103B4000F0BD3A46314620460AF098F90446FCF7A3
:103B500027FBA30703D12268024B9A42EED02C60C8
:103B60000120ECE7D416060810F00102034604D049
:103B700040F001030B6001207047A8B110F0030072
:103B800013D11A793A2A11D19B680B6013F0010006
:103B9000F1D19A070AD11868054B9842EBD0054B32
:103BA000C31A58425841704770471046704700BFCB
:103BB000C01F0608681D060810F001021CD110F095
:103BC00003030CD000F00F03062B15D00A2B11D1E4
:103BD00000090D3803288CBF00200120704770B108
:103BE00002793A2A08D02D2A08D18068B0FA80F0EC
:103BF00040097047104670470120704718467047CB
:103C0000C20702D540F001007047830710D00309B6
:103C100000F00F00062803D1D80040F002007047E2
:103C2000A3F10E00022809D8064B53F82000704774
:103C300030B103793A2B03D180687047024870474E
:103C400002487047340A060888260608BC2A060877
:103C500038B505460C46FFF7AFFF38B12846FFF7E9
:103C6000CFFF0BF0E1FA031B5842584138BD2DE954
:103C7000F0410F4605461446114689B9204612F018
:103C8000BBFE014600F10808A4B90A462846394699
:103C9000FFF7FDFE01462846FFF705FF012007E07C
:103CA00001392846FFF7B9FEFFF786FF0028E4D167
:103CB000BDE8F0812846FFF7A9FE0646FFF7A0FF02
:103CC000013C48F82400002EDED0B307DCD1686A3E
:103CD00000F108039E42D7D3426813449E42D3D2D8
:103CE00073681B0A0233A2EB83024260CCE7000038
:103CF000F7B5866996F83C20A2F1080305460F4601
:103D0000042B52D8DFE803F003232B384C00D6E90C
:103D10001110FDF70DF9902F04460ED1C1000022BD
:103D200041F0020105F128000AF014FE28B14268B2
:103D3000D3071CD542F0010002E0200140F0020050
:103D40000146284603B0BDE8F040FFF7ACBE0022B4
:103D5000D6E91110334608F0F7FB0246E8E7009673
:103D6000D6E911100023012208F026FD0246716BEE
:103D70002846FFF78CFEE3E7D6E911100A2906D89A
:103D8000FDF7D6F830B1000140F00600D8E7FDF7A6
:103D900081F8F7E7D6E91121064810F015FFE5E7AD
:103DA000D6E9111010F0F0FFE0E7120142F00A002E
:103DB000C6E700BFB029060810B5FFF7D5FE50B121
:103DC0000B6813F0010007D19A0704D11868034B60
:103DD000C31A5842584110BD0120FCE7C01F060815
:103DE0000021FFF735BF0121FFF732BF2DE9F04F6A
:103DF0002D2A85B00446884616461D460BD1002163
:103E0000FFF70BFEC0B1820702D10379922B13D0CA
:103E100005B0BDE8F08F922A2ED10021FFF7FDFDFD
:103E2000014648B1830707D14768FBB2952B18D1EB
:103E30002046FFF7EBFD013DA6F12303DFB2092F7A
:103E400000F2EB80092B00F2CF80DFE813F0ED00E9
:103E5000ED00ED001E011E011E014501ED00CD002B
:103E60008F01962BE8D127F0FF07204647F09207F5
:103E7000FFF7CCFD4F60CBE7962A13D1D0E90123A1
:103E800003EBC203013513F8153C2D2B40F0AD8038
:103E90002A46FFF7ECFE002800F0A7806368023B8B
:103EA0006360B5E7A2F11E03012B5FD9202A00F061
:103EB0008380052AC0D10021FFF7AFFD0746002807
:103EC00000F0938010F0030A05D1436803F0FE036D
:103ED000562B00F08A8001212046FFF79EFD00F05E
:103EE0000F03022B40F08180BAF1000F7DD13B79A6
:103EF0002C2B7AD1BB6803F00F02022A75D11B0963
:103F0000482B72D1FB68002B6FD09A076DD11A79BC
:103F1000302A6AD1D3F808B04FEA10195846FFF793
:103F20004BFE002840F0FD80B749B8480DF0A2F8DC
:103F3000A1693A680968054653460DF07DF928469F
:103F4000FCF770F91E2E0AD1FFF74DFF18BB38465B
:103F5000FFF746FF00B9D3460BF1FF3A0BE0FFF73E
:103F60003FFFC0B93846FFF73EFFF3E705F1FF3AE0
:103F70008DB1AB46A94609F1FF3949462046FFF706
:103F80004CFD23696269A3EB0B03074642F823004B
:103F9000B9F1000FD6D10021514508D16D1A012D7C
:103FA0003FF436AF362E00F04281332E3DE12046FD
:103FB000FFF72CFD0131EFE70021FFF72EFD07464B
:103FC000FFF70EFF68B93846FFF70DFF68B1EA2129
:103FD0002046FFF71BFD204605B0BDE8F04FFFF778
:103FE00062BD4FF48571F3E72B26A91C890020469A
:103FF000FFF71AFD46EA05230746C0F80080436034
:1040000000F10801002D40F01B81962E03D13946A6
:104010002046FFF748FD3946DDE7922E00F0FE808E
:10402000062E00F00481BDE7691E2046FFF7F5FC6F
:1040300001A9FFF799FD0028B7D0022F9ABFA6F17A
:104040000D095FFA89F94FF02209AF1E002F09DA36
:10405000002D40F0CD80019AD30740F1CE8042F090
:104060000101B8E739462046FFF7D7FC02A9FFF760
:104070007BFD002899D0DDE9011201AB4846FFF72E
:1040800053FD002891D0013FE0E7691E2046FFF76D
:10409000C4FC01A9FFF768FD002886D0AF1E002FE1
:1040A000D6DD791E2046FFF7B8FC02A9FFF75CFDBC
:1040B00000283FF47AAF39462046FFF7AEFC0009EE
:1040C0002438DDE9011201ABC0B2FFF72DFD002855
:1040D0003FF46BAF023FE2E700212046FFF79DFC73
:1040E00001A9FFF741FD00283FF45FAF0121204601
:1040F000FFF793FCC0F30710332801990BD1CF07CA
:1041000007D488077FF451AF0A68414B9A427FF485
:104110004CAF022001E03F38C0B209F0E1F8019055
:1041200096E75846FFF76CFD4FEAC9030A46074673
:1041300043F0020104F128000AF00CFC47604846F5
:10414000FCF7BBFF03785F2B204608D1FFF75EFC2E
:1041500000252046FFF75AFCA84608266CE6FFF724
:1041600055FC59462046FFF79EFC3EE701212046BC
:10417000FFF753FC00F00F03022B07467FF415AF47
:1041800000212046FFF749FC00283FF40EAF10F055
:1041900003027FF40AAF0379322B7FF406AF3909AB
:1041A000C900D0F808901B4841F002010AF0D2FB88
:1041B00000283FF4FAAE406802AA4FEA191108F04D
:1041C000D1FF029B002B3FF4F0AED9070AD49A0727
:1041D0007FF4EBAE1A680E498A4203D00E498A4238
:1041E0007FF4E3AE039A002A7FF4DFAE01932FE75A
:1041F0002046FFF70BFC013D2AE729462046FFF742
:1042000046FC0146E7E600BF8FBB0508141A060806
:10421000C01F0608400A0608681D0608D4E90123E5
:1042200003EBC20313F8053C2D2B7FF4DEAE2A46C8
:1042300041462046FFF71BFD00287FF4E9ADD4E698
:104240002046FFF7E3FB013D41F82500DAE600BF19
:104250000346006830B550B184070AD14468E5B21E
:104260008D4206D100F10803200A136030BD0346D9
:10427000FBE70120F9E700002DE9F04FA94B97B0CB
:10428000CDE9073102900D4605A8A7490192002407
:10429000FBF78EFF40234FF40070CDE90934FBF7A4
:1042A000E9FF20230B908020CDE90C34FBF7E2FFDF
:1042B0002146CDE90E0513A8CDE911440AF014FBFF
:1042C000019B002B48D0022B0CBF3F22224600232B
:1042D000696B964F09A8FFF7FDFB00230A9C002C91
:1042E00000F06481013C0B9991480A9401EBC402EF
:1042F00051F83410D6785268C1F3170A8D4911F875
:1043000006B08D49895D632E88BF41F4807100EB52
:1043100041080BF0300110290BF00F091ED02029A5
:104320004BD0002B00F01B81B9F1020F40F00A8145
:10433000012A40D000211BF0010F02F1FF3306D00B
:10434000B8F802003840B0F5805F08BF5308012B71
:1043500040F0E580E1B1E2E03D22B8E702B1BBB157
:1043600008EB420825E0C34638F8023B03EA0701A0
:10437000B1F5805F0ED195F83C10C3F30B03994261
:1043800016D109A83146FFF7B3FC2846FEF728FFEF
:104390000023A3E7531C4B4504D23246514609A8DB
:1043A000FFF798FBBBF8001009A8FFF7B4FBEFE795
:1043B00001329145D7D8012390E773B102F1004350
:1043C000013B38F813303B40B3F5405F21D1002169
:1043D00009A80392FFF767FB039A08EB4204914593
:1043E0002BD8019B83B1052E0ED1002109A8FFF720
:1043F00014FB48B9012109A8FFF70FFB830744D03C
:1044000000F00F00022845D1002408EB4903A14623
:104410005AE0012ACFD995F83C30062B40F0F480C1
:10442000464947480CF026FE6A6B2968044600237B
:104430000CF002FF2046FBF7F5FE039434F8021B54
:1044400001EA0700B0F5805F16D195F83C00C9B2CB
:1044500088420ED1082805D1314609A80392FFF7FA
:1044600047FC039A03922846FEF7BAFE039A0132EC
:10447000B5E7002A9FD0CEE7531C5146324609A823
:10448000FFF728FB039B19888EE70028BCD003792F
:104490003A2BB9D109A8FFF7B9FA09A8FFF7B6FA7C
:1044A00000230822514609A8FFF7A0FC70E733F863
:1044B000022D02EA0701B1F5805F10D1D2B2082ABD
:1044C00002D1013409F101094345F0D1B9F1010FDD
:1044D0001CD11BF0400F19D00026314610E02146B8
:1044E00009A80393FFF799FA039B08B109F10109A1
:1044F0000134E9E7FFF78AFA0136002818BF0146C0
:10450000A64209A8F6D1FFF7CEFA41E71BF0800FCB
:1045100004D0002109A8FFF7C6FA01342346324629
:10452000C0E700BFD739020867D0020800F0FFFFDC
:104530002C0B0608B40E06087C0A06089BBB05086F
:10454000F0190608012A3FF436AF12F001013FF4DA
:10455000F2AEB9F1030F7FF45EAF0121EBE609EA99
:10456000020303F0010338F8134004EA0701B1F530
:10457000805F13D195F83C10C4F30B04A14202F103
:10458000010409D11BB9314609A8FFF7B1FB284640
:10459000FEF726FE2246E2E72246C5E6531C5146B8
:1045A000324609A8FFF796FA2146FDE613A80AF05D
:1045B000AFF9129850B1416822460831FBF780FEEE
:1045C000129B5A681A60119A5A60119395F83C3000
:1045D000002B7FF420AF0D9B002B3FF41CAF0E9BF4
:1045E0000B981B681093FBF76DFE0E98FBF76AFEA5
:1045F0000120FBF7E5FDDDE91001029B83E80300E4
:10460000184617B0BDE8F08F022B01D1034908E727
:10461000042B0CBF02490349034803E7ADBB05085F
:10462000CFBB0508E2BB0508141A060838B50446D6
:10463000406808B9606038BD4568FBF743FE28460E
:10464000F7E70000F8B5054630200E461746FBF7A1
:104650002AFE072D04460570C66001D0012D0FD13A
:10466000B368C3F30F13A38208F07EF9042320611B
:104670002783E3842020FBF7FDFDE0622046F8BDA0
:10468000014B5B5DEFE700BF640F060810B5044601
:10469000C06AFBF717FE2046BDE81040FBF712BECC
:1046A00030B5058D04460022954201D8002030BD6A
:1046B000E36A03EBC20043688B42F8D00132F3E7B0
:1046C00070B504460D461646FFF7EAFFC0B9E38C05
:1046D000228D9A4208D30633D900E06AFBF7E5FD44
:1046E000E38CE0620633E384238DE26A591C02EB1B
:1046F000C300218502F83360002343704380456086
:1047000070BD034618465B68002BFBD1FFF7C8BF9E
:10471000F8B544680E462CB9F8BD042BFCD105232E
:104720000370F9E7254628466D68002DF4D07768B8
:104730003946FFF7B5FF0028F5D00378043B022B7C
:10474000EAD806253570002239462046FFF7B8FF23
:104750000378002BE1D105706468F4E7036A1B8BD2
:10476000012B1EBFC3685B18C3607047836A10B516
:1047700004469B6F406A9847238B226A0133918CD1
:104780009BB29942238338BF938410BD038B10B52D
:10479000013B0383836A0446D3F88430406A984718
:1047A00020460121BDE81040FFF7D8BF2DE9F04FAA
:1047B00085B004460D46039298461BB1CB8A43F060
:1047C0000803CB82039BEB83236ADA8A42F0300230
:1047D000DA821B78002B46D1A36A039AD3F8B4601F
:1047E000606A43462946B44605B0BDE8F04F6047CD
:1047F000DB6A03EBC60B13F83630053B012B1DD8E3
:104800004FF0000917E0EB6A03EBC90213F83930E7
:10481000062B0ED1DBF804105368994209D1A36A24
:10482000BBF802201B69606A1F460023B8470AF1E3
:10483000010A09F101092B8D4B45E4DC0136236A9D
:104840001A8DB242D4DCBAF1000FC5D0A36ACDF8FC
:104850000080D3F8B860606A039B52462946B0478F
:1048600005B0BDE8F08F0026B246E8E7836A10B5D0
:104870000446D3F88830406A00219847A36A606AEA
:104880001B6B0F219847A36A606AD3F8CC300121D3
:10489000984720460321BDE81040FFF75FBF38B5B9
:1048A000836A04465B6C406A00229847A36A606A88
:1048B000D3F8C05000231A461946A8472046BDE841
:1048C0003840FFF7D3BF836A89681B6D406A0022B6
:1048D00009091847836A8968DB6B406A184710B575
:1048E0000446084611461A46FFF7ACFE236A4360A9
:1048F00000238360E3690BB9E06110BD1A469B6831
:10490000002BFBD19060F8E72DE9F04F87B005460A
:1049100000AF0C4611B90121116013E011F003063C
:1049200019D10B79682B19D1CB681B0913608C68DE
:10493000002CF0D0012604F00F03022B0DD1210929
:10494000002EE9D0AB6A686ADB6A002298471C3700
:10495000BD46BDE8F08F0026EDE716B9A3681B0938
:104960001360A04658F8043F4FEA132A08EB8A0365
:104970000AF1FF3BBB60C14659F8040F0009FCF780
:1049800091FBBB6899458344F6D10BF1070323F0F3
:104990000703ADEB030DC7F80CD0E946002358F828
:1049A000040F3B6007F114010009FCF792FB7A69E0
:1049B0007A600146484625F065FE3B687A68013317
:1049C0009A454A4405D091464FF02E0209F8012B32
:1049D000E5E75946F868FCF7ABFAAB6A0146DB6AD3
:1049E000686A00229847002EB1D00834BB689C4208
:1049F000ADD054F8041FAB6A686A1B6D0022090928
:104A00009847F3E731B1826801F00303134304BF11
:104A10000B68836070472DE9F04107461E4659B187
:104A200011F0030510D14B68D8B290420CD14FEA77
:104A300013280C1D454501DBBDE8F08154F8041F27
:104A40003846B0470135F5E738463346BDE8F04112
:104A500018470000F8B504460E4611461A460023D2
:104A600085780769837003610E4BFFF7D4FF636895
:104A7000BBB9618A51B1228A42B9A36A606AD3F88C
:104A8000A0309847A36A606A1B6C9847238A628AA1
:104A900031462046FFF78AFE003D18BF0125A5706C
:104AA0002761F8BD0153020870B54378012B054614
:104AB0000C4606D1036A0A461B8B0221FFF70FFF43
:104AC0002061A268216928464C23BDE87040FFF7A9
:104AD000C1BF70B513464278012A05460C4604D181
:104AE0000A460721FFF7FBFEA061A669E268284697
:104AF00046233146FFF7AEFFB08A70BD024B89688E
:104B00009D22FFF788BF00BF0D580208024B89683D
:104B10006B22FFF780BF00BFA573020838B543685A
:104B20000D46044611464BB905480CF0A3FA294638
:104B300060602046BDE83840FFF764BF38BD00BF65
:104B4000141A0608014AFFF7E9BF00BFE6BB0508D3
:104B50000B79092B70B50CBF858AC58A4FF6FF7398
:104B60009D42044602D1064AFFF7D8FF218B628B93
:104B7000A36A606A5B6F8A1A2946BDE870401847CD
:104B8000F3BB050838B5054679B101F00F03022BD8
:104B90000DD10C09204609F023FD002806DA06494C
:104BA000064822460CF0FCFA6860002038BD044A32
:104BB000FFF7B4FFF9E700BF0CBC0508A819060809
:104BC00011BC050870B51446054612780E4683B12F
:104BD00032B1032A04D0104ABDE87040FFF79EBFEF
:104BE000032626706168286AFFF78BFD00B1067006
:104BF00070BD62B901232370006A2146FFF788FD6A
:104C00002378012BF4D1054A31462846E4E7062AE9
:104C1000EED0034AE0E700BF21BC05082EBC050822
:104C20003BBC05082DE9F3414378012B04460D46B2
:104C30001AD10B79102B0CBF4FF001084FF0000870
:104C400008D0036A1B782BB9114A02B0BDE8F041C5
:104C5000FFF764BF01AA6D2105F10800FFF7F8FA1C
:104C600000260746B74202D102B0BDE8F081019BA1
:104C7000206A53F8261000220909FFF721FD434658
:104C8000024629462046FFF79DFF0136EAE700BFAE
:104C900042BC05084278012A0B4602D1006A02F0A4
:104CA00013BE816A026A406A203102F01CBE42785B
:104CB000012A0B4602D1006AFFF702BD816A026A2F
:104CC000406A103102F00FBE70B505460C4600294F
:104CD0002ED0CA0706D5836A5B6B4910686ABDE8A7
:104CE000704018478B0717D004F00F04022C4FEACE
:104CF00011110AD0062C0CD0052919D0836A406AFC
:104D00001B6BBDE87040C9B21847BDE87040FFF7A3
:104D1000CEBF836A9B6BE1E7836A0968DB68406A00
:104D200098472279034B214653F822302846D6E78C
:104D300070BD00BF6C0F06082DE9F74F05460C4605
:104D400016461F462046FFF74BF840B16EB9AB6AD6
:104D50009B6E3946686A03B0BDE8F04F184720469D
:104D6000FFF741F820B1002EF1D103B0BDE8F08F7C
:104D7000002C48D0A30746D163684FEA132BDBB25F
:104D80001E2B18D1DEB1043404EB8B0B5C45ECD048
:104D900054F8041F3B4632462846FFF7CDFFF5E79F
:104DA0005AF8041F019243462846FFF7C5FF09F150
:104DB0000109019A11E01F2B1FD1002EE3D0D5F875
:104DC0000C8008F10103EB600BF1FF3304F1040ADE
:104DD0004FF00009009386F00102009B4B45DFDC99
:104DE0000BF101013B4654F8211032462846FFF7EB
:104DF000A3FFAB6A41469B6AACE7202B03D1A468B2
:104E000086F001069EE721462846FFF75DFFAB6A64
:104E1000686ADB6E3A46314603B0BDE8F04F18478A
:104E200038B5026A1278072A04460B4606D0022AD1
:104E300004D0BDE83840144AFFF770BE9D6885B9BC
:104E4000A36A606A1B6B0F219847A36A606AD3F854
:104E5000CC300021984720460121BDE83840FFF7BB
:104E60007DBCAB070BD12B79AF2B08D12046A968AD
:104E7000FFF72AFF2046BDE83840FFF7F7BC294678
:104E80002046FFF721FFE0E754BC050870B54378E2
:104E9000CE68012B0446154606D1036A0A461B8BD1
:104EA0002946FFF71CFD7061002371691A462046F0
:104EB000FFF77CFCF1682046FFF706FF062D05D1C1
:104EC000A36A606AD3F8883000219847A36A606AB1
:104ED000D3F8BC500023AC461A46BDE8704001210F
:104EE000604738B50C460546C968FFF7EDFEA16876
:104EF0002846BDE83840FFF7E7BE0B79342B70B584
:104F000004460D4610D18968FFF7DEFEED68AD68F6
:104F100085B9A36A606A1B6B0F219847A36A0422B4
:104F2000D3F8A03002211AE0836A406A1B6B0F217C
:104F30009847ECE7AB071FD12B799A2B13D1A36AC3
:104F4000606A1B6B0F219847A9680029E6D02046AC
:104F5000FFF7BAFEA36AD3F8A03004220321606AE7
:104F6000BDE8704018479B2B06D1A9682046FFF783
:104F7000ABFEEB689968E8E729462046FFF7A4FEF8
:104F8000CCE710B504468968FFF79EFEA36A606A05
:104F9000DB6CBDE810400021184700002DE9F74305
:104FA0008D68044616465DB9002A75D0836AD3F829
:104FB000A03002222946606A03B0BDE8F0431847DA
:104FC00015F0030740F08A802B79372B13D132B1CB
:104FD000836A406AD3F8A030022201219847204614
:104FE0002946FFF771FEA36A606AD3F8A43003B0C4
:104FF000BDE8F04318479F2B70D1EB681A79A12ABE
:105000005AD1A22101AA03F10800FFF721F9A968EA
:10501000804621B38B0722D10B79372B1FD136B1B4
:10502000A36A411CD3F8A030606A02229847A9689D
:105030002046FFF749FEA36A606AD3F8A430984778
:105040004FF00109474510D1B9F1000F24D1A36AEF
:10505000606AD3F8A0300322791C98471CE02046F0
:10506000FFF732FE4FF00009ECE7019B53F82710E1
:10507000A9B18E0713D10E79A6F1370046424641F9
:105080002046FFF721FEB9F1000F11D04EB9184AA2
:1050900029462046FFF742FD03B0BDE8F083002615
:1050A000EEE7A36A606AD3F8A43098470137C9E7EE
:1050B000002EFBD00F4AEBE7AB685BB19A0709D132
:1050C0001B79372B06D10422294603B0BDE8F043F3
:1050D000FFF7DCBE052229462046F6E72946204692
:1050E000FFF7F2FDA36A0322D3F8A030012162E7A3
:1050F0005FBC050870BC05080122FFF74FBF70B503
:105100000D46C9680446FFF7DFFDA968A36A606A17
:10511000D3F89830C1F30711332918BF3F39BDE8E0
:10512000704014BFC9B202211847F8B54F680C4649
:1051300089680546FFF7C8FD3F0A0C340026023691
:10514000B74204F1080400DCF8BD54F8041C2846FA
:10515000FFF7BAFD54F8081CAB6A686AD3F89C30B4
:1051600009092439C9B29847E9E72DE9F0410C460D
:105170004E6854F8081F0546FFF7A6FDA6F10D0876
:105180005FFA88F8360A0127B74201DBBDE8F081F3
:1051900054F8041F2846FFF797FDAB6A686AD3F8F6
:1051A0009C30414698470137EEE72DE9F0414E68C3
:1051B00004460D46360A8968FFF786FD032E83BF35
:1051C000D4F80C8008F10103E3604FF000080127D8
:1051D0007B1C9E4222DC032E55D9E568606A6B1C5D
:1051E000E360A36A29469B6E9847A36A606A9B6A3C
:1051F00041469847A36A606A9B6801219847A36A61
:10520000606A1B6E9847A36A606ADB6D9847A36A61
:10521000606A9B6A2946BDE8F04118472969204623
:105220000237FFF751FDB74207DAA36A606A5B6D88
:105230009847A36A606A5B6E9847EB68A26A606AE7
:10524000D2F89C2003F00F010A2911D1C3F30713F0
:10525000252B1ABF343BD9B206219047B74205DA55
:10526000A36A606A1B6F4246002198470835AFE782
:105270001979852901D13221EFE79B680BB9072104
:10528000EBE73321E9E7BDE8F08110B50446896812
:10529000FFF71AFDA36A606AD3F89830BDE81040A2
:1052A000032118472DE9F0470D46D0F80C8055F83A
:1052B000046F5FFA86F9A9F11E03D3F1000949EBE7
:1052C000030908F101030446C360360A0027B74208
:1052D00006DBA36A606A9B6A4146BDE8F04718474F
:1052E00055F8041F20460137FFF7EEFCB742F0DA0D
:1052F000A36A606A1B6F424649469847E7E7000089
:1053000001F00F03022B70B5044612D00B79492B24
:1053100009D0483B082B18D8DFE803F00817071717
:105320001717170507000123A37070BD8E680D695C
:1053300075B9A378002BF8D1638A002BF5D02046ED
:105340001D4ABDE87040FFF7E9BBD1E90265EFE710
:10535000A3783BB3238A01339BB2012B23820ED166
:10536000618AD4E90903D1B1D3F8A030002298476B
:10537000A36A606AD3F8A030022200219847294628
:105380002046FFF7A1FCA36A606A9B6B310998472E
:10539000A36A606AD3F8A430BDE8704018471B6C5C
:1053A0009847E5E7638A0133638229462046BDE8D2
:1053B0007040FFF789BC00BF7BBC05082DE9F041B8
:1053C000C568D1F80C800E46AB1C04460022D8F804
:1053D0000810C3602B46FFF7AFFCB1682046FFF70B
:1053E00073FCA36A606A9B6E6F1C39469847A36A78
:1053F000606A9B6A29469847A36A606A9B684FF077
:10540000FF319847D8F80C102046FFF75DFCA36ADF
:10541000606A9B6A3946BDE8F04118472DE9F047BC
:10542000C668D0F814A0B0F81A908682B31CC36086
:1054300006F10108038BA0F81680044643838868B0
:105440000D46FEF7CDFCF8B9E768A8687B1CE36061
:10545000FEF7C9FC20B9A36A606A9B6E4146984773
:10546000A36A606A9B6A39469847E9682046FFF755
:105470002BFCA36A606A9B6A41469847A9683B4631
:1054800001222046FFF758FC2969C4F814A02046E1
:10549000A4F81A90FFF718FCA36A606A9B6A314669
:1054A000BDE8F04718472DE9F347C668731CC36091
:1054B000044688680D46FEF793FC0246E8B9E768A3
:1054C000A9687B1CE36020463B46FFF735FC20467D
:1054D000E968FFF7F9FBA868FEF785FCD8B92B69E6
:1054E0000BB96B6923B1A36A606A9B6E314698471A
:1054F000A36A606A9B6A3946984701AA712105F13F
:105500001000FEF7A5FE002781464F450BD16969C3
:105510002046FFF7D9FBA36A606A9B6A3146984729
:1055200002B0BDE8F087019B53F82780D8F8080047
:10553000FEF756FC024600BBD4F80CA0D8F80810C1
:105540000AF10103E36020465346FFF7F5FBD8F864
:105550000C102046FFF7B8FBD8F80800FEF743FC14
:10556000D4E909230028D6D19B6E314610469847CE
:10557000A36A606A9B6A514698470137C5E70000F5
:10558000184B2DE9F041D3F8107204460D463FBB8D
:10559000C6688968731CC36001223346FFF7CCFBE1
:1055A000A36A606A5B691F2101229847E96851B1CB
:1055B0002046FFF789FBA36A606AD3F8BC503A46DD
:1055C0003B460121A847A36A606AD3F8C83001218D
:1055D0009847A36A606A9B6A3146BDE8F041184764
:1055E000BDE8F081B404002070B58D6804463DB973
:1055F000836AD3F8C8302946606ABDE8704018470E
:10560000AB070ED12B795E2B0BD1A968FFF75CFBA2
:10561000E9682046FFF758FBA36A0221D3F8C83097
:10562000EAE729462046FFF74FFBA36A0121D3F89A
:10563000C830E1E710B504468968FFF745FBA36A67
:10564000606ADB6DBDE81040184700002DE9F041AD
:10565000026A1278072A044604D0BDE8F0411A4ACB
:10566000FFF75CBA8D685DB9836A406A1B6B0F21D6
:105670009847A36A606AD3F8C430BDE8F041184780
:1056800015F003021DD12B791B2B1AD1C668EF68C8
:10569000731CC360B9683346FFF74EFBA968204608
:1056A000FFF712FBA36A606AD3F8C4309847A36A75
:1056B000606A9B6A31469847F9682046FFF704FB09
:1056C000D7E72946F9E700BF99BC05082DE9F04165
:1056D0000C46054654F8046F360A04EB8607BC42B4
:1056E00008D1AB6A686AD3F8A03031460022BDE821
:1056F000F041184754F8041F2846FFF7E5FAEEE793
:10570000896810B4034641B9826A406AD2F8A04061
:105710000A4623465DF8044B18474A68120A022AD3
:105720000BD1CA684AB1940707D11279AC2A04D1C7
:105730005DF8044B0622FFF7A9BB5DF8044B184641
:10574000FFF7C4BF2DE9F0410E46054656F8043F69
:105750000F464FEA13280024444501DBBDE8F081E1
:1057600056F8041F2846FFF7AFFA6B683BB10234C6
:10577000284657F82410BDE8F041FFF743B901343B
:10578000EAE710B50446FFF7DDFFA36A606AD3F8C5
:105790009C30BDE810402221184770B58D68044642
:1057A00045B9836AD3F8A03001222946606ABDE872
:1057B00070401847A9071ED16B68DAB2922A1AD135
:1057C0001B0A022B0CD1EB6853B19A0708D11B7945
:1057D000AC2B05D129460322BDE87040FFF756BB2C
:1057E00029462046FFF7AEFF6968A36A0122D3F875
:1057F000A030090ADAE729462046FFF765FAA36ACE
:105800000122D3F8A0301146D0E7000001F00F03C9
:10581000022B2DE9F04705460C4604D1BDE8F047C0
:105820000909FFF737BA002955D011F0030652D104
:105830000B792C2B38D18968FFF746FAE668002EE1
:1058400049D016F0030846D17768FAB28E2A33465B
:1058500009D13F0A06F1040907F1FF3AC24510DCFD
:10586000013756F827301A79312A12D1996828461B
:10587000FFF72AFAAB6A686ADB6CBDE8F0470221E1
:10588000184759F8041F2846FFF71EFA08F10108C7
:10589000E4E7322A1FD19968AB6A686A1B6DBDE8DC
:1058A000F0470222090918472D2B14D18C6894B1B6
:1058B00063681B0A022B06D0271D6368B6EB132F03
:1058C00010D3BDE8F087E368002BF5D09A07F3D139
:1058D0001B79AC2BF0D121462846064ABDE8F0479B
:1058E000FFF71CB957F8041F2846FFF78FFF013652
:1058F000E3E700BFA5BC05082DE9F8430446006AAC
:10590000C68A1746B2070D4606D5374A29462046AD
:10591000BDE8F843FFF702B901F00F02022A18D1DF
:10592000A37809098BB1838B013383834FF000097E
:105930004FF00108002955D00022FEF7C1FE037880
:105940000646002B38D0294AE0E7438B01334383D6
:10595000ECE70A79BA4289460BD18968A37809092C
:105960001BB1838B01338383E2E7438B0133438392
:10597000DEE79A4218D1A378002BC6D10122A2708B
:10598000896879B301F00F02022A18BF894646F0F0
:10599000040618BFD9F80810C68206BF090999463F
:1059A00009094FF00308C5E7896846F002060909AE
:1059B000C6824FF00508BDE70423037080F801801C
:1059C000236A1B8B032B0DD1482F0BD1B9F1000F8C
:1059D00008D0D9F80C102046FFF7D4F8737843EAC2
:1059E00000137370BDE8F883E2BB0508B9BC050875
:1059F00049234822FFF780BF4F234E22FFF77CBF89
:105A00002DE9F04F0E468DB0016200214270C16059
:105A10003378072B0446154605D08B4A0DB0BDE8F8
:105A2000F04FFFF77BB8012A05D0036B021D1B68FE
:105A3000C06A294698476378D6F80C80032B10D1AA
:105A40000BAA462108F10C00FEF702FC236B0B9A0F
:105A50009B680146E06A984763687083002B40F0BA
:105A6000BC80D8F81010C1B101F00F03022B10D187
:105A70000B09752B3FD006D83E2B3ED05E2B0CD0A9
:105A8000724A2046CAE740F253529342F8D10323A8
:105A900004E06F4A2046FFF741F80223049309AA65
:105AA000D8F814300893192108A8FEF7D1FB4FF05D
:105AB00000090690069B994521D16378012B16D9E0
:105AC000236B04995B68E06A98476378042B0ED1D6
:105AD000206A049BE26A0393438B02930023CDE97F
:105AE00000330521D2E90232006906F04DFF6368F8
:105AF000002B72D114E00023D0E70123CEE7099BED
:105B000053F829100B79082B4FEA890B02D109F1C0
:105B10000109CFE7052B06D04E4A2046FEF7FEFFCF
:105B20000DB0BDE8F08F8B68002BF5D09A07F3D14C
:105B3000CA68002AF0D11A792C2AEDD19E6806F0A5
:105B40000F02022AE8D1D3F80CA0BAF1000FE3D07B
:105B50001AF0030FE0D19AF80430302BDCD10AAAF6
:105B6000A4210AF10800FEF773FB360940F2554301
:105B70009E4207461BD1012805D10A9A136803F0FB
:105B80000F03022B04D0344A099B53F80B10C4E7CF
:105B9000E168012D01F10103E3601AD01268236B63
:105BA000E06ADB681209984798B92C4AECE740F2A2
:105BB00083339E4215D1012803D10A9B1968CB0774
:105BC00001D4274AE0E7012D03D0E06A491002F032
:105BD000BFFB6368002B9AD0D046D8F80030A36092
:105BE0009EE7B6F5747F23D1012804D90A9B1A6871
:105BF00012F0010601D11B4AC6E7012DE9D053106E
:105C000007930A9A0BA952F82600FEF7D5F808B9AF
:105C1000154AB9E7E36A0B9805930CF0F4FC0136DA
:105C200002460799059802F09AFBB742E9D1D0E7FE
:105C3000012DCED0236B0246D3F810B0E06A0A9B48
:105C40003146D847C5E700BFC3BC0508D9BC050825
:105C5000DDBC0508EEBC0508FCBC050808BD050850
:105C60000CBD050818BD05082ABD05084278012AA3
:105C70000B4602D1006A01F027BE816A026A406ABF
:105C8000183101F030BE00002DE9F14F8F070446B6
:105C90000D46164613D001F00F03022B18D102F067
:105CA000FD06012E4FEA111104D001B0BDE8F04FFE
:105CB000FFF7DCBF01B0BDE8F04FFEF7F8BF496861
:105CC000CBB22D2B7FD00BD8062B0ED02C2B13D084
:105CD000514A2946204601B0BDE8F04FFEF71EBFED
:105CE0002E2B00F084809D2BF2D1002EF0D105F1F7
:105CF0000802090A20467FE0022A02D0A968FEF7BE
:105D0000E3FFEF68002FE3D017F00309E0D17B68D1
:105D1000DAB28E2AB8460DD1022E4FEA132805D0EA
:105D200007F1040A08F1FF3BD94515DB08F101082A
:105D300057F8288098F80430312B27D1022E13D140
:105D4000A36A606A5B6E9847A36ADB6C0121606A94
:105D500001B0BDE8F04F18475AF8041F2046FEF77F
:105D6000B3FF09F10109DFE72046D8F80810FEF774
:105D7000ABFF012ED4E9090305D19B6D9847A36AB7
:105D80000021DB6CE3E7DB6C0121E1E7322B9FD1E3
:105D9000012ED4E909030CD15B6D9847A36AD8F8AA
:105DA00008101B6D0022606A090901B0BDE8F04FC0
:105DB0001847022E01D11B6E9847A36AD8F8081025
:105DC0001B6D0122EFE7AA68002A81D0002E7FF424
:105DD0007FAF5168090A022907D1D3682BB1980710
:105DE00003D11B79AC2B3FF473AF083282E7002A52
:105DF0007FF46EAFA96821B901B0BDE8F04F00F0A3
:105E000073B88E0703D10B79922B0A46E1D005F1C6
:105E1000080201216EE700BF35BD05082DE9F047F6
:105E2000C7681E46BB1CC360836A04460D469B6A56
:105E3000406A394690469847A36A606AD3F88C3026
:105E400007F1010949469847A96800222046FFF753
:105E50001BFF2D6965BB41462046FEF735FF236ACF
:105E600019780629D4E909031CD1D3F8CC30294686
:105E7000984720460121FEF771FCA36A606ADB6D3A
:105E80009847A36A606A9B6E39469847A36A606A1E
:105E90009B6A49469847A36A606AD3F89030BDE888
:105EA000F0471847B200D3F8A83005329847E8E722
:105EB0002B79AD2B07D1A9683B4600222046FEF77F
:105EC0003BFFED68C6E7E9682046FEF7FDFEA36AE2
:105ED000606AD3F8883001219847731C42462946EE
:105EE0002046FFF79BFFCCE72DE9F84304460D461B
:105EF000904601F1FF3900264FF0FF37B9F1FF3F1F
:105F00000CD17B1C05D1A36A606AD3F8AC3029465A
:105F100098470026AE421DD1BDE8F88358F82610F8
:105F200071B18A070CD10B79222B09D101370BD122
:105F3000A36A606AD3F8B0304A463146984737467C
:105F4000013609F1FF39D9E72046084ABDE8F84390
:105F5000FEF7E4BD58F82610B74208BF8968002252
:105F60002046FFF791FE0136D4E700BF49BD050882
:105F70002DE9F0470446904699460F4621B9BDE801
:105F8000F0471946FEF7A0BEC668731CC3601568CB
:105F900035B315F0030A23D12B797B2B20D1A968C7
:105FA000FEF792FE524631462046FEF7DFFBE968D7
:105FB00052462046FFF768FE4B4608F10402791E60
:105FC0002046FFF7D5FFA36A606ADB6F314698472A
:105FD00020460321FEF7C2FBBDE8F047FEF7D6BB23
:105FE00029462046FEF770FE204600223146FEF785
:105FF000BDFBA36A606ADB6D9847DDE737B50C46E9
:10600000054601AA7A2104F10800FEF721F9E368A8
:10601000019A01462846FFF7ABFF03B030BD2DE9DA
:10602000F04F8B6803F00F03022B89B004460D4636
:1060300040F00081CB68002B00F0FC80980740F016
:10604000F9801A792C2A40F0F5809A6802F00F0145
:10605000022940F0EF8012097C2A40F0EB80DB68D7
:106060001A79302A40F0E6809B68069307AAA4219B
:1060700006A8FEF7EDF8431E022B00F2DB80079B1B
:1060800001281A6800F0C980022800F0C4809E68C8
:10609000F10740F1CF80710800F0CC80D3F8049074
:1060A00032B1930704D11179A639022940F2C28096
:1060B000B9F1000F08D019F0030F05D199F80410B9
:1060C000A639022940F2B680AB6801932B696F694B
:1060D0000293E5686369218B0493638B039305F155
:1060E000010BAB1C618319F0010805F10401059354
:1060F000A582A4F816B005F1030AE16005D149466E
:1061000020460592FEF7E0FD059A11462046FEF76F
:10611000DBFDA26A606A926E51469047A26A606A8D
:10612000926AA91C9047A26A606A526D9047002249
:1061300001992046FFF7A8FD02992046FEF7C4FD0D
:10614000A26A606A926A5946904731462046FEF735
:10615000BBFDA26A606AD2F89C200E219047A26A19
:10616000606A926A51469047D4E90902B8F1000F7B
:1061700057D1936D9847A36A606A1B6E9847A36ACC
:10618000606AD3F89C30002EACBF002101219847F3
:10619000A36A606ADB6EAA1C01219847049B6361B5
:1061A000039B6383002F43D0A36A606ADB6D98472B
:1061B000B8F1000F03D1A36A606ADB6D98473946D6
:1061C0002046FEF781FDE668606A731CE360A36AFF
:1061D00031469B6E9847A36A606A9B6888F001010C
:1061E00001319847A36A606A9B6A29469847A36A67
:1061F000606ADB6D9847B8F1000F03D1A36A606A4B
:10620000DB6D984727B1A36A606A9B6A314698475D
:1062100009B0BDE8F08F032640E791460326024609
:1062200046E7526D904749462046FEF74DFDA6E7EA
:106230003E46D7E7E668238BB4F81A9063836FEA8B
:1062400046436FEA5343D4F814A0A382771CF31C8F
:10625000E968E3602046E782FEF736FDA36A606ADC
:10626000D3F8883001219847A36A606A9B6A39464F
:106270009847A36A606AD3F88C3006F10208414659
:1062800098470022A9682046FFF7FEFC29692046AE
:10629000FEF71AFDA36A606A9B6E39469847A36AA7
:1062A000606A9B6A41469847A36A606AD3F8903057
:1062B00098476969C4F814A02046A4F81A90FEF71C
:1062C00003FDA36A606A9B6A314609B0BDE8F04FDE
:1062D00018472DE9F74F0446174698460E4629B948
:1062E000194603B0BDE8F04FFEF7EEBCC5682B1DA4
:1062F000C360136805F1010A05F1020B05F10309FA
:10630000002B00F0D28013F0030240F0CE80197908
:106310007B2940F0CA80996801920093FEF7D4FC73
:10632000A16A606A496D884740F25E312046FEF7F7
:10633000B6FADDE900322046D968FFF7A5FC022253
:1063400029462046FEF712FAA36A606A9B68032179
:1063500098473A1D4346711E2046FFF7BAFFA36ACD
:10636000606A9B686FF002019847A36A606AD3F87D
:1063700080602A4651465B46B047A36A606A5B6DFF
:106380009847A36A606A5B6E9847A36A606A1B6E4F
:106390009847A36A606A5B6C002240F25F319847BD
:1063A000A36A606A5B6E9847A36A606A5B6E9847EF
:1063B000A36A606A5B6D9847A36A606A1B6D0022DE
:1063C0000A219847A36A606A1B6E9847A36A606AAD
:1063D0001B6B0F219847A36A606AD3F8C050002353
:1063E0001A460321A8472046FEF740FAA36A606ACE
:1063F000DB6E4A4600219847A36A606ADB6D9847C6
:10640000A36A606A1B6B0F219847A36A606A9B6E40
:1064100049469847A36A606A9B6802219847A36A25
:10642000606A9B6A59469847A36A606A5B6E9847A0
:10643000A36A606A5B6E9847A36A606A9B6A51466A
:106440009847A36A606A5B6C002240F25F3198470C
:10645000A36A606A1B6B0F219847A36A606A5B6D31
:106460009847A36A606A5B6D9847A36A606AD3F82D
:10647000C05000231A460321A8472046FEF7F6F92C
:10648000A36A606ADB6D9847A36A606A9B684FF0F5
:10649000FF319847A36A606A9B6A4946984720463D
:1064A00003B0BDE8F04FFEF771B919462046FEF77C
:1064B0000BFCA36A606A5B6D9847204640F25E3130
:1064C000FEF7EDF9A36A606ADB6D984737E72DE9BF
:1064D000F041CD6804460E4665BB0378C3B1036A3C
:1064E0001D78ADB94FF45B71FEF7E1FBB168204652
:1064F000FEF7EAFBA36A606AD3F8BC602A462B4623
:106500000121B047A36A606ADB6DBDE8F04118471E
:10651000B1688B0707D001F00F03022B08D120468A
:10652000FEF7D2FBEEE70029F9D00B793A2BF6D132
:10653000BDE8F081AF0740F0AF806B68DAB25B2A4C
:1065400011D1ED68002D4AD1006A0378072BEFD1F5
:10655000896801F00F03022BEAD10422BDE8F04163
:10656000D140FEF7ADB8562A13D101228968FFF752
:106570008BFBE9682046FEF7A7FBA968A36A606A5F
:10658000D3F89C3009093E39C9B298470222B16854
:106590007DE0572A25D11B0A5F1E013355F82310D1
:1065A000FEF792FB002F03DDA36A606A5B6D9847DC
:1065B000B16800222046FFF767FB04350026BE4283
:1065C000B6DA0136BE4203DAA36A606A5B6D9847A9
:1065D00055F8041F00222046FFF756FBEFE7A907F6
:1065E0005AD16B68DAB2062A56D1B768002F53D059
:1065F000BA0751D17A68D1B206294DD11B0AB3EB43
:10660000122F4FEA122847D1A8F10203012B43D8D9
:10661000BB6823B1980702D11B79222B3CD0FB68C1
:1066200023B1990702D11B79222B35D0B8F1020F83
:1066300006D03B6923B19A0702D11B79222B2BD0BC
:10664000A9682046FEF740FBE9682046FEF73CFBC0
:10665000B8F1030F07D120462969FEF735FBA36A7D
:10666000606A5B6E9847A36A606A1B6E9847B96858
:1066700000222046FFF708FBF96800222046FFF7BA
:1066800003FBB8F1030F7FF453AF396900222046B2
:10669000BDE8F041FFF7F8BA29462046FEF714FBA3
:1066A000002274E70023032A2DE9F04104460D4639
:1066B000164642700162C36080F8342002D1C08E59
:1066C00050BBA063A36A606A1B684FF000083146A4
:1066D000A4F836802A46984706212046FEF73EF861
:1066E0006778EE68012F04BFA5F82280A5F8248002
:1066F000B6B1B20714D133793F2B11D1B168FEF78F
:10670000E3FAA36A606AD3F8C4309847A36A606A60
:106710005B68BDE8F04118478000F9F7C4FDD0E799
:106720002B78072B00F29380DFE803F004912541DA
:106730004141410E31462046FEF7C6FAA36A606A1F
:106740001B6B0F219847DCE7012F12D10023A370A8
:10675000F168574B46222046FEF75DF92B8B032B41
:1067600007D131692046FEF70DFAEB8A43EA801320
:10677000EB827169DFE7A36A3168DB68606A98477A
:106780006378012B07D10023A370B168494B4C22D9
:106790002046FEF740F9F1682046FEF795FAEB8AAD
:1067A000DB07AED5A36A606ADB6D9847C6E7012FA9
:1067B000D6F80C8005D1206A04223946FDF780FF07
:1067C0006F83A36A3168DB68606A98472B78032B74
:1067D00024D1A36AD3F8A0300122606A002198472F
:1067E0002B78062B28D1A36A606A1B6C984701217D
:1067F0002046FEF75CFAA36A606A1B6C9847A36A9E
:10680000606A1B6C98470023B26841462046FFF738
:1068100005FB2B78062B7FF474AF8FE7042B04D194
:10682000A36A0222D3F8A030D7E7052BD8D1A36AF8
:106830000322D3F8A030D0E720460121FEF737FA33
:10684000A36A606AD3F8883001219847DBE7012FFB
:1068500004D104220A212846FDF732FF17212046E1
:10686000FEF725FA16212046FFF700FAB168A36A61
:10687000606A9B6B090998471A212046FFF7F6F9D1
:1068800031692046FEF720FA0A212846FDF708FF65
:106890000246D4E909031178042902D11B6B0F21A8
:1068A00050E71D69528800230A21A84729E700BF45
:1068B000F1590208F9590208036A10B51A8B044607
:1068C000FEF707F901462046BDE81040FFF7CEB9B4
:1068D0002DE9F04F8D682B79032B85B004460AD142
:1068E0002946FFF7E9FFAA69D38A43F00103D3825F
:1068F00005B0BDE8F08F026AD28AD20706D4624A98
:10690000294605B0BDE8F04FFEF708B9162B40F058
:10691000AD80C668E968331DC360FEF7D5F9A36A88
:10692000606A5B6C00224FF458719847A36A606AF2
:10693000D3F8C07000231A461946B847E768636960
:106940000093638B0193BB1CE360238B6383A36A77
:10695000606A9B6AA78207F1010806F1010B4146B4
:10696000A4F816809847012259462046FDF7FEFEFE
:10697000A36A606A5B6D9847204640F26231FDF77A
:106980008EFFA96820460022FFF77EF9A36A606A9D
:10699000D3F8943006F10209002249469847A36AC9
:1069A000606A9B6A59469847A36A606AD3F8D030F8
:1069B0009847A36A606A5B6D9847A36A606A5B69DF
:1069C00001224FF443719847A36A606AD3F89C3060
:1069D00008219847A36A606ADB6E06F1030A5246F3
:1069E00000219847A36A606ADB6D9847A36A606AD2
:1069F000D3F89430012231469847A36A606A9B6AB3
:106A000051469847A36A606A9B68012198472046CF
:106A1000FDF7BCFEA36A606AD3F8D4309847A36A36
:106A2000606A9B6A4946984729692046FEF74CF9F7
:106A3000A36A606A9B6E41469847009B6361019B15
:106A40006383A36A606A9B6A3146984769692046F6
:106A5000FEF73AF9A36A606A9B6A39469847A36AC7
:106A6000606ADB6D05B0BDE8F04F184703AA7A21D4
:106A700005F10800FDF7ECFBEB68039A01462046A0
:106A8000FFF727FC34E700BF50BD05082DE9F04FA4
:106A900085B0C5681E460E9B03936B1C0293AB1C0E
:106AA0000446C3600F46934629460122FDF75EFE69
:106AB00039462046FEF708F9A36A606AD3F8943095
:106AC0000022691C9847A36A606A9B6A2946984716
:106AD000A36A606AD3F8D0309847D4F80C9009F1D3
:106AE0000103E36000275F4518DB2046FDF74EFEFB
:106AF000A36A606AD3F8D4309847A36A02999B6A64
:106B0000606A984703992046FEF7DEF8A36A606A38
:106B10009B6A494605B0BDE8F04F18473346D4F8A4
:106B20000CA01A6801920AF10102E260019AD2F8FF
:106B3000088004360137B8F1000F4FD1BB4542D170
:106B4000A36A606ADB6D98470025A846019B204632
:106B5000D968FEF7B9F825B3A36A606A1B6B0F21E9
:106B60009847A36A606A9B6A41469847A36A606A2D
:106B70009B6801219847A36A606A1B6B0F219847A5
:106B800029462046FFF772F829462046FEF782F88C
:106B9000A36A606A9B684FF0FF3198472046FDF773
:106BA000F5FDA36A606AD3F89430012249469847FC
:106BB000A36A606A9B6A51469847A36A606A9B68A9
:106BC000012198478FE720461E4A1968FDF7A6FF66
:106BD000204605B0BDE8F04FFDF7D8BD18F003051D
:106BE0002DD198F80420762A434603D1DD68D8F8E1
:106BF00008802D09A36A606A5B6D9847414620466C
:106C0000FEF762F8A36A606AD3F89C3008219847BF
:106C1000A36A606ADB6E524600219847002D8FD030
:106C200029462046FFF722F8D4F80C8008F101032A
:106C3000E360022241462046FDF798FD86E70025E5
:106C4000D8E700BF67BD05082DE9F347C768984638
:106C50007B1C16460D46C36002223946DDE90AA9AF
:106C60000446FDF783FD002E2DD1A36A606A9B6860
:106C70000321984729462046FEF726F8A36A606A52
:106C80009B686FF002019847A36A606A1B6B0F2133
:106C90009847A36A606A9B6A39469847A36A606A04
:106CA0009B680121984749462046FEF70DF8A36AE4
:106CB000606A9B684FF0FF319847204602B0BDE8FC
:106CC000F047FDF763BDCDF800A0434632462946A4
:106CD0002046FFF7DBFED7E7F0B5CE683379782B97
:106CE00085B005460C4609D1B36801930023009393
:106CF00089681A46FFF7A8FF05B0F0BD742B03AAF8
:106D00004FF0770113D106F10800FDF7A1FA3769BA
:106D1000A168039B0246F06827B900902846FFF758
:106D2000B5FEE9E7BC68CDE900042846E2E704F1D6
:106D30000C00FDF78DFA00230093A168039B024627
:106D4000ECE7000001F00F03022B70B504460D467E
:106D5000164602D01E4AFDF7E1FE31462046FDF7F9
:106D6000B3FFA36A606A5B6D98476378012B4FEAB3
:106D7000151610D1226A1378033B032B0BD85068E9
:106D8000314600F0A1FD0346206A1A78032A08D193
:106D90003146FDF795FC31462046BDE87040FEF7D0
:106DA00065BF00223146FDF78BFC236A5B685B6898
:106DB000002B02460CBF0123002304D001780129D7
:106DC00004BF0021017029462046FDF7FBFEE2E7E3
:106DD00035BD05082DE9F04F87B0CDE90221044605
:106DE00005AAA42103A81D46FDF732FA002601904A
:106DF000B1463746B0464FF0010B019B9E4211D180
:106E000027B1A36A606A5B6B49469847029AD4E946
:106E10000903002A76D0D3F8C0403B4642462946B3
:106E2000A04713E0059B53F826A0BAF1000F5BD0F2
:106E30001AF0030F58D19AF80420A62A1AD1B807DD
:106E400007D5324A51462046FDF768FE07B0BDE837
:106E5000F08F1D2E01D92E4AF4E70BFA06F2DAF86C
:106E60000810204649EA0209FDF72EFF01350127E7
:106E70000136C2E7A72A0DD1A26A606A126C904758
:106E8000DAF8081047F002072046FDF71DFF08F169
:106E90000108EDE7A82A27D1DAF80C2072B1910792
:106EA0000CD11179AA2907D19268DAF80810204686
:106EB000FFF748FF0135DBE7AC290FD0DAF80810FF
:106EC00001F00F02022A01D0124ABBE7A26A606AEF
:106ED000926B09099047DAF80C10D5E70622514663
:106EE0002046FDF7D3FFE5E7BB0701D50A4AA9E72E
:106EF000B8F1000F01D0094AA4E751462046FDF73A
:106F0000E3FED7E7D3F8BC4087E700BF7FBD0508A5
:106F100086BD05088EBD05089BBD0508A2BD0508F8
:106F200070B50D46417801290446134603D12A461F
:106F3000FDF7D5FC6861A36A606A9B6C98476E692F
:106F400000231A4631462046FDF730FCA36AB18A79
:106F50009B6B606A9847E96829B18B0703D10B796D
:106F6000A32B08BF0021204602230022FFF732FF97
:106F7000B08A70BD002389681A46FFF72BBF000056
:106F80002DE9F8430C4689680546FDF79DFEE66845
:106F9000002E56D07768296AFBB209788E2BA36839
:106FA00019BF04F10C0601273F0A0836072903F030
:106FB0000F024AD1022A46D11A099A2A47D13368C8
:106FC0001A79302A3FD19B68002B3CD10A212846F0
:106FD000FDF76DFE2A6AD36A128D32B93168404AD4
:106FE0002846BDE8F843FDF799BD5978C9070FD584
:106FF00059682846FDF75BFE022FD5E909030AD838
:10700000D3F8BC4000231A460221A047012416E011
:10701000013A0833E1E7726811793229F0D1B46896
:1070200021793029ECD191685B6C012209099847DC
:10703000A168002301222846FFF7CCFE0324A742C3
:1070400025D8BDE8F8830024F9E7022AFBD11B0903
:10705000B3F5127FF7D133681A79302AF3D19B68E0
:10706000002BF0D013F00304EDD11B792F2BE6D1C8
:10707000AB6A686AD3F8BC80224623462146C047E3
:107080003368224699682846FDF788FFBEE704F179
:107090000108B84556F824104FEA84031AD20A7939
:1070A000322A17D13344D3F8049099F80430302BA6
:1070B00010D18968AB6A686A5B6C0022090998473D
:1070C000D9F80810002301222846FFF783FE08F1B3
:1070D0000104B4E72846FDF7F7FDA046F7E700BF37
:1070E000A9BD050810B5026A1278072A04460B46A6
:1070F00006D0022A04D0BDE81040064AFDF70EBDB6
:1071000020461946FFF73CFF2046BDE81040FDF73A
:10711000ADBB00BFBCBD0508D1E90212FFF712BE2E
:10712000036A10B51A8B0446FFF7FAFE01462046A3
:10713000BDE81040FEF79ABD2DE9F04F044685B03A
:10714000884602AA422108F10800FDF781F8236A67
:1071500000271E8B8346BA465F450AD1D8F80C102B
:107160000B79032B51D132462046FDF7B2FC054680
:1071700059E0029B53F82730019303AA6C2103F1D5
:107180000800FDF765F8039B19680A09732A05468C
:107190000DD02046FDF798FD4FF00109A94528D3F1
:1071A000019BD96869B12046FDF78EFD09E00228F0
:1071B00009D02A4A2046FDF7B1FC35460AF1010AFA
:1071C0002E460137C8E759680B09412B0DD040F214
:1071D00095429342F2D040F26552934207D040F27A
:1071E0008E329342E5D10425E8E70125E6E7032541
:1071F000E4E7039B606A53F82910A36A00221B6D21
:107200000909984709F10109C8E7442B17D18F688C
:10721000324639462046FDF75CFCBA69D38A43F012
:1072200001030546D3820027ABEB0A0ABA450BD807
:1072300029462046FEF71AFD05B0BDE8F08F32461C
:107240002046FFF76DFE92E7A36A606AD3F8BC6040
:1072500000231A460121B0470137E7E7C7BD0508FB
:107260002DE9F3418D6805F00F030A2B04460E4605
:1072700007D0002D31D015F003012ED12B79652BCD
:107280001ED10095002501AA65216846FCF7E0FFA4
:10729000019B002103EB800040F2CA52834215D1CA
:1072A000F26840F21A439A4237D1236A1F78B7B185
:1072B0003B4A3146204602B0BDE8F041FDF72EBC06
:1072C000622BEDD1AB680093ED68DCE753F8047BEB
:1072D00097420CBF01310331E0E70021E0E7A36AE8
:1072E000606A5B6B9847A36A606A9B6B052198474D
:1072F000A36A606AD3F8A0303A460121984701AAF0
:1073000029462046FDF700FBA36A606ADB6A022279
:10731000394602B0BDE8F0411847A36A606A5B6B6A
:10732000984706F10C006A466A21FCF791FF002796
:107330000646B742D4E9090313D1D3F8A03000229E
:1073400031469847294601AA2046FDF7DDFA002577
:10735000B542D4E909030DD1DB6D984702B0BDE811
:10736000F081009A9B6B52F8272091680909984791
:107370000137DEE7009ADB6A52F82580D8F80870FA
:107380003F09394601229847D8F80C1029B93946E7
:107390002046FEF76BFC0135DAE70909F8E700BF84
:1073A000DFBD0508836A37B504460D465B6B406A4E
:1073B00000219847A36A606A1B6B0F2198472946F2
:1073C000204601AAFDF7A0FA0199204603B0BDE8C6
:1073D0003040FEF74BBC00002DE9F04F9BB0CDE9EB
:1073E000020110209D4D1446F8F744FF2B694360BD
:1073F00058220021064604A823F088F94FF0FF33F5
:10740000012113A809938DF8104007F06DFA039B32
:10741000D900012241F0020113A807F09BFA0123D1
:107420004360002116A80BF04BFC029A95F8143229
:107430001268002104A8FDF752FA054611A800F0D1
:1074400029FF874B0B9F01900D900E934FF0000B7F
:107450000FB1059C1CB30B9C14B1059B002B3ED0B7
:107460000198DFF8FC91DFF8FCA1594600F019FF04
:107470000B9C0027DDF81480002C00F03981B8F156
:10748000000F00F0F1800C9C04A8E168FDF7BAFA47
:10749000A38A069A0399404609F0CEFE2CE13B8B65
:1074A000042B4FF00102394604A807D1FEF7A8FAD1
:1074B000079BBF689B4538BF9B46C9E7FFF7F2F8BB
:1074C0003B8D9C42F4D2FB6A03EBC40113F83430C9
:1074D000012B02D13846FDF71BF90134F0E7E28AAF
:1074E000520716D5218D013913D3E76A07EBC10284
:1074F0004FEAC10E507810F0020F25D04BB1D3E9FE
:10750000008C92E8030083E8030047F80E80C2F87D
:1075100004C04FF0000323840027B4F828C0674557
:1075200018DB00239C454ED1D4F804E0BEF1000FD7
:1075300008D00020BEF828A00346504553DB002B9E
:1075400040F08A80A46887E7002BCCD1012808BFCF
:107550001346C8E72378D4F82C80012B4FEAC70ADA
:1075600008EBC70905D1D9F804300A2B12D101372D
:10757000D3E718F837300DD9012B0BD14FF00303A7
:1075800008F83730238B032B16D0E38A43F010031F
:10759000E38203E018F80A30032BF3D018F80A301E
:1075A000042B03D099F80130DB07E0D5238C5A1C5B
:1075B0002284A9F80230DAE7D9F8040007F010F8BD
:1075C0000128EBDCE1E7E26A02EBC30112F83320A9
:1075D000052A06D14A78D7075FBF228C4A8001323C
:1075E000228401339EE7DEF82C2002EBC00912F85A
:1075F0003020053A012A14D8002710E0E26A02EB95
:10760000C70812F83720062A08D1D9F80410D8F88C
:107610000420914204BFA8F8023001330137BC4571
:10762000ECD1013089E7E06A00EBC20110F83200CA
:10763000062802D14878C00702D5488818444880F7
:1076400001329445EFD1628B12FA83F26283228C6D
:1076500012FA83F3238475E70022F2E7B4040020D2
:10766000581006085C110608238B042B17D10F9BBA
:107670001BB9584604F036FC0F9000230D930322EB
:107680004A4B1093214604A8FEF7BAF9059B23B98B
:107690000422214604A8FEF7B3F9A468EAE6023BF7
:1076A000012B21D837B95B4607AA05A911A803F019
:1076B0007DFD0746CDE90D7A0222214604A8FEF79A
:1076C000F1FF059B002BE8D10322214604A8FEF719
:1076D000E9FF059B002BE0D10422214604A8FEF718
:1076E000E1FF0028F8D0D8E7019BCDE90D39E3E7A9
:1076F000B8F1000F7FF4C7AEDDF81490D5F8108014
:10770000B9F1000F16D0019800F0D3FD002F41D140
:107710000F9808B104F0FBFB0298FCF787FF28469E
:10772000AD68FCF7B3FF002DF9D10598002835D0DE
:10773000F8F778FD139C1898C4F3DC046400033454
:1077400000EB94008000F8F795FD24F00304044456
:10775000F460DDE91441B06001F1040CA1450BD1E6
:10776000189A00239342CED0199951F82300F1685A
:1077700041F823000133F5E751F839303BB1042BD0
:107780001FBF5CF839205210DB0820F8123009F1D5
:107790000109E3E7384603F02BFDB9E72A463146F5
:1077A00040461BB0BDE8F04F05F000B9381206089E
:1077B000F0B52DED028B884283B007460C4604D10C
:1077C000012003B0BDEC028BF0BD244B984201D1E7
:1077D0000020F6E79942FBD007F0ECFA0546204678
:1077E00007F0E8FA8542F3D11D4B9D4213D17A6828
:1077F00063689A42ECD13E1D043400257B68AB429D
:10780000DED954F8041F56F8040FFFF7D1FF002803
:10781000DED00135F2E72146384607F0A5FD002805
:10782000D6D0104B9D42CBD1384609F061FEB5EE63
:10783000400AF1EE10FAB0EE408AC1D1204609F0BC
:1078400057FE8DED010A18EE100A019B00F0004072
:1078500003F00043C31A58425841B2E774130608B4
:10786000F82A0608681D0608C90010B5012204465A
:1078700041F00201083007F06DF843683BB9A36896
:10788000C3F3DC03013B5B0043F001034360C3F33C
:107890004F0010BD70B505460E460024EB69A342AB
:1078A00008D8314605F114000BF0C7F8EC69013C2B
:1078B000204670BD2B6A314653F82400FFF778FF4D
:1078C0000028F5D10134E9E710B501220446FCF7A0
:1078D000F7FE0378012B05D12378012B8CBF0423FD
:1078E0000223037010BD70B505460E4610461946BA
:1078F0001C46FCF7D5FE03785A1E012A06D8736889
:10790000002221462846BDE870401847032B02D1CB
:1079100073680122F5E736684288042B2146284621
:10792000B44608BF0023BDE8704018BF012360477C
:107930004379012B07D083681944036981605A8C0D
:107940009142C8BF59847047002383714379012B4A
:107950001EBF036AC26A43F8212070476FF003011B
:10796000FFF7E6BF0421FFF7E3BF6FF00201FFF767
:10797000DFBF426A03464079032888BF586B114431
:1079800094BF1846801859627047827903460AB13D
:1079900018467047C26A40790328114401D8D96259
:1079A000F6E7986AD9620244586B1044704710B5E4
:1079B0000C460121FFF7E9FF047010BD10B5144615
:1079C000FFF7B6FF0121FFF7E0FF047010BD53225F
:1079D0000121FFF7F3BF54220121FFF7EFBF572228
:1079E0000121FFF7EBBF58220221FFF7E7BF592221
:1079F0004FF0FF31FFF7E2BF5A220021FFF7DEBF51
:107A00005B220021FFF7DABF5D224FF0FF31FFF765
:107A1000D5BF19B103215F22FFF7D0BF5E22FBE77C
:107A2000A1F13002D2B20021FFF7C8BF62226FF08D
:107A30000101FFF7C3BF10B5632204464FF0FF31C9
:107A4000FFF7BCFF0123A37110BD10B501F1640263
:107A50000446D2B24942FFF7B1FF0123A37110BD22
:107A600010B501F167020446D2B24942FFF7A6FF02
:107A70002269D38A43F00103D38210BD38B504468E
:107A80001D46FFF79BFF2A4620460249BDE83840C5
:107A900013F0F0BD8B79020870B504460D46C0683E
:107AA00019461646FFF7E0FE3246034629462046B1
:107AB000BDE87040FFF7E2BF0B4610220121FFF73F
:107AC000EBBF11320B46D2B20121FFF7E5BF20B464
:107AD0000B4602F114055100C1F10101EAB25DF853
:107AE000045BFFF7D9BF16320B46D2B24FF0FF311D
:107AF000FFF7D2BF19320B46D2B20021FFF7CCBF3D
:107B000070B4C4682678042E1D4608BF6668638872
:107B100008BF46F823505D1C658070BCFFF7AEBF00
:107B200003F128011346CAB20021FFF7A7BF022ABA
:107B300002F12A020B46D2B214BFC1F101010121A8
:107B4000FFF79CBF03290AD004290AD101210B4663
:107B50000A4443EA8203C9432F22FFF78FBF002163
:107B6000F5E700210223F3E70B4630220139FFF746
:107B700085BF10B4144641EA0223214431225DF846
:107B8000044BFFF77BBFF8B516461F46FFF7D0FE44
:107B90008479054604BB4379022B25D9C46A036A5C
:107BA000C4F1FF2453F8273004F57F04FE34442E3B
:107BB0001C4412D814F1400F14DB3F2CD4BF002713
:107BC0000127E41BB91C2846FFF7DFFE06706FB9DA
:107BD000442E98BF40344470F8BD7F2C94BF0027DA
:107BE0000127EEE70127ECE70127EBE76B79442E4D
:107BF00098BF04F58044042B05D1B4F5004F24BF91
:107C0000012385F8383064F07F03E41143708470F9
:107C1000E2E710B50B46044642220021FFF7B3FF0E
:107C20000123A37110BDF8B505460C4621F40047A9
:107C30001646CAB90B040ED55921FFF7B8FE5921D3
:107C40002846FFF7B4FE59212846FFF7B0FE592118
:107C50002846FFF7ACFE3B46422200212846FFF7AC
:107C600092FF0123AB71F8BD3B4640220021FFF794
:107C70008AFF210A21F07F013143C9B22846FFF76C
:107C800096FEEEE70B46B2FA82F120B4490902F102
:107C90004705EAB249005DF8045BFFF774BF0B4685
:107CA0004B220121FFF76FBF10B50B4604464A2255
:107CB0000021FFF768FF0123A37110BD264BD3F805
:107CC0001032022B2DE9F047044689460ED886690A
:107CD000B1420BD9C56A43698E1BED1A40F2FF779A
:107CE00056EA050304D1E36AC4E90539BDE8F08723
:107CF000062E01D90F2D1AD91F2DAA4628BF4FF0E5
:107D00001F0A1F2D10D8032EB04628BF4FF00308BE
:107D100001212046FFF72DFE4AEA48130370A5EB28
:107D20000A05A6EB0806DBE74FF00008F0E7BE42C5
:107D3000B0464FF0020128BFB8462046FFF719FEB3
:107D40004FEA181303F070032B4363F07F030370B3
:107D500080F80180AA46E2E7B404002010B504468A
:107D600031B955224FF0FF31BDE81040FFF726BE74
:107D7000022904D1FFF72BFE2046FFF741FE5622D1
:107D80006FF002012046EFE7134621B143224FF086
:107D9000FF31FFF7F8BE4422F9E7134621B145222F
:107DA0004FF0FF31FFF7EFBE4622F9E7322938B531
:107DB000044611D0332912D000252939CAB22046F1
:107DC0004FF0FF31FFF7FAFD65B12046D322BDE841
:107DD00038400021FFF7F2BD01250621EDE701251E
:107DE0000721EAE738BD012A10B40B46044608D043
:107DF000022A0ED15DF8044B69224FF0FF31FFF7E4
:107E0000DDBD11461B322046D2B25DF8044BFFF7B0
:107E100043BE4FF0FF31F5E770B50D4604461146FD
:107E20002AB92B461322BDE87040FFF735BE022A5F
:107E300004D1FFF7CCFD2046FFF7DEFD2B461822CC
:107E40006FF001012046EEE710B4044643B90F2A53
:107E500006D8503A5DF8044BD2B20121FFF7AEBD0F
:107E600003F12401204613465DF8044BCAB20121F8
:107E7000FFF704BE10B404464BB90F2A07D8403AA6
:107E80005DF8044BD2B24FF0FF31FFF797BD03F11D
:107E90002601204613465DF8044BCAB24FF0FF316D
:107EA000FFF7ECBD70B4DDE90365D2B203EB460425
:107EB00043EA062315B101320134D2B2091B70BC6A
:107EC000FFF7DCBD07B5CDE900230B4634220021C6
:107ED000FFF7E8FF03B05DF804FB07B5CDE9002329
:107EE0000B4636224FF0FF31FFF7DCFF03B05DF8A1
:107EF00004FB10B50446C068FFF7CCFC2322034600
:107F000001212046BDE81040FFF7B8BD01F1100384
:107F10003F2B73B506460C4608D8A1F18002D2B2B9
:107F2000012102B0BDE87040FFF748BD01212222C7
:107F30000DF10505FFF742FD294604F07F00E3B28D
:107F4000E4112A4605F8010D601C0128F5D801341A
:107F500003F0400314D11BB97F2305F8013C951EA3
:107F6000491B3046FFF711FD01AC6A1E014612F8AD
:107F7000013FA24208D11044401B037002B070BD03
:107F8000002BEDD00023E8E763F07F0301F8013B0D
:107F9000EDE770B51446D6B2049A134305460B6953
:107FA00007BF2022C4F10101E1432122FFF7A8FD10
:107FB00031462846BDE87040FFF7F9BC1A4308BFB8
:107FC00032220B6916BF332201214FF0FF31FFF738
:107FD00097BD00000D2910B504460BD10949C068B2
:107FE000FFF758FC2322034601212046BDE810403C
:107FF000FFF744BD4231CAB2BDE810400121FFF78E
:10800000DDBC00BF8826060838B504460D460F21A2
:10801000FFF7E0FF20462946FFF796FC02215C228D
:10802000FFF7CCFC20466FF00301BDE83840FFF7B6
:108030007FBCF8B504460F460F211D461646FFF7D4
:10804000C9FF2046FFF7D8FC39462046FFF7E1FD7F
:1080500031462046FFF778FCFFF7C1FC012220469D
:108060002121FFF72EFD20460821FFF79FFE2A461B
:1080700020460021BDE8F840FFF786BE4379012B7A
:1080800070B5044614D0C26B436A00259B1AC363C3
:1080900005642069038DAB420CD86379032B1BD197
:1080A000606AE36AA06223631844F8F7FCF860632F
:1080B000012070BDC36A03EBC50213F83530052BF0
:1080C00008D1012120469678FFF753FC0670236CF7
:1080D000013323640135DCE7042BE9D1D4E90A1329
:1080E000626A8A4202D1216B994203D0A262236361
:1080F0000020DEE794F838301BB10649064805F049
:1081000095F8E268C38A5268616B006904F033FC39
:10811000CEE700BFF1BD05085C1A06082DE9F74F50
:1081200016460023C0E90423378C83608371C36241
:10813000436280F83830738CB6F82490B6F81A8011
:10814000B6F816A0B6F81EB0417101221F4497423E
:10815000B8BF17464FEA8905013F826105F0040563
:1081600008F003021543FA0002F07802B38B0446CC
:108170000AF00F0A15433F094FEA59094FEA9808D8
:1081800047EA090242EA0A0242EA08021A4352EAAC
:108190000B0234D101212046FFF7EBFB0570637918
:1081A000022B18D9D4E90F787D0008F0010305F0FF
:1081B0007E054FEA5808BF091D4358EA07094FF0EA
:1081C0000101204618BF45F08005FFF7D2FB05707E
:1081D000B9F1000FE8D1636AB18AE363E068FFF7A1
:1081E00043FB2B490246204613F044FA0025738BCB
:1081F000B28B1344AB4248DD318D002241E00121B6
:1082000020460193FFF7B5FB65F07F053A01057045
:108210004FEA8A15019B02F0300205F04005154334
:108220000BF001021543DA0002F0080215434FEA91
:10823000880202F0040215434FEA490202F00202EA
:108240001543BF084FEA59094FEA5A0A4FEA58083E
:108250005B084FEA5B0B93E7F36A03EBC2035878C2
:10826000C0070DD55888A8420AD15968E068FFF7C1
:10827000FBFA07490246204613F0FCF90135B6E740
:1082800001329142E8DC0521F0E703B0BDE8F08F50
:108290007379020810B504464420F8F704F8C46066
:1082A00010BD10B50446C1618800F7F7E3FF2062F6
:1082B00010BD10B50446006AF8F704F82046BDE882
:1082C0001040F7F7FFBF10B5044601618800F7F7CB
:1082D000D1FF606110BD10B5044611B1C068F7F759
:1082E000F1FF6069BDE81040F7F7ECBF012938B530
:1082F00004460D460BDC0269406992004FF0FF31E5
:1083000022F004FA002325706370636038BD406872
:10831000F7F7B0FF6368E060A360F3E702464078D8
:1083200010B548B913785468022B08BFD3682144AC
:1083300008BF1819516010BD0020FCE700234370EE
:108340000378012B9EBF4369426843F821207047A0
:1083500042684B1E134449420B404360704738B596
:108360000C461546FFF7DAFF10B10444A04200D1D5
:1083700038BD00F8015B2D0AF8E710B50C46022164
:10838000FFF7CCFF10B10470240A447010BD38B55B
:108390000D4604211446FFF7C1FF28B10570847013
:1083A0002D0A240A4570C47038BD012970B50546F0
:1083B00006DC002909DA023921F00104FE2606E074
:1083C0008B1E012BF7D80024F8E70024F22646F490
:1083D00035412846FFF7D1FF44B17F2C09D844F43A
:1083E000304141F080012846FFF7C7FFC5E9066428
:1083F00070BDA300A201DBB202F4E0421A4342F4D2
:1084000050624FF2AD212846FFF7C1FFEEE7C16988
:1084100010B5044629B17F290BD841F43041FFF74C
:10842000ACFFA169204641F43D41BDE81040FFF793
:10843000A4BF8B008A01DBB202F4E0421A4342F48B
:1084400050624FF20D21FFF7A2FFEAE7114341EA24
:10845000C301FFF792BF072A85BF083AD200D200B6
:1084600042F04002072985BF08391143114341F00A
:10847000800141F48C41FFF780BF30B4DCB244EAA4
:1084800002225C101D0104F48064C3F3033305F47D
:10849000E04523432A43194330BCFFF778BF38B582
:1084A000436953F821404368E41A043C0546C4F389
:1084B0004A0141F46041FFF760FF2B78022B0AD19B
:1084C000B4F5006F07D36FF30A0414F5006F14BFFF
:1084D0000020012038BD0120FCE7F8B5446954F8BC
:1084E00022404268A41A043C074665101E46BBB9E8
:1084F000EDB245EA012141F45041FFF73EFF3B78E0
:10850000022B0BD1FF2C09D924F0FF0414F5807F36
:1085100014BF0024012426463046F8BD0124FAE7A2
:108520006211C5F30A0502F400522A43A512231270
:1085300005F48065C4F3053403F4006325431A434E
:1085400045EA811142F4004241F47041FFF71FFFF8
:10855000E2E738B5436953F821404368E41A043C24
:108560000546C4F34F02C4F30A3142F4784241F4A1
:108570007041FFF70CFF2B78022B0AD1B4F5800F66
:1085800007D36FF3150414F5800F14BF00200120EA
:1085900038BD0120FCE7F8B5476804460D4616468D
:1085A00013460A464FF24021FFF767FF2046330C7F
:1085B0002A464FF2C021FFF760FF3846F8BD072971
:1085C00010B4044609D8FF2A07D842EA01215DF811
:1085D000044B41F40051FFF7D0BEB2F5803F08D202
:1085E000134620460A465DF8044B4FF24021FFF740
:1085F00044BF20465DF8044BFFF7CDBF2DE9F8439B
:1086000041EA0207072FDDF8209006460C46154682
:108610004AD803FA09F7FF2F0CD8914201D0FFF78F
:108620001AFF47EA042141F440513046BDE8F843BF
:10863000FFF7A3BEFF2B4FEAC10814D8914218D010
:1086400043EA012343F40051FFF797FE44EA8911FE
:1086500041EA08013046FFF790FE48EA85112143C0
:1086600041F4C051E1E7914203D03A46FFF7A7FF3A
:10867000F3E784F00709012505FA09F545F43441CB
:108680003046FFF77AFE3A4649463046FFF797FFF5
:1086900044EA891141EA080141F4C0513046FFF72C
:1086A0006CFE45F43C41C0E7BDE8F88308B50378AB
:1086B000012B04D9FF2902D9054805F0A5FDC9B24F
:1086C00041EA0221BDE8084041F41041FFF755BEE0
:1086D000FCBD050808B50378012B04D9FF2A02D98F
:1086E000054805F091FDD2B242EA0121BDE80840FB
:1086F00041F41841FFF741BEFCBD0508D2B242EA81
:10870000012141F42841FFF738BE38B5436953F8D9
:10871000223042689B1A43F001030C4605460A4684
:108720000A3B4FF24021FFF7A8FE23462846224687
:108730004FF43241FFF78AFE210101F0800104F07D
:108740000704214341F48841284641F07801BDE8FF
:108750003840FFF712BE000073B51F2B069E05467A
:108760000C4611D8114307290ED81A49895D44EAED
:10877000C20241F0010142EAC12141EA831102B083
:10878000BDE87040FFF7F9BD03FA06F1B1F5805F6F
:108790000DD242EA461641EA043246F4784141F0ED
:1087A0009001284602B0BDE87040FFF7F0BD1F3BC6
:1087B000214628460096FFF721FF064B9B5DE1000E
:1087C00043F0010341EAC321214341F4F861284603
:1087D000D5E700BF301106082DE9F7431F2B0A9F8C
:1087E00006460C461546984610D841EA0203072B68
:1087F0000CD8204BD95D44EAC12141EAC20141EACB
:10880000881103B0BDE8F043FFF7B7BD08FA07F2DF
:10881000B2F5805F0DD245EA471141F4784142EA52
:10882000043241F08001304603B0BDE8F043FFF769
:10883000AEBD4FF0010909FA05F949F4344130465B
:10884000FFF79BFDA8F11F032A46294630460097F3
:10885000FFF7D4FE074BDB5D44EAC50141EAC321C3
:1088600041F4F8613046FFF788FD49F43C41304659
:10887000C7E700BF30110608436953F82110436869
:10888000CB1A043B013110B4C3F34A0204460ED0A4
:10889000D91C0CDA23F4FF6121F0070111F5006FF8
:1088A00005D15DF8044B42F46041FFF766BDC3F3A8
:1088B0000A33204642F438425DF8044B43F47041D9
:1088C000FFF765BD436953F822204368D31A043B80
:1088D000013230B405464FEA63040ED0DA1C0CDADC
:1088E00023F0FF0212F5807F07D1E4B244EA0121B0
:1088F00041F4504130BCFFF740BD5A11C4F30A04A3
:1089000002F4005222439C12181204F48064C3F350
:10891000053300F400602343024343EA81112846F3
:1089200042F4004230BC41F47041FFF730BD37B52E
:10893000144602220B460092214607220546FFF705
:108940000BFFE10041F48F41284603B0BDE8304001
:10895000FFF713BD07289ABF024B33F8100040F20F
:108960003B20704734110608C36C19440369C16485
:10897000012B04DD436D5A8C9142C8BF5984704766
:1089800070474FF0FF31FFF7EFBFFFF7FABF6FF00F
:108990000301FFF7E9BF704738B5C36C1944036A98
:1089A0009942054608D9083121F00304406AE100E4
:1089B000F7F77BFCC5E9084038BD70B504460E46A4
:1089C00001211546FFF7E8FFE16C626A02EBC10383
:1089D00002F83160012159705D602046BDE87040A9
:1089E000FFF7C2BF70B504460E4601211546FFF7DA
:1089F000D3FFE16C626A02EBC10302F8316002222C
:108A00005A705D6020460121BDE87040FFF7ACBFA1
:108A100000221146FFF7E6BF0A460221FFF7E2BF38
:108A200070B50D1E044605DDFFF7B6FF00231E4698
:108A3000AB4205DB29462046BDE87040FFF794BFF6
:108A4000E26C616A1A4401EBC200012D46700CBF52
:108A500094F82800002001F832000133E8E7F8B567
:108A6000D0E90B530133AB4204460E46174606D9F4
:108A70000435406BA900F7F718FCE5626063D4E9A0
:108A80000C30C6F30E015A1C226300EB830541EA49
:108A9000C73220F823204FF6FF73A06D6B8032465B
:108AA0000021FFF732FEA06D0022BDE8F84003214F
:108AB000FFF7FCBD0246007D28B1D36C526A5B1AF9
:108AC000013B12F83300704737B5456DED8AED076D
:108AD0000B46144608D502220092806D06222146DC
:108AE000FFF77AFE03B030BD806D03B0BDE83040C3
:108AF000FFF7DCBD70B5002405462646EB6CA342AB
:108B000000DC70BD6B6A03EBC4035A78012A07D1FD
:108B10005E70B5F84A105A6821442846FFF7D4FF22
:108B20000134EBE7F8B504461E4617460D46FFF73D
:108B3000E1FFA06D3A463146FFF741FDA06D2946A1
:108B40000322BDE8F840FFF7F2BE38B504460D46F3
:108B5000FFF7D0FFA06D29460322BDE83840FFF79C
:108B6000E6BE10B508210446FFF7EFFF00222046BD
:108B70001146BDE81040FFF720BFF8B50446174680
:108B80001E460D46FFF7B6FFA06D3A460021FFF7DF
:108B900016FDA06D32460121FFF711FDA06D29469B
:108BA0000322BDE8F840FFF7C2BEF8B5C76C044623
:108BB0000E46BF1A0025E36CAB4200DCF8BDBD4297
:108BC00011D0636A03EBC5035A78012A0BD15A68A6
:108BD000B24208D100225A70B4F84A1032462944F1
:108BE0002046FFF771FF0135E5E738B5002205465D
:108BF0000C461146FFF7D9FFE200A86D42F00202D1
:108C00000021FFF7DCFC002228461146BDE8384071
:108C1000FFF7D3BE13B5446DE48AE407134607D5C6
:108C200002220092806D0622FFF796FD02B010BD71
:108C3000806D02B0BDE81040FFF74CBDF8B5C369C8
:108C40009E5C602E0446154606D1476813480A46C6
:108C5000134908F0A5FA3860022D0DD8636D9A8C7F
:108C600052B9DB8ADB0707D40E4B5A5D31462046EA
:108C7000BDE8F840FFF7A1BE002211462046FFF7ED
:108C800094FFB4F84A20636C1A44521B013A002145
:108C90002046FFF7BFFF0022E8E700BFA81906083B
:108CA0000EBE05083412060873B503681A785D888D
:108CB000042A04BF5A6842F825106A1C044602269A
:108CC0005A800021B0F84820FFF7A4FF0096002248
:108CD000A06D33461146FFF73FFD00960022A06DC0
:108CE0002B461146FFF738FD02B070BD73B5002268
:108CF00004460D461146FFF758FF626D2068D38A7F
:108D000043F02003D3822946FEF7C4FD0226B4F8BF
:108D10004820054600212046FFF77CFF00960022F0
:108D2000A06D11460123FFF717FD00960022A06DEC
:108D300011460323FFF710FD00960022A06D114697
:108D40002B46FFF709FD00221146204602B0BDE880
:108D50007040FFF732BE00000D2902D10749FFF72E
:108D6000C5BF0F2903D100225421FFF73BBEB1F14B
:108D70000E0218BF01220121F7E700BF882606086E
:108D8000F8B5C76C446A07F10053023B04EBC30417
:108D90000546D4E9020184E80300667856B9B5F8BF
:108DA0004A203A44013A31462846FFF733FF01236F
:108DB0006370666028464FF0FF31BDE8F840FFF76A
:108DC000D3BDF8B504461E4617460D46FFF792FE82
:108DD000A06D3A463146FFF7F2FBA06D294603220B
:108DE000BDE8F840FFF7A3BD10B402F12904002349
:108DF0000A46E1B25DF8044BFFF7E3BF70B50446E5
:108E00000E46154662B1037D53B1084605F0E8FBF6
:108E1000021E05DD20467021BDE87040FFF7E2BD6F
:108E200006353246E9B220460023FFF7CAFF00228A
:108E300020461146BDE87040FFF7BFBD07B5134699
:108E4000022200920722FFF787FC03B05DF804FBC3
:108E500038B50D4614463BB9037D2BB1806D526881
:108E6000FFF7ADFB207838BD237833B96268806D99
:108E70002946FFF7A4FB0020F5E7012B06D1626825
:108E80000132806D2946FFF7D9FFF4E79A1E012AC7
:108E900004D86268520042F00102E8E7542B01D185
:108EA0000022EEE7014805F0AFF900BF23BE050838
:108EB000F8B50546FFF71EFE00242746EB6CA342DB
:108EC00000DCF8BD6E6A06EBC4025378022B0ED1AB
:108ED0005770012100232846FFF7BAFF06F8340037
:108EE000B5F84A10012221442846FFF7EDFD013470
:108EF000E4E738B504460D46FFF7DAFFA06D2946D2
:108F0000FFF7BAFCA36D01225A7038BDF8B50446CC
:108F10000E4617460A4619461D46FFF746FEE36C05
:108F2000616A9B1B01EBC30211F833303B7053782D
:108F3000012B0DD0022B14D0CBB9B4F84A20E36C2E
:108F40001A44921B29462046BDE8F840FFF762BE4E
:108F50005268AA420BD0A06D2946BDE8F840FFF741
:108F60007ABA002329462046FFF772FF3870F8BD11
:108F700010B5134604460A460121FFF7C7FF2046F5
:108F80004FF0FF31BDE81040FFF7EEBC70B5049E16
:108F900004461D46FFF7ECFF324629462046BDE851
:108FA0007040FFF7E5BFF0B585B001250DF10F0367
:108FB0000DF10E01009500220446FFF7E7FF9DF832
:108FC0000F709DF80E602A4639462046FFF7F5FCE3
:108FD000314620460022FFF7F0FC2A46394620465B
:108FE000FFF7EBFC00223146204605B0BDE8F0401B
:108FF000FFF7E3BC2DE9F041DDE9068604461D4696
:10900000089FFFF7B5FF424629462046FFF7B0FF0D
:109010003A4631462046BDE8F041FFF7A9BF2DE9A9
:10902000F04186B002260DF11703012501930DF1E1
:1090300015010DF116030296009500220446FFF774
:10904000D9FF9DF817809DF815109DF816702046E1
:109050000022FFF7B2FC324641462046FFF7ADFC46
:109060002A463946204606B0BDE8F041FFF7A5BCC8
:1090700030B587B00DF11703002501930223044694
:10908000009301220DF116030DF115010295FFF772
:10909000B1FF20461921FFF758FD2A4629462046F0
:1090A00007B0BDE83040FFF788BC73B504460E46F4
:1090B000154672B901220DF10701FFF759FF0C3572
:1090C00000233246E9B2204602B0BDE87040FFF707
:1090D00078BE0021FFF7EEFC20B901220DF1070157
:1090E0002046EAE70A4620460DF10701FFF740FF58
:1090F0009DF80720204601230421FFF713FDA06DF2
:1091000000220121FFF7A7F9D9E7000037B50022B7
:109110000DF107010446FFF72BFF9DF807302BB137
:1091200007490848656808F03BF828602221204676
:10913000FFF70BFDA36D01225A7003B030BD00BFD5
:1091400031BE0508A8190608022A7FB504460E4656
:10915000154614D8436D9A8C8AB9DB8ADB070ED486
:10916000184B0DF10F015A5DFFF702FFE3699DF8FF
:109170000F10585D602813D1595504B070BD0DF122
:109180000F0120460022FFF7F3FE626CB4F84A306C
:1091900013445B1B0022591E2046FFF795FCE5E7B0
:1091A0008842EAD0FFF7D6FB02460846FFF7D2FB1B
:1091B00005496468009013460448324607F0F0FF02
:1091C0002060DAE7341206083BBE0508A819060835
:1091D00070B504460D4616464BB90F21FFF7BCFD8E
:1091E000324629462046BDE87040FFF7ADBF70BD4E
:1091F00003297FB50446164613D101220DF10F0154
:10920000FFF7B6FE18253146204600230DF10F0268
:10921000FFF77CFE2946204604B0BDE87040FFF70A
:1092200094BC052906D101220DF10F01FFF7A0FE24
:109230001725E8E70223009301220DF10F030DF13A
:109240000E01FFF7A3FE1925DDE7F0B5044685B052
:109250000E461546CAB90223077D02750DF10E01AF
:10926000009301220DF10F03FFF790FE27752B46A7
:10927000324623212046FFF7A4FD00221146204656
:1092800005B0BDE8F040FFF798BB012A09D10023E3
:109290000DF10F022946FFF739FE2B4632462421F5
:1092A000E8E70DF10F010022FFF762FE25212046BD
:1092B00005B0BDE8F040FFF748BC10B50446D0E962
:1092C0000C3003F18043013B00EB8303DA7822F09A
:1092D0008002DA70043B98420BD893F90320002AED
:1092E000F8DA1A88A06DC2F30E020021FFF70DFA1A
:1092F00005E059B9A06D4FF40051FFF73EF8A06D9D
:109300000022BDE810400321FFF7D0B910BD10B511
:1093100004460121FFF7D1FFA06D01220021FFF7D4
:10932000D9F9002220461146BDE81040FFF745BBA1
:1093300073B5046B05460E46DCB1436B04F1804403
:10934000013C03EB840292F90120002A20DA33F871
:109350002430C3F30E038B421AD100230DF1070210
:109360000121FFF7D3FDA86D00220121FFF79EF92F
:1093700001242846FFF79CFDA86D3146FEF7DEFF6D
:1093800044B10021284602B0BDE87040FFF795BF08
:109390000024EEE702B070BD38B50D460446114614
:1093A0007AB1806D4FF40051FEF7E7FFA06D002207
:1093B0000121FFF77BF929462046BDE83840FFF739
:1093C00098BDFFF77AFFF6E72DE9F04104460D4618
:1093D00072B3D0E90C3C03F18043013B0CEB8303F7
:1093E0000021184616460F4690F901E0BEF1000F25
:1093F00009DA90F903E0BEF1000F04DA002F08BF8C
:109400000746E1B90146013EA0F10400ECD1A06D90
:1094100021BB6FF0030672439E18B44518D94FF470
:109420000051FEF7AAFFA06D00220321FFF73EF9CD
:1094300025F400412046BDE8F041FFF75ABDB0F8E1
:109440000080B1F802E068F30E0EA1F802E0D9E75F
:109450009A5AC2F30E02FFF758F9E4E74B8847F631
:10946000FE7262F30E034B8025F400423146FFF793
:109470004CF9A06D32461321FFF718F9A06D324662
:109480003146FFF79CF8A06D32460121FFF70EF937
:109490003D88C5F30E05CBE77FB504460E4615465D
:1094A0008AB90DF10F01FFF763FD32462046012313
:1094B0000921FFF786FC2A462946204604B0BDE86C
:1094C0007040FFF77ABA012A35D11146FFF7F2FA58
:1094D000024688B9022300930DF10E010DF10F032E
:1094E0002046FFF753FD012332460E21204604B0EB
:1094F000BDE87040FFF765BC0DF10F022046002368
:109500000221FFF703FD2B469DF80F202046042182
:10951000FFF708FBA06D00220221FEF79CFF0DF172
:109520000E0120460022FFF723FD4FF0FF312046B9
:10953000FFF71AFAD7E70DF10F010022FFF718FD28
:10954000A06D4FF40851FEF718FFCCE738B5FFF7D0
:1095500018FA04460122806D0021FFF7BBF8222192
:109560002046FFF7F2FAD4E90C35013B05EB830501
:1095700023636B8847F6FF72C3F30E03934228D030
:109580001322A06D0021FFF7A5F8A06D4FF4205124
:10959000FEF7F3FEA368A06D1A680021FFF792F9A9
:1095A000698847F6FE73C1F30E029A420BD1A06D93
:1095B0004FF48E41FEF7E1FEA36820461968BDE82E
:1095C0003840FFF7B5BEC1F30E012046FFF791FC0E
:1095D000F2E738BD2DE9F3410E4600211746044657
:1095E0001D46FFF767FA024648BB0DF1070120460A
:1095F000FFF7BEFC1DB901212046FFF7B5F9102188
:109600002046FFF7A2FA1DB99DF8073084F82830EC
:109610002046FFF74DFCA06D4FF420515EB3FEF7DE
:10962000ACFE3A460121A06DFFF74CF945BB4FF067
:10963000FF31204602B0BDE8F041FFF795B90A4678
:1096400020460DF10701FFF793FC1DB901212046CB
:10965000FFF78AF99DF80700431E022BD3D9FFF7C5
:1096600079F90949D4F804800246084807F098FDC2
:10967000C8F80000C7E7FEF780FE3A463146D2E759
:1096800002B0BDE8F08100BF4BBE0508A81906086E
:109690000023FFF79FBF0123FFF79CBF426D836844
:1096A0002DE9F341D58A928C1E68C66005F011033E
:1096B0001343044600F0F98015F0010506F1020796
:1096C00021D1B0F8482029464FF00208FFF7A2FA4E
:1096D000CDF80080A06D01232A462946FFF73CF80B
:1096E000CDF800802A46A06D01232946FFF734F803
:1096F00005212046FFF729FAB4F848102A4601311F
:109700002046FFF7E1F9D4E915309A8C002A67D199
:10971000D98A11F0010508D14FF42051FEF72DFE32
:10972000A06D3A462946FFF7CDF800221146A06DFC
:10973000FEF7E4FF20212046FFF707FA4FF42051FF
:10974000A06DFEF71AFE3A460021A06DFFF7BAF8A9
:10975000636DD98A11F0010100F08E80A06D0122A5
:1097600000210225FEF7B6FF0095A06D0523062215
:109770000021FFF731F8A06D2A460021FEF71FFFF8
:10978000A06DFEF744FE39462046FFF7D1FD636D1C
:10979000DB8ADB0740F18980B4F84820204601329B
:1097A0000021FFF737FAA06D4FF48E41FEF7E5FD7B
:1097B000A06D4368236414220021FEF78BFFA06D87
:1097C0004FF40451FEF7D9FDA06D01221421FEF7DC
:1097D0006DFF2221204602B0BDE8F041FFF7B5B988
:1097E0004FF40051FEF7C9FDA06D00221321FEF7D2
:1097F0005DFFA06D00220121FEF758FF751C3A465F
:10980000A06D0421FEF781FF29462046FFF790FD59
:1098100000221146A06DFEF771FF20212046FFF7C0
:1098200094F90336A06D4FF42051FEF7A6FD3246A1
:10983000A06D0121FFF746F8A06D4FF40051FEF72F
:109840009CFD0022A06D0321FEF730FFA06D44F2C5
:109850002071FEF792FD31462046FFF769FD032295
:10986000A06D0421FEF736FF4FF43051A06DFEF7D6
:1098700084FD2A46012168E7B4F8482020460132D9
:10988000FFF7C8F905212046FFF75FF9D4E9153045
:10989000D98A11F001017FF461AF0122FEF71AFFAE
:1098A00022212046FFF751F96DE702B0BDE8F081B3
:1098B00070B50546D0E91560F68AF6070C460BD55B
:1098C00044EAC4049200FEF77AFEA86D44F4CC5139
:1098D000BDE87040FEF751BDBDE87040FEF70EBF19
:1098E0002DE9F84F04460F469146FFF703F900258E
:1098F000A8464D4510D10026B3464E452BD17142A6
:109900002046FFF731F8B4F84A20E36C39461A4490
:10991000BDE8F84FFFF7CCBFE66CD4F824A0013EB9
:10992000761B0AEBC6025378022B12D182F8018013
:10993000012339462046FFF78BFA0AF83600B4F8BF
:109940004A10E36C194401393A46491B2046FFF797
:10995000BBF80135CDE7E36CD4F824A003F1FF3860
:10996000A8EB06081AF83820BAB1B4F84A501D44DA
:10997000013DAD1B2A4600212046FFF74BF91AF89E
:109980003820012304212046FFF7CCF80022294685
:109990002046FFF799F80AF838B00136ADE7000025
:1099A000037D37B504460D4613B15F4804F02CFC27
:1099B000426DD38A43F00103D382FFF779FA012D78
:1099C0000BD1A368196820460231FFF792FAA36809
:1099D000196820460131FFF7ABFC01220021204627
:1099E000FFF77EFF002202212046FFF76DF8A06DF1
:1099F00001220021FEF7E3FDA06D00221221FEF7F7
:109A000055FEA368A06D1A680021FEF77EFEB4F82B
:109A10004810002201312046FFF756F8E168A06D9A
:109A2000FEF72AFFA368A06D1968FEF787FC236B79
:109A3000BBB1626B03F18043013B02EB83039A42AB
:109A40000FD893F90310002926DA1A88A06DC2F303
:109A50000E020021FEF759FEA06D00220321FEF741
:109A600025FE01212046FEF7DBFFBDB9A06D1422C3
:109A70002946FEF72FFEA06D4FF40451FEF77DFC42
:109A8000A06D01221421FEF711FE2221204603B011
:109A9000BDE83040FFF759B8043BD0E7A368196828
:109AA00020460231FFF744FCA06D14220221FEF78C
:109AB00011FEA06D00220121FEF781FDA06D0122A3
:109AC0001421FEF7F3FD0DF1070120460122FFF7F7
:109AD0004FFA00230DF1070220460121FFF716FA85
:109AE000204602220021FEF768FF012220460221C3
:109AF000FFF7F6FE20463021FFF727F8A06D4FF460
:109B00002051FEF73AFCA368A06D1A6801210132CA
:109B1000FEF7D8FE20460121FEF782FF204603B063
:109B2000BDE83040FFF72CB961BE0508F8B5164610
:109B300004460D46520093B1CB1C1A440221FFF794
:109B4000CFFE45EA062301221D212046FFF715F826
:109B5000002220461146BDE8F840FEF72EBF8B1CC0
:109B60001A440221FFF7BCFE33462A461C21ECE7CB
:109B70002DE9F74304460F4616460121B0F8482068
:109B8000DDF828904FF002081D46FFF743F8012347
:109B9000CDF80080A06D1A461946FEF7DDFD55EAA6
:109BA00009052DD12046FEF7A5FFA06D2A464146A6
:109BB000FEF705FD39692046FFF776F8A06D032210
:109BC0001A21FEF7B4FEA06D32460121FEF7F7FC24
:109BD000324602212046FFF783FE25B16FF00101D6
:109BE0002046FEF7C1FEA06D03222B21FEF79FFE4B
:109BF00000221146204603B0BDE8F043FEF7DDBE6B
:109C000006F102094A4641462046FFF769FE4946E9
:109C10002046FEF7A9FEFEF76DFFCBE72DE9F341E5
:109C2000044615460F46B0F8482001214FF00208BF
:109C30001E46FEF7EFFF0123CDF80080A06D1A4607
:109C40001946FEF789FD354318D12046FEF752FF2D
:109C5000A06D2A464146FEF7B2FC39692046FFF75F
:109C600023F8A06D03221A21FEF761FE002211469F
:109C7000204602B0BDE8F041FEF79FBE20464246B6
:109C80004146FFF72DFE2046FEF734FFE5E770B5AD
:109C9000042A86B004460E4615462AD102294FF002
:109CA000000518D101220DF1170100950DF11603E1
:109CB000FFF76CF9A06D2A463146FFF7BFF8262161
:109CC0002046FEF742FF00221146204606B0BDE8BE
:109CD0007040FEF772BE0DF115030193012300934E
:109CE00002950DF1160302220DF11701FFF782F91B
:109CF000E5E7012A01D9032A04D132460121204691
:109D0000FFF7EEFD133500233246E9B22046FEF799
:109D100009FFD8E738B5042204460D460021FFF7B5
:109D2000DFFD20460421FEF71FFE1F21FEF70DFF79
:109D3000A06D4FF42051FEF720FBA06D2A460021B4
:109D4000FEF7C0FD002220461146BDE83840FEF770
:109D500034BE37B504460D460021FFF7AEFA204663
:109D60004FF0FF31FEF700FEA36819680231FFF7DC
:109D7000DFFA204600225421FEF734FE204600225E
:109D80005421FEF72FFE204600225421FEF72AFE22
:109D9000204605220221FFF7A3FD032220460023CF
:109DA0001C21FEF7EAFEA36820461968FFF7A1F818
:109DB000A06D2946FEF7C2FA20460121FFF77DFA81
:109DC00020460221FEF72CFEA06D01220021FEF7A5
:109DD00081FCA06D4FF42051FEF7CFFAA368A06D6F
:109DE0001A68022502320021FEF76CFD002300955F
:109DF0001A46A06D0121FEF7AFFC2046012200218A
:109E0000FEF7DBFD002211462046FEF7D6FD204678
:109E100000225421FEF7E6FD294620460522FFF7E1
:109E20005FFD0023032220461C21FEF7A6FE2046EC
:109E30001021FEF78AFEA06D4FF42051FEF79DFA27
:109E4000A368A06D1A6800210132FEF73BFDA368EC
:109E500020461968FFF76CFAA06D4FF40051FEF729
:109E60008CFAA06D00220121FEF720FCA36819687E
:109E700020460131FFF75CFA0121204603B0BDE81E
:109E80003040FEF771BD0000436D73B5DD8A15F0FB
:109E90000106044613D001220021FFF721FD002214
:109EA00002212046FEF710FE0022A06D1146FEF7AB
:109EB00086FBA06D00221221FEF7F8FB1BE0027D5D
:109EC000002A47D03146FEF7F5FD5428C5F3871523
:109ED00025D12046FEF755FDADB9A06D2A4629468D
:109EE000FEF7ACFF636D9A8C002AE2D1DB8A03F0A7
:109EF0001103002BDDD1226BE168204602B0BDE8E2
:109F00007040FFF761BAA06D32463146FEF757FB4D
:109F100001232A4604212046FEF704FEE2E70DF164
:109F2000070132462046FFF723F89DF80710A942A3
:109F30000DD02846FEF70EFD02460846FEF70AFD44
:109F4000074966680346074807F02AF93060002D84
:109F5000C8D0DDE70DF10701FFF70AF8C2E700BF3F
:109F600069BE0508A8190608F8B5164604460F4646
:109F7000FEF7C0FD31462046FEF70EFD0025E36CDE
:109F80002A46B5420CD1B4F84A20394620461A4434
:109F9000FFF78EFC29462046BDE8F840FEF7E4BCFA
:109FA0005819616A013521F83020EAE773B50D468A
:109FB00016460DF1070100220446FEF7D9FF721C78
:109FC0002A4420460221FFF7CFFF012345EA06225B
:109FD0002821204602B0BDE87040FEF7A3BD37B58A
:109FE00004460D4600220DF10701FEF7C1FF2A4687
:109FF00020460221FFF7B8FF01232A4627212046E9
:10A0000003B0BDE83040FEF78DBD37B50D460022E8
:10A010000DF107010446FEF7ABFF5DB120460422B7
:10A020000121FFF7A1FF1E21204603B0BDE830400B
:10A03000FEF78BBD2A46A06D0121FEF7C0FA20462F
:10A040001E21FEF782FD2A462946204603B0BDE8C0
:10A050003040FEF7B2BC37B504460D468AB1032244
:10A060000121FFF73DFC022201212046FFF77CFF82
:10A0700000232A460B21204603B0BDE83040FEF7FE
:10A08000A0BE0DF10701FEF773FF02221146204624
:10A09000FFF76AFF01232A460A21ECE77FB5012575
:10A0A00004460DF10F030DF10E0100950022FEF79D
:10A0B0006DFF9DF80E109DF80F6020460022FEF700
:10A0C0007CFC2A463146204604B0BDE87040FEF7CD
:10A0D00074BCF8B504460F4601211D461646FEF72E
:10A0E0009FFC2046FFF7DAFF0F212046FEF734FEE3
:10A0F0002046FFF7D3FF39462046FEF7FAFE2046FA
:10A100004FF0FF31FEF78CFC31462046FFF710F987
:10A110002046FEF736FCA06D01220021FEF7DAFA98
:10A12000002211462046FEF748FCA06D4FF4205156
:10A13000FEF723F9A06D2A460021BDE8F840FEF79E
:10A14000C1BB0000138B2DE9F34104460161D81E09
:10A1500043424341237500230E46E364118CA369F7
:10A1600062658B42154605D2E069F6F79EF82B8CA6
:10A17000E061A361626D538B928B1344EA8A5107AD
:10A1800048BF013392074FF0000248BF0133114628
:10A19000934240F0DB80227D002A40F0EB80A269F0
:10A1A0009A4200F2E980226A002360219A4240F03C
:10A1B000EC80042E14BF01210221A06DFEF796F859
:10A1C000626D0023A4F84830938CD28A02F011010A
:10A1D000194305D0D20740F1DD801523A4F848309B
:10A1E0008B492068FDF756FB2F8C6B8C94F81480FC
:10A1F0003B4406466364A06DB8F1000F00F00C818B
:10A20000626D918C002940F0CA80D28A12F0010F51
:10A210000CD13946032F6F8BA8BF0321032F88BFB2
:10A2200001F1FF3112F0110F00F0BB80B4F84820AB
:10A23000023292B2A4F84A201A44511A0227FEF7B9
:10A24000B4F80097A06D012300220721FEF784FADD
:10A25000072200971146A06D0323FEF77DFA07221F
:10A26000009733461146A06DFEF776FA636D9A8C1F
:10A270001AB9DB8A03F030032BB1B4F84810A06D93
:10A280000022FEF713FAA06D01220021FEF7E3F889
:10A29000A06D02220121FEF7DEF80322A06D062147
:10A2A000FEF7D9F8A06D4FF42451FEF766F8A368C5
:10A2B000A06D1A6801210432FEF704FB6A8BA06DC1
:10A2C0000221FEF77CF9A06D022300224FF48541A4
:10A2D000FEF7BCF8A368A06D1A6800210532FEF7EE
:10A2E000F1FAA368A06D19680431FEF727F86B8BAB
:10A2F000A06D4FF002125A430221FEF760F9A06DE3
:10A3000003222C21FEF713FBA368A06D1968053109
:10A31000FEF714F800250226636D5A8BAA4248DC2A
:10A32000032A0DD99A8C5AB9DB8ADB0708D4B4F812
:10A330004A20636CA06D1A44033A0621FEF7CAF95D
:10A34000204602B0BDE8F041FFF7A8B9E0698154AA
:10A3500001321DE7C86A00EBC20001324178CF0725
:10A3600041BF4788E0690909C155616D088D904278
:10A37000F0DC14E70022F8E7227D002AE2690CBF36
:10A3800000216021D154013309E7606A20F83310BD
:10A3900001330BE70BB9132320E714231EE7002139
:10A3A00044E7EF8AB4F84820BF067FF543AF013297
:10A3B0003FE700962B460622A06D0021FEF7CCF960
:10A3C000E3695A5D22B1012303212046FEF7AAFB6F
:10A3D000022D12DC636D9A8C7AB9DA8AD2070CD41A
:10A3E000022D02D15B8B032B07D10A4BA06D595D67
:10A3F0000022FEF730F801358EE7B4F84A10636C9E
:10A40000194401390022491B2046FEF75DFBF2E7A3
:10A410007413060834120608E26B0421FDF79FFF4F
:10A42000D4E91530DF8A17F0010742D0226C0421ED
:10A43000FDF795FFB4F84810A06DFDF7B6FF4FF497
:10A44000A023A364A06D42460621FEF704F802276C
:10A45000A06D01221421FEF729F90097B4F84830C5
:10A46000A06D06224146FEF777F90097A06D012303
:10A4700042464146FEF770F90097A06D032342461D
:10A480004146FEF769F90097A06D33464246072121
:10A49000FEF762F92046FFF701F9636D9A8C002AF6
:10A4A00049D0002319462A8D9A425BD802B0BDE8F4
:10A4B000F081B4F84830616C05339BB24FF002086C
:10A4C000A4F84A301944FDF770FFCDF80080A06D64
:10A4D0003A4601230721FEF73FF9CDF80080072215
:10A4E000A06D11460323FEF737F9CDF8008007224F
:10A4F0003346A06D1146FEF72FF9B4F84810A06D51
:10A500003A46FEF7D3F8626CA06D3946FEF757F86D
:10A51000B4F848103A4620460331FEF7D5FAB4F8AD
:10A520004820A06D3946FEF7E9F8A06D04222D21E0
:10A53000FEF7FDF9AEE7DE8A16F00106B1D1104F45
:10A540002B8CB342ADDDB4F84A20636C17F8011BC5
:10A55000A06D1A44013A921B0136FEF7BBF8032E98
:10A56000EED19EE7EA6A02EBC30012F83320052A17
:10A5700004BF4288E06903F1010308BF815492E7F8
:10A58000341206082DE9F3410E4601EB4201044660
:10A5900015461F46FEF78EFA70288DF8060035D155
:10A5A000E26C636A03EBC2030021204613F80C6CD3
:10A5B000FEF780FA072805460DD888B12046FEF739
:10A5C000DFFBE36C626A03F10053013B02F8336086
:10A5D00002B0BDE8F0815428F0D01F4803F014FE0B
:10A5E00002460DF107012046FEF7C2FC2046FEF7A9
:10A5F000C8F9324603210123FEF794FA2A46314670
:10A60000204602B0BDE8F041FEF7D7B946EA05287A
:10A610006FB18A1C20460221FFF762F943460022EF
:10A620001D212046FEF7A9FA00221146E8E735432E
:10A6300004D00A4620460221FFF752F90DF1060127
:10A6400020460022FEF794FC012342461B212046AF
:10A65000FEF768FAE8E700BF71BE05082DE9F04192
:10A66000C66CD0F824C0DDF81880013E0CEBC6079C
:10A6700015467A78012A044613D1D7F804E09E459E
:10A680000FD0C6450DD01CF836300B7079682960A4
:10A69000FEF78BFA20464FF0FF31BDE8F041FEF7A0
:10A6A00063B90A462B6801212046FEF72FFCF1E72B
:10A6B0007FB5002303934FF0FF33009303AA0DF1FE
:10A6C0000B010446FFF7CAFF9DF80B50039E294675
:10A6D00032462046FEF771F932462946204604B03C
:10A6E000BDE87040FEF769B9F7B504460E46154659
:10A6F000002A57D1134601210DF10702FEF706FC8F
:10A70000022211462046FFF72FFC012320460D228E
:10A710000A21FEF756FB0DF1070120460222FEF743
:10A7200027FC0DF1070120460122FEF721FC2A46F5
:10A730000DF107012046FEF71BFC9DF8077020462F
:10A7400039460122FEF739F9394620460222FEF742
:10A7500034F9022211462046FFF706FC0123204669
:10A760000C220A21FEF72DFB022211462046FFF79C
:10A77000B7F82B462A4620461C21FEF7FEF92A464A
:10A7800029462046FEF719F92046FEF791FB2046A0
:10A7900001223146FEF763F9204603B0BDE8F040E0
:10A7A000FFF786BFFEF784FBAB1E5A425A41314683
:10A7B000204603B0BDE8F040FEF751B970B504463D
:10A7C00086B00D46164623B906B0BDE87040FEF7C8
:10A7D000BBBC00221146FEF7E8F920460022012109
:10A7E000FEF7E3F9324629462046FEF727FA002312
:10A7F00004934FF0FF33009304AA0DF10F0120469C
:10A80000FFF72CFF049D009501262B4605AA0DF1AC
:10A810000F0120460596FFF721FF022300930599BB
:10A82000A06D33462A46FDF7D7FF06B070BD7FB551
:10A8300004460D46164623B904B0BDE87040FEF745
:10A84000FDB900221146FEF7B0F9324629462046EE
:10A85000FEF7F4F94FF0FF330025009303AA0DF142
:10A860000B0120460395FFF7F9FE02230093039A9C
:10A87000A06D29460123FDF76FFF2A462946204691
:10A8800004B0BDE87040FEF798B800007FB50E46F2
:10A8900000210446FEF70EF9831E012B05468DF8B4
:10A8A0000B0038D8002E34D0012E19D10B4603915D
:10A8B000009103AA0DF10B012046FFF7CFFE039D87
:10A8C00044F240212B462A46A06DFDF7BFFD9DF8BE
:10A8D0000B102A46204604B0BDE87040FEF76DB864
:10A8E000022E0ED10B460391009103AA0DF10B012C
:10A8F0002046FFF7B3FE039D44F2C0312B462A46A3
:10A90000E2E7104B64689A5D0F49104806F048FC76
:10A91000206004B070BD70B901220DF10B0120461A
:10A92000FEF726FB324611212B462046FEF7FAF8A9
:10A930002A462946CEE7FEF70DF805496468024627
:10A94000E3E700BFB02B060879BE0508A819060882
:10A9500082BE05082DE9FF410D4601210446FEF7A0
:10A96000A9F8002107468DF80A002046FEF7A2F854
:10A97000BB1E012B06468DF80B0000F2D380831E10
:10A98000012B00F2FA80A5F109030C2B9CBF0D35B9
:10A99000EDB21F2D01D0212D24D1002300930122DF
:10A9A0000DF10A030DF10B012046FEF7EFFA9DF8B9
:10A9B0000A30022B07D07A4B7A495A5D7A4866688A
:10A9C00006F0EEFB30601F2D0CBF2E212F212046FC
:10A9D000FEF7BBF800220221204604B0BDE8F0419A
:10A9E000FDF7EBBF01260223039303AA0DF10B0130
:10A9F000204600960023FFF731FE32460DF10A0192
:10AA00002046FEF7B5FA1D2D7DD8DFE805F04C4C49
:10AA10004C4C4C4C7C7C7C7C7C7C7C7C7C7C7C7C36
:10AA20007C7C7C7C252D320F0F374347192DA06D80
:10AA30009DF80A60039B4FF0010206D14FF481415B
:10AA4000FDF704FD01223146C6E7032E0CBF44F298
:10AA5000C0014FF48241F3E7039B01224FF486418A
:10AA6000A06DFDF7F3FC11E0039B012244F24001CD
:10AA7000F6E7039B01224FF48041F1E7039941F689
:10AA80000903A06D43EA8111FDF777FC9DF80A10D8
:10AA90000122A1E7039941F60923F2E7039B012272
:10AAA00044F24031DCE79DF80A609DF80B30B34278
:10AAB00005D03E493C48676806F072FB38600022CA
:10AAC000032E1146204614BF06260026FEF76DF819
:10AAD0000122039BA06D4FF48541FDF7B7FC2E4486
:10AAE000334BA06D33F81610FDF747FCA06D42F212
:10AAF0000101FDF742FC4FF40051A06DFDF73DFC54
:10AB00000022012168E720460121FDF72DFF244B9B
:10AB100028495A5D2448646806F042FB206004B06E
:10AB2000BDE8F08157EA000827D1012600960DF113
:10AB30000A0302220DF10B012046FEF727FA322DFF
:10AB400017D0332D17D0464600232A46122120461F
:10AB5000FDF7E8FF56B1A06D00220121FDF77BFC57
:10AB60000023032211212046FDF7DCFF00221146BD
:10AB700032E70625E8E70725E6E720464FF0FF31F4
:10AB8000FDF7F2FE3846FDF7E5FE02463046FDF7DA
:10AB9000E1FE094964680346034806F001FBBDE78E
:10ABA000B02B060892BE0508A8190608A2BE050823
:10ABB00044110608B5BE0508C3BE05082DE9F043DB
:10ABC0000446C16885B0FEF7B3FB626DD18A928CF2
:10ABD00001F0110313432ED011F0010117D1B4F885
:10ABE000482020460132FEF715F8636D9D8C55B95B
:10ABF000A06D4FF42051FDF7C0FBE268A06D01325B
:10AC00002946FDF75FFE05212046FDF79EFF212125
:10AC10002046FDF79AFF636DDA8AD20706D49B8C33
:10AC200023B9E16820460131FEF782FBA06D1222B4
:10AC30000021FDF74FFDA06DFDF7E9FB237D002B03
:10AC40005ED1A36D656C5B68A36323685B88E36377
:10AC5000636D013D5E8BDF8AB3F81C90B3F81E80F4
:10AC6000EA0006F0030302F0780207F00F071A4328
:10AC70002D09B60845EA0703334343EA090353EABB
:10AC80000803A06D65D10121FDF769FBB4F85060A0
:10AC9000B4F85270A06D720007F0010302F07E025A
:10ACA0007F08B60957EA060542EA030218BF42F0D8
:10ACB00080020121FDF753FB002DEBD1636DA76DE1
:10ACC000998A20687E68FCF7CFFD474902463846DE
:10ACD00010F0D0FC626D538B918B108D0B44AB4206
:10ACE00071DCA36D9F88BE1BA4F850600025D4E9D9
:10ACF00015301A8DAA4268DC4368DB1BA4F8523079
:10AD00002369042B21D1A36DD3E902762368586807
:10AD1000237D5BB9A56BE16B3544002962D001311D
:10AD20008900F5F7C2FAE36B40F823500023656D04
:10AD3000217DCDE90233EB8ACDE900030331286997
:10AD40003B463246C9B201F01FFE012005B0BDE806
:10AD5000F08342F080020121FDF701FBBA012B01D3
:10AD600003F0300302F040021A4308F001031A43D3
:10AD70004FEAC90303F008031A43B30003F00403C6
:10AD80001A43AD087F0876084FEA59094FEA580878
:10AD900070E7D36A03EBC1035F78FF070ED55F88C6
:10ADA000AF420BD159682068A76DFCF75DFD0E49D5
:10ADB0000246384610F05EFC01358BE701318142D6
:10ADC000E7DB0521EFE70021F9E7DB6A03EBC502CA
:10ADD00013F83530052B03D152880121FDF7BFFA56
:10ADE000013584E72846A1E71D8302082DE9F041DB
:10ADF00088B004460D4607AE002940F0BD80012111
:10AE0000FDF758FE07468DF8170078BB014620462F
:10AE1000FDF750FEC0B9012231462046FEF7A8F8E2
:10AE200000220DF117012046FEF7A2F804220F219F
:10AE300002232046FDF776FE00221146204608B088
:10AE4000BDE8F041FDF7B9BD3A4631462046FEF770
:10AE50008FF89DF81C20204601230421FDF762FE97
:10AE6000A06D3A460121FDF7F6FAD9E7E36C626A74
:10AE7000013B02EBC30032F8332040F202239A4236
:10AE80002BD147684FF001082046FDF77AFD434675
:10AE900032460DF11701CDF800800795FFF7DEFB74
:10AEA00020462A462946FDF780FE9DF81700062811
:10AEB0000DD007280ED0052854D10095079AA06D13
:10AEC0003B462946FDF748FC00220221B6E7CDF8B3
:10AED0000080F3E702230093F0E72B460791324608
:10AEE00006A920460095FFF7B9FB2A460DF1170188
:10AEF0002046FEF73DF820462A462946FDF755FE36
:10AF00009DF81800831E012B08D9FDF723FDA149E8
:10AF100065680246A04806F043F928609DF81700CE
:10AF200006280BD0072813D005281BD107998901C3
:10AF300041F4B841A06DFDF720FAC5E70799A06D6F
:10AF4000C90041F04201FDF718FA4FF4B541F1E7AD
:10AF50000799A06DC90041F08201FDF70EFA4FF488
:10AF6000B141E7E7FDF7F6FC8C49656802468A487F
:10AF700006F016F92860A7E7012940F0FB80FDF7ED
:10AF800099FD07468DF8150050BB01462046FDF798
:10AF900091FD022105468DF818002046FDF78AFD37
:10AFA00005438DF81C0008D0394620460322FEF7E1
:10AFB00097FC03212046FDF7D7FC0223CDE901636E
:10AFC0000023009306A920460DF115030122FEF788
:10AFD00011F80F21204608B0BDE8F041FDF7B5BDDE
:10AFE000E36C626A013B02EBC30132F8332040F2AA
:10AFF00002239A423ED12046D1F80480FDF7C1FCDD
:10B0000002230022CDE90623009306AA2B460DF168
:10B010001501FFF723FB069F00953B46204632466D
:10B020000DF11701FFF71AFB9DF81700431E022BC5
:10B0300008D9FDF78FFC5A4965680246564806F064
:10B04000AFF828609DF8150006280FD007280FD00C
:10B05000052840F08580002300930799A06D4346A2
:10B060003A46FDF7B9FB08B0BDE8F0810123F3E7EC
:10B070000223F1E702230793009306AA00230DF1B0
:10B08000160120460695FFF7E9FA204600220DF149
:10B090001501FDF76DFF9DF81600831E012B08D9E1
:10B0A000FDF758FC3F49656802463B4806F078F8D2
:10B0B0002860069D00950023204632460DF11701B9
:10B0C000FFF7CCFA9DF81700431E022B08D9FDF7B5
:10B0D00041FC3349666802462F4806F061F830604B
:10B0E0009DF8150006280ED0072825D0052837D151
:10B0F000079941EA851141F4A841A06D08B0BDE867
:10B10000F041FDF73AB90126AE40A06D46F4344156
:10B11000FDF733F945EAC50141F04001A06DFDF7A7
:10B120002CF9079941EA851141F4A441A06DFDF77E
:10B1300024F946F43C41E0E70126AE40A06D46F418
:10B140003441FDF71AF945EAC50141F08001A06DCF
:10B15000FDF713F9079941EA851141F4A041E5E7AC
:10B16000FDF7F8FB1049646802460B4806F018F832
:10B17000206078E70025334606A900950122FDF7F7
:10B1800005FF02232A460F21204608B0BDE8F04102
:10B19000FDF7C8BCE6BE0508A8190608DDBE05080F
:10B1A000F0BE0508FBBE0508F5BE05082DE9F04117
:10B1B00080465C2016460F461D46F5F774F88660FB
:10B1C00008260446C0E9008706624020F5F752F8D9
:10B1D000E66260622020F5F74DF860632020F5F705
:10B1E00062F82946A065FDF76EF82046BDE8F081BB
:10B1F00010B504460021806DFDF76DF8A06DF5F7E0
:10B2000061F8606BF5F75EF8E069F5F75BF8606A86
:10B21000F5F758F82046BDE81040F5F753B80000A0
:10B2200002F00F03022B10B5044608D00A460C4961
:10B230000C4805F0B5FF636A1860002010BD836AF2
:10B2400012090020834204D1238C042BF5D1064936
:10B25000EEE7E16A51F820109142EFD00130F1E7BA
:10B2600002BF0508141A060808BF050870B506468F
:10B27000B2B1900714D110792E2811D194687CB105
:10B28000A2070DD16568EAB2922A09D12D0A022DD2
:10B2900006D1A2681A60049BE2681A60012070BDA2
:10B2A0000A460448044905F07BFF736A18600020D1
:10B2B000F5E700BF141A060814BF05087FB5044659
:10B2C0000D46104603A91E46F8F776FD48B90C490D
:10B2D0000C482A4605F064FF636A1860002004B039
:10B2E00070BD039803F068FE30EA06020346F6D00C
:10B2F000054900962A46034805F052FFECE700BFD7
:10B3000030BF0508141A060836BF0508038C032B46
:10B3100070B5C46A03D1856A00239D4205D144F803
:10B320002120FDF70BF8012070BD54F823609642F0
:10B3300001D00133F1E70020F6E7FDF768B80329F3
:10B3400010B50446018442620FD1826AC06A0021AE
:10B3500092001FF0DBF901212046FCF7C7FF2046D1
:10B360000021BDE81040FDF720B8042914BF0121D9
:10B370000221F1E700F00F03022B02D10009F5F7DB
:10B380009CBE0148704700BF2CD8050870B5054623
:10B3900010460E46FFF7EEFF0378732B19D1437862
:10B3A000BBB103460A22002013F8014F5CB91F28E5
:10B3B00008D90B490B481F23324605F0F1FE6B6A92
:10B3C0001860002070BD303C092C02D802FB004000
:10B3D000EAE705490348324605F0E2FEEFE700BF21
:10B3E0004CBF0508141A060859BF0508F8B50546EC
:10B3F00010460E461F46FFF7BDFF174C017800228E
:10B40000A44663788B421BD190F801E0A3789E4557
:10B4100016D190F802E0E378734511D16BB91CF8AE
:10B420002200B84208D90D490D483B46324605F086
:10B43000B7FE6B6A18600020F8BDC378002BEED011
:10B440000132152A04F10404DBD1064904483246CE
:10B4500005F0A6FEEDE700BFEC1206084CBF05089C
:10B46000141A060862BF05082DE9F34706460F4681
:10B47000002A3CD093073AD113792F2B37D1926809
:10B4800002F00F03022B08D10F23FFF7AFFF0124B7
:10B490008440204602B0BDE8F08742B312F0030AB0
:10B4A00025D113799F2B22D1D5682B79A12B1ED1C1
:10B4B00092680F23FFF79AFF4FF0010909FA00F491
:10B4C00001AAA22105F10800F8F7C2FE8046C24594
:10B4D000DFDA019A0F2352F82A2039463046FFF767
:10B4E00085FF09FA00F004430AF1010AEFE7044975
:10B4F00004483A4605F054FE736A00241860C8E711
:10B5000068BF0508141A060810B50446024805F07D
:10B51000B1FD206010BD00BF141A060804292DE9F2
:10B52000F84380460C460DD8151F01F1300930262E
:10B530004E450DD055F8040F00F00F03022B0AD032
:10B540000D4900E00D49D8F82400FFF7DDFF002485
:10B550002046BDE8F8830009F5F7AFFD07461FF068
:10B5600013F90228ECD13B78722BE9D17B78B342F6
:10B57000E6D10136DCE700BFA2BF050879BF0508A8
:10B580002DE9F0470F4686B0044603A938461E460B
:10B590009146F5F79EFD0378762B054640F018811D
:10B5A000B9F1020F40F0C580A7F25F570D2F00F2EE
:10B5B0000681DFE817F00E003600390004010401AF
:10B5C000040104018C0004015E003C0031002E00E7
:10B5D000BB004EF6B4684FF42C6932682946204609
:10B5E000FFF7D4FE7268074629462046FFF7CEFED5
:10B5F000FA0249EA500902F47042400142EA0902A3
:10B6000000F02000B90101F04001024348EA0101C5
:10B6100029E04EF6B168DEE74EF6B1684FF42469D2
:10B62000DBE74EF6B868D6E74EF6BD68D3E730687C
:10B63000FFF7A0FEA9491FF0B5F8C0B132680F238B
:10B6400029462046FFF7D2FE07467068FFF792FEB4
:10B65000A3491FF0A7F8002840F0B1803A0342F454
:10B6600021624EF6F1612046FCF791FEE6E10F27DC
:10B67000EBE73068FFF77EFE03783268722B17D154
:10B680000F2329462046FFF7B1FE29467268074678
:10B690002046FFF77BFE4EF6106180464FEAC81247
:10B6A000D2B242EA073242F4216241EA5801DAE7B3
:10B6B00029462046FFF76AFE2946726880460F2316
:10B6C0002046FFF793FE4FF46E410746E6E74EF63D
:10B6D0009058326829462046FFF758FE05AB009384
:10B6E0000746726804AB29462046FFF7BFFD0028D5
:10B6F00000F0A481049A072329462046FFF776FE2E
:10B70000059A064629464FF47F732046FFF7D6FD7B
:10B71000FA02B90102F4704201F0400142EA9002DB
:10B7200041EA080142F4206231439CE74EF680581A
:10B73000CFE7B9F1030F42D1DFF8BC81002700F158
:10B74000010A0322414650461FF044F890BB2B7972
:10B7500083BB644B326813F8278029462046FFF7E5
:10B7600015FE7268074629462046FFF70FFEB268AD
:10B77000814629462046FFF709FE4FEA0813DBB24F
:10B7800043F4206343EA5003400100F02000FA0232
:10B7900002F470420343134308F0F0084FEAC91261
:10B7A000D2B248F46E48B90148EA590801F04001A4
:10B7B0001A432BE70137042F08F10408C1D14B4687
:10B7C00049494A482A4605F0EBFC636A186035E1AE
:10B7D000B9F1030FF3D8DFE819F0040015001501E3
:10B7E000C40240F29A439F4205D14FF43F412046A4
:10B7F000FCF7C3FD22E140F26E539F42DFD14BF6CE
:10B800003071F4E7B7F5657F10D101463268204604
:10B81000FFF706FD01462046FCF741FE002840F0F8
:10B820000D813349606AFFF76FFE07E140F29E32F7
:10B83000974209D1014632682046FFF7F1FC0146E4
:10B840002046FCF786FEE9E7B7F56A7F09D1014695
:10B8500032680F232046FFF7C9FDC10041F48E4135
:10B86000C5E7622B4AD1039B032B0CD0052B40F07C
:10B870008C80C3785F2B40F0888003796E2B02D0D8
:10B88000772B40F0828069781A4B00224FF0FF3707
:10B890005878884205D195F802C09878844508BF49
:10B8A0001F7801320E2A03F10303F1D17B1C86D0ED
:10B8B000326829462046FFF7B3FC039B052B02465E
:10B8C00009D12B79A3F1770673427341394620469B
:10B8D000FCF703FEA2E70023F8E700BFC0BF05089E
:10B8E000CABF05084C120608DDBF0508141A060871
:10B8F000EABF0508B01206084D120608692B44D1AC
:10B900004378742B41D13068FFF734FDB64B017892
:10B9100000221F465E788E4222D190F801C09E78A8
:10B92000B4451DD18678DEB9AE1C31460B460131D7
:10B9300018780028FAD1691D8B423FF640AF02EB20
:10B9400042020821BF5CFA43D200F800013B0A40E2
:10B9500008409E420AD941EA071141F43F4146E7B7
:10B9600001320E2A03F10303D4D128E713F801C9E9
:10B97000BCF1740F4FEA510101D10143E9E7BCF179
:10B98000650F7FF41CAF1143E3E740F2C9339F42D8
:10B9900002D14BF272612AE740F2CA339F4202D1D0
:10B9A0004BF2626123E740F2C5439F4213D13268F4
:10B9B00029462046FFF758FD10F43F4F024607D1B5
:10B9C00045044ABFC1B240F4344141F435410EE769
:10B9D0004EF62D1147E6782F7FF4F1AE32682946F6
:10B9E0002046FFF741FD10F4FE4F024607D1100438
:10B9F0004ABFD1B242F43C4141F43D41F7E64EF634
:10BA0000BD0130E6736803F00F03022B40F09D8008
:10BA100040F28C439F4214D1014632680F232046E6
:10BA2000FFF7E4FC7268074629460F232046FFF71C
:10BA3000DDFC394602462046FCF70DFD06B0BDE8A8
:10BA4000F08740F2B9339F421CD14FF6B0294FF234
:10BA5000800732680F2329462046FFF7C7FC72682B
:10BA6000804629460F232046FFF7C0FC47EA000224
:10BA700042EA082249EA0001F5E54FF690294FF223
:10BA8000A007E6E7B7F59A6FF7D0B7F5926F2AD11E
:10BA900032680C2301462046FFF7A8FC0746706871
:10BAA000FFF768FC0146064650481EF07BFE034641
:10BAB000A0B14F4831461EF075FE70B12A464D497F
:10BAC0004D4805F06DFB636A0022186042EA0722C8
:10BAD00042F400424FF2EF31C5E50123474A03EB40
:10BAE000C303D25CF2E740F286339F4215D14FF494
:10BAF00080473268294607232046FFF777FC7268A3
:10BB00008046294607232046FFF770FC424603463D
:10BB100039462046FCF79AFC90E7DFF8E8800027DA
:10BB20000322414628461EF055FE40B9EB7833B952
:10BB3000334B13F827703F0147F48047D9E70137AB
:10BB40000F2F08F10408EBD139E6B7F5926F2AD22E
:10BB500040F28B439F421ED840F2BB339F423AD003
:10BB600040F259439F4200F08480B7F55F7F35D0A3
:10BB700040F257439F4200F0DC80B7F58B6F00F036
:10BB8000DA8040F25A439F4200F0D780972F40F06E
:10BB90009D800323A0E0A7F28D47022F21D8DFE884
:10BBA00007F04A334D00B7F5A66F40F08B804FF495
:10BBB00060573268072329462046FFF717FC2946BD
:10BBC00080467268FF232046FFF778FB47EA0001B2
:10BBD00041EA08210BE64FF42057EAE74FF44057BB
:10BBE000E7E74FF40057E4E7B0120608DB12060857
:10BBF000E4120608D0BF0508141A0608DA1206086F
:10BC000074120608751206084FF2402832680F2396
:10BC100029462046FFF7EAFB726807464FF6FF7396
:10BC200029462046FFF74AFB3A460346414620464E
:10BC3000FCF723FC02E74FF2C028E7E70146326831
:10BC40000F232046FFF7D2FB2946074672684FF0C4
:10BC5000FF332046FFF732FB3A4683B205464FF2E8
:10BC600040212046FCF709FC2B0C3A464FF2C0213C
:10BC7000DDE7014632680F232046FFF7B7FB05AB2F
:10BC800000930746726804AB29462046FFF7EEFA98
:10BC900000283FF4D3AE049A0F2329462046FFF72D
:10BCA000A5FB059A06462946FF232046FFF706FB1B
:10BCB000820842EA073246F4684142F4706241F079
:10BCC0005001D0E440F22C539F4238D040F22E5322
:10BCD0009F427FF474AD0523814A294632F82370D0
:10BCE000326807232046FFF781FB05AB00938046AF
:10BCF000726804AB29462046FFF7B8FA00283FF4E3
:10BD00005EAD049A294607232046FFF76FFBF9042E
:10BD1000059A064615D51F2329462046FFF7CEFA79
:10BD200047EA0807800147EAC60700F4F86139438B
:10BD30005DE50023D0E70123CEE74B46CCE70423A3
:10BD4000CAE73B0406D53E2329462046FFF7B6FA4C
:10BD50004008E5E77C2329462046FFF7AFFA800834
:10BD6000DEE7B7F58D6F21D100273268072329461A
:10BD70002046FFF73BFB7268814607232946204691
:10BD8000FFF734FB29468046B2681F232046FFF7A1
:10BD900095FA47EA090747EA801747EAC80126E506
:10BDA0004FF40067E1E74FF48057DEE740F2694364
:10BDB0009F42F5D040F28F339F42F4D0B7F55F7FBA
:10BDC0002BD14FF4C0583268072329462046FFF78D
:10BDD0000DFB72680723074629462046FFF706FB3E
:10BDE000B26802F00F03022B81460ED107232946C9
:10BDF0002046FFF7FBFA47EAC90141EA080141EA98
:10BE00008011F4E44FF4D058DDE70723294620469B
:10BE100048F48068FFF752FAEDE740F202539F4280
:10BE200021D14FF6903832680F2329462046FFF77C
:10BE3000DDFA726881460F2329462046FFF7D6FABD
:10BE4000B268074629460F232046FFF7CFFA40EA9B
:10BE5000092040F4704242F0F00248EA070102E48F
:10BE60004FF6B038DFE740F252539F42F8D0B7F5B3
:10BE7000A66FC7D040F22D539F427FF4A0AC01467D
:10BE800032680F232046FFF7B1FA72680F23294664
:10BE900007462046FFF7AAFA05AB00938046B26832
:10BEA00004AB29462046FFF7E1F900283FF4C6AD70
:10BEB000049A0F2329462046FFF798FA059A06466A
:10BEC0002946FF232046FFF7F9F93F0247EA0837E2
:10BED00046F4684147EA900241F04001FFF7C3BBD6
:10BEE0005C12060838B505463020F4F7C3F9202265
:10BEF000044600211EF00AFC29462046FCF7E3F91F
:10BF0000A562A800F4F7B6F9E062204638BD10B586
:10BF10000446C06AF4F7D6F920460021FCF7DBF9A5
:10BF20002046BDE81040F4F7CDB92DE9F04F099F48
:10BF3000DDE90BC4DDE90D5650B1884208D3710725
:10BF400047BF0137013401350A2158BFB0FBF1F07A
:10BF500016F0020E39D0002D37D00BDB0A998D4236
:10BF600033DA2C44A74203DC07F1FF3CA4EB0C0CB2
:10BF700000252AE0291D28DB69424FF000084FF018
:10BF80000A0AB0FBFAF90AFB19041CB108EB050414
:10BF9000414604E008F1010888454846F1D11D46B4
:10BFA0004FF0300905F8029B7F1A091B4FF02E084D
:10BFB0004C1E83F801802346A846002B5DDC002937
:10BFC00008BF00242B190025FF2407F1FF38414644
:10BFD0004FF00A09002954DA611CB94260DBFE2CDB
:10BFE000D4BF002101213B44BCF1000F07D0A4EBDA
:10BFF0000804A4EB0C0C2E203027644555D1BEF16B
:10C00000000F09D041B119460B4611F8010D302837
:10C01000FAD02E2808BF0B4606F00101294327D08D
:10C02000710725D4002DBABF6D422D212B2106F0BA
:10C030002004632D597044F04504C8BF64211C706E
:10C040004FF00A00C9BFB5FBF1F19C1CDC1C30317C
:10C05000C8BF9970B5FBF0F62346B6FBF0F100FBC4
:10C060001161303103F8021B00FB16513031617051
:10C0700000211970981ABDE8F08F08F8019B013B68
:10C080009BE78C42B4BF01F1010B8B46B0FBF9FA80
:10C0900009FB1A00303003F80B000139504699E7CC
:10C0A00001332E21195501219DE714B903F8010B25
:10C0B000012103F8017B013C9FE700002DE9F04FCF
:10C0C0002DED028B884610EE101A97B000291C4601
:10C0D000B0EE408A9DF888300E902ADAB4EE400A1D
:10C0E000F1EE10FA25D6B1EE408A2D230E9F07F807
:10C0F000013B08F1FF389FED7D7AF0EEC87AF4EE4F
:10C10000477AF1EE10FA02F0200316DD43F04904FD
:10C1100043F04E00FA1C43F04601002378703C7057
:10C12000B97013700E9BD01A17B0BDEC028BBDE82E
:10C13000F08F002BDAD10E9FDDE7B4EE488AF1EEE6
:10C1400010FA06D743F04E0143F04100FA1C0C46AA
:10C15000E3E742F02002662A4FD143F0040B002CA3
:10C16000A8F1030650DA0624A6423346A8BF2346A8
:10C170000C9318EE103A002B099353D0C3F3C75316
:10C180007F3B07EE903A9FED5A7AF8EEE77A18EE89
:10C19000103A67EE877AB3F17E5FFDEEE77A38BF3B
:10C1A0004FF0000917EE905A28BF4FF0010909EB34
:10C1B0000500B7EE000A00F047FA099BB3F17E5F75
:10C1C0002CBF4FF0010A4FF0FF3AB4EEC80AF1EE6F
:10C1D00010FA94BF012300234B451BD01BF0040F22
:10C1E0004CD0002D20DD6319023398451CDA8BF00A
:10C1F000040343F0020B013444E0672A0CBF43F010
:10C20000020B43F0010BAAE7632CADD110230C9372
:10C210000924AEE7554405EB0900B7EE000A00F02B
:10C2200013FAD2E7099DD9E7A8F10202A242D4BFCE
:10C2300033462346002D1EDA022B15DDAA1C17DA21
:10C240006E429E42A8BF1E46023E9C1B092C0DDD7D
:10C250001BF00403A4F1090207934FF009041CD05A
:10C2600004230793032319E05C1C00260022F7E750
:10C270005C1C0026EAE76C1C1C44FAE71BF0020F6A
:10C28000B9D034B1092C4FF00006E1DC32460796F4
:10C2900003E026462246079401240723062CA146E4
:10C2A000A8EB0408A8BF4FF00609A8EB0308A9EB08
:10C2B0000503013B0D939045D4BF04EB0803A3187D
:10C2C0001193119BA3EB09030F93099B002B00F023
:10C2D000CB80079B002B00F0C380002D80F2BD8037
:10C2E00046B909F1FF3008963B4613E0FFFF7F7F18
:10C2F0009B209A3E3B46302103F8021B2E227A7087
:10C30000184632461EF002FAFF220346334409EB78
:10C31000060008920A214FF0010C0A91E14500F352
:10C32000A880B9F1060F40F3AF80012840F3AC803C
:10C33000B9F1070F00F0A480022800F0A1800238B4
:10C340004FF06408B0EE480A0B9300F07DF9F6EE6A
:10C35000007A30EE270A0A99BCEEC00A3A4610EE7F
:10C36000103A08FB03F8089B03930F9B02930C9B66
:10C37000CDE9045BCDE9009340460B9B1093FFF79A
:10C38000D4FD15AA01460B90384600F08DF9DDED7D
:10C39000157A0B9977EEC87A17EE902A002A58D0B2
:10C3A000B9F1060FC4BF09EB4902123A4FF0010A76
:10C3B000C8BF0AFA02FA0C22109BCDF82C80F0EECE
:10C3C000678A109217EE902A002A089A03920F9A11
:10C3D00002920C9A0A991393B4BFD044A8EB0A08AE
:10C3E000CDE90092CDE9045B3A464046FFF79DFD5A
:10C3F00015AA01461290384600F056F9DDED157A7F
:10C40000129977EEC87A17EE902A12B3B0EEE77A57
:10C41000F0EEE86A37EE667A139B17EE102A002AD0
:10C4200035DB4FF00A0CB8FBFCF00CFB108002432C
:10C43000002A0B9A08BF42460B9208BFF0EE678AAB
:10C44000BAF1010F28D0109A013A4FEA5A0A109215
:10C45000B8D10E9B3944C81A66E60D98089543E793
:10C46000079B0D9808933FE7099A08923B461046B0
:10C4700050E70A990A2251430A910CF1010C4DE749
:10C4800001384FF00A085DE74FF001085AE7CDF890
:10C490002C80F0EE678AD3E70D9AA14502F10102E4
:10C4A0000D9202DA09F101090BE70B9A9045D0D001
:10C4B000089A03920F9A02920C9ADDE90A10CDE9CC
:10C4C0000092CDE9045B3A46FFF72FFD0146C0E735
:10C4D000012910B5136823D90178302920D141787A
:10C4E00041F02001782900F1020406D133F0100355
:10C4F00014D110231360201A10BD6F2904D133F01A
:10C5000008030BD10823F5E7622904D133F00203B5
:10C5100004D10223EEE70BB9012313600446EAE7D6
:10C52000002BFBD10A23F8E708B5044631B1054BCF
:10C530004A6B03600968002304F07EFE2046F3F78F
:10C5400071FE00BF141A06082DE9FF41044601924E
:10C550001F4646182AB1023A222A02D9374801F06A
:10C5600085FCB442254626D34FF00008711B2846AF
:10C5700001AAFFF7ADFF019B054428460024B04205
:10C5800001462AD3B8F1000F00D06442640044F0A1
:10C590000104A94204D00D46B5422B4642D348D0EF
:10C5A000019A27492748012A08BF002204F0F8FD14
:10C5B0003946FFF7B9FF14F8010BF5F767FB804622
:10C5C0000028CED12B782B2B01D12546CEE72D2B61
:10C5D000CAD125464FF00108C8E710F801CBACF1ED
:10C5E0003002092A0AD9BCF15F0FC8D04CF02002F2
:10C5F000A2F1610CBCF1190FC4D8573A9342C1D9CA
:10C6000083FB0441B1EBE47F03D1144494EA440278
:10C61000B5D5711B424603A8039505F0DCFF0399CD
:10C620000446B6E718780135F5F730FB0028B3D19A
:10C63000B6E7204604B0BDE8F08100BFF5BF0508AD
:10C640000AC005088419060808B52DED028BE8B16B
:10C65000B5EE400AF1EE10FA18D010EE103AC3F31E
:10C66000C752024462F3DE5310F10A0F08EE103A8B
:10C670000FD3434200EE903AB1EE040AF8EEE00A1E
:10C680001CF0E0FCF0EE407A88EE270ABDEC028B4D
:10C6900008BD07EE900AB1EE040AF8EEE70A1CF0B6
:10C6A000D1FC28EE000AF1E700232DE9F047014410
:10C6B000044690469E461D4618461F469A461E460C
:10C6C0008C4257D2A4461CF8012BA2F13009B9F1D3
:10C6D000090F38D8022E07D1354A904202DC0A22CF
:10C6E00002FB00906446EBE7B9F1000F14D0314A29
:10C6F000974211D80A24B5B975460A24CDB9974294
:10C700001ED8012E4FF00A0208BF03F1FF3302FBCF
:10C7100007974FF0000EE5E70EB90135E2E70EF19D
:10C72000010E0126DEE7974294BF67430133013DC6
:10C73000E1E797429CBF03F1FF336743013DDDE72B
:10C740007EBB0133E5E78EB92E2AEAD042F02009FC
:10C75000B9F1650F0CD1614504D962782B2A19D142
:10C7600004F1020C8C4520D00226BBE7022EEDD14D
:10C770005F2AB7D0BAF1000F15D107EE907A1D44A9
:10C78000B8EE670A2844FFF75FFF88ED000A2046ED
:10C79000BDE8F0872D2AE7D104F1020C4FF0010A21
:10C7A000E0E7AE46BDE74042E7E70024EFE700BF21
:10C7B00064666606979999192DE9F04F2DED048B63
:10C7C00083B09FED658ADDF840909FED649A054641
:10C7D00090461F4646184FF0000AF0EE488ACDED0D
:10C7E000018AB5422C466CD34FF0000BA31C9E422D
:10C7F00040F28980237843F02003692B73D163785A
:10C8000043F020036E2B7ED1A37843F02003662BE8
:10C8100079D14FF0FF430193E31D9E4204F10300E1
:10C820001AD9E37843F02003692B15D1237943F01B
:10C8300020036E2B10D1637943F02003692B0BD1B9
:10C84000A37943F02003742B06D1E37943F020034E
:10C85000792B01D104F10800B8F1000F0ED0B042DD
:10C860000CD2037843F020036A2B07D1844204BF23
:10C870004FF07E53019301304AF0020ABBF1000FE2
:10C8800005D0DDED017AF1EE677ACDED017A8442D3
:10C8900040D00446B442254643D348D1BAF1010FF3
:10C8A00038D09DED010ABAF1000F4AD0F0EE400AEF
:10C8B000B0EE480A03B0BDEC048BBDE8F04F03F0C6
:10C8C000AFBB15F8010BF5F7E1F98346002888D1D5
:10C8D00023782B2B01D12C4688E72D2B84D12C4695
:10C8E0004FF0010B82E76E2B0DD1637843F02003EC
:10C8F000612B08D1A37843F020036E2B03D1E01CF9
:10C900008DED019AA8E701AA311B2046FFF7CCFE66
:10C910000028A1D11249134804F0ACFB4946FFF7A7
:10C9200003FE28780134F5F7B1F90028B2D1002FC1
:10C93000F0D0BAF1000FEDD19DED018A4FF0010A60
:10C940004DE717B1DFED040AB4E703B0BDEC048B8B
:10C95000BDE8F04F04F064BD000000000000C07F9F
:10C9600016C005088419060808B51020F3F79BFCCB
:10C970000123837008BD10B503F001030224C0E950
:10C9800001128470C37010BD9DF80430426003F042
:10C990000103C370009B8360029B0373C368039A07
:10C9A000817062F31F23C3607047000070B50446B6
:10C9B0000D4623881046CBB10A460023214605F0D8
:10C9C000E1F82346002213F8011B1D1B090605F19F
:10C9D000FF3503D4D30725D51C4B19E013F8011BF1
:10C9E000C1F3801606FA05F52A43EEE7A3786668D8
:10C9F000042B0FD0052B16D0032B0A46A368314613
:10CA00001DD105F0BFF8124B0360E37853B1114B11
:10CA1000036007E01049A468102002F0BFF9C0E9E4
:10CA20000154C66070BD0D49257BE468102002F0FA
:10CA3000B5F9C4F31724C0E90156C460F2E705F064
:10CA4000A1F8E378002BEDD0C6E700BF2C1F060845
:10CA5000E41D0608101F0608CC1D0608B41D0608B4
:10CA600038B5144612F4807218BF1A461D46FFF7F7
:10CA70009DFF620902F008022A44E1B2BDE8384095
:10CA800003F068BAD0E90003184770B505460C46B4
:10CA90008E18B44200D170BDD5E90003984704F860
:10CAA000010BF6E738B504460025D4E900039847A2
:10CAB00000F07F0343EAC5150306F6D4284638BDC7
:10CAC0002DE9F04186B00546FFF7DCFFC4B2042C27
:10CAD00006D8284B53F82440204606B0BDE8F08124
:10CAE0002846FFF7DFFF064630B9062C04D128465A
:10CAF000FFF7C8FF204CEFE70A2C10D10021304689
:10CB000009F07AFF0027044600F10408B742E3D099
:10CB10002846FFF7D5FF013748F8040FF6E73146FE
:10CB200002A8F4F7B3FB049932462846FFF7ADFF9D
:10CB3000631F012B0CD82846FFF7A4FF052C02A881
:10CB400003D108F07BF80446C6E708F07DF8FAE761
:10CB5000072CDDE903104FF0000303D10A22FFF791
:10CB6000F3FCF0E7093C624200936241FFF724FEC8
:10CB7000E9E700BF40130608E02606082DE9F84360
:10CB80002B4E04460F46904600252068FFF77AFF9B
:10CB90005FFA80F9B9F1FF0F01D1BDE8F883C10751
:10CBA0000CD52068FFF77EFFC20748BFA3684FEA95
:10CBB00050054FEA850554BFED19ED184FEA5903AA
:10CBC000082B21D8DFE803F0050505050505171B2F
:10CBD0001E00DB070DD52068FFF764FF5FEA9909A7
:10CBE00023D0B9F1010F0CBFA368E36802462946C0
:10CBF00016E00120F2E763689B680120F6E76368AE
:10CC0000DB68FAE73346F8E703F18043084A093B5B
:10CC100052F82330F1E751F804CB9C4441F804CC9E
:10CC2000013AF8D205EB8005AFE74346DEE700BFE7
:10CC3000741306082DE9F04F8FB080460991FFF775
:10CC400031FF00F003039A1C0492C20800F00409AB
:10CC50000792002B3FD11046F3F70CFB4FF0000A70
:10CC60000146079A06464046FFF70FFF5746CDF8A4
:10CC700020A05446CDF814A05546B9F1000F00F09D
:10CC800098804046FFF70EFF049B8146032B08BFA8
:10CC900001308000F3F7EEFA4FF0000B0690CB4521
:10CCA0007DD1FFF761FE049B022B834640F08C8010
:10CCB0003246002312F8011B901B090600F1FF30D9
:10CCC0007AD4069A9BB231465846FFF754FE58462E
:10CCD0000FB0BDE8F08F0798F3F7CCFA079A01463A
:10CCE00006464046FFF7D1FE049B032B404618D171
:10CCF000FFF7D8FE04463018335D411C00270A1A9E
:10CD00001D0602F1FF3204D44FF0000ACDF820A036
:10CD1000B0E711F8013BC3F3801505FA02F217439F
:10CD2000EDE7FFF7BFFE049B052B07460BD14046FE
:10CD3000FFF7B8FE08904046FFF7B4FE0024824695
:10CD40000594254699E710F0200B23D04046FFF7C5
:10CD5000A9FE824617F0400002D04046FFF7A2FE2F
:10CD60001AEB000418D0C51C25F003050AEB0500DA
:10CD7000F3F799FA05900544BBF1000F04D0524631
:10CD800029464046FFF781FE4FF0000ACDF820A06B
:10CD9000544672E7DA46DDE7A2460894D0E70999DF
:10CDA0004046FFF747FF069B43F82B000BF1010BB2
:10CDB00075E7CDF8189074E712F8011BC1F38014E1
:10CDC00004FA00F0034377E7099BCDF82880CDE90A
:10CDD0000B35059B0D93FB0610D5154DD5F8CC00F2
:10CDE00020B9014606F0B4F8C5F8CC00314605F08C
:10CDF00024FE324631460AA8FFF7C0FE049B032BEF
:10CE000006D13444B9F1000F03D0069B43F8294002
:10CE1000069C089B0293BFB2CDE90047079B04998B
:10CE2000CDF80CA032465846FFF7AEFD4FE700BFE5
:10CE3000B40400202DE9F04786B0836804930446CB
:10CE40000368059302A80F463E49F3F7B1F904229F
:10CE50000DEB02012046FFF718FE9DF806509DF8E5
:10CE60000420AB084D2A03F02F030CD19DF80520B8
:10CE7000062A08D11BB105F00302032A03D19DF84D
:10CE800007201F2A02D9304800F0F0FF23B1043BED
:10CE9000032B01D92D48F7E715F04005F3D12046C3
:10CEA000FFF700FE81462046FFF7FCFD4FEA4906EA
:10CEB0000336804600EB96008000D7F800A0F3F719
:10CEC000D9F926F00306CAF808003044CAF80C0065
:10CED0004D450DD10025454539682AD12046FFF73B
:10CEE000A9FE78600120F3F76BF906B0BDE8F08782
:10CEF0002046FFF7D7FDC3074FEA500613D430464C
:10CF0000F3F7B8F93246014682462046FFF7BDFDE9
:10CF10002046FFF7B7FD31465046F4F709F80646BC
:10CF20005046F3F7CFF93B689B6823F8156001354D
:10CF3000CEE72046CE68FFF7C3FD46F82500013551
:10CF4000C9E700BF67D002081CC0050828C0050853
:10CF50001FB50C46014601A817F0DAFF214601A8CB
:10CF6000FFF768FF04B010BD024B82681A61C26807
:10CF7000DA607047B4040020838803F4C071B1F50F
:10CF8000C07F02460FD0190604D5C37B00EB830295
:10CF90001069704713F4807006D0D37B02EB8302D4
:10CFA0001369586870470148704700BF0983030838
:10CFB00070B5274CF3F762FF00250123E561A4F863
:10CFC0001C32D4F820320BB1A4F81C52A4F8285219
:10CFD00003F0D8FF1F4B204E20486564C4E90F358D
:10CFE00003211F4BA364C4F8105284F8145203F0B9
:10CFF0004DFD0121304603F049FDAA22BA213046F9
:10D0000003F04EFE00210846C4E90366C4E92C552E
:10D01000C4E96B55E566C4F8CC50C4F8B85005F0C7
:10D0200097FF0A21C4F83C0105F007FD40F2E261D8
:10D03000D4F83C0105F001FD002106F1440005F0A3
:10D040003FFE40F21A7240F2DA63C4E9502370BD29
:10D05000B4040020E41C0608100500200005002090
:10D06000BC2A06087047D0E90230184708B5074BBC
:10D07000D86E08B9064808BD002241F622310430B6
:10D0800001F068FC0028F5D04068F4E7B404002003
:10D09000A8310608034BC0000A4640F00201D868D8
:10D0A00003F0FEBDB4040020034BC10041F00201B7
:10D0B000D86803F003BE00BFB4040020034BC000D7
:10D0C0000A4640F00201186903F0EABDB4040020EA
:10D0D000034BC10041F00201186903F0EFBD00BF2E
:10D0E000B4040020F8B51C46930707460E461546C3
:10D0F00008D113689A88910615D5520610D5B388C1
:10D100009B0501D52560F8BD50B9114B9E4207D053
:10D1100010490C2001F042FEC0E901652060F2E7F1
:10D12000C4E90057EFE70C4A934202D16B682360D1
:10D13000E9E70A4A9342E5D130B101F03BFE084BE2
:10D14000834214BF06463E466B68C4E90036DAE700
:10D150006022060854130608442B06082C2B0608E8
:10D160008C2B060800232DE9F041C2E900330E465E
:10D170000746144601F01EFE0A2E054602D1206025
:10D18000BDE8F081192E07D1838803F4C0731BB169
:10D19000144BC4E90037F3E76B7B5BB105EB83030A
:10D1A00022461B693146384698476368042BE7D10D
:10D1B00000236360EB7C002BE2D005EB8303F100DE
:10D1C0001869002241F00201043001F0C3FB00287D
:10D1D000D6D04268234629463846BDE8F041FFF7DD
:10D1E00081BF00BF1C310608F0B593B00546684604
:10D1F0000E4617461C46F2F7FDFF40B93A46314647
:10D200002846FFF7AFFFF2F7CBFF13B0F0BD002CBD
:10D21000FBD1019B044918680AF0D0FB0028F4D127
:10D220000198F2F7FFFF00BFA01B060808B519B967
:10D2300003F01AFFF2F7F6FF03F01CFFFAE70EB453
:10D2400003B503AA52F8041B019203F041FFF2F761
:10D25000E9FF000070B5124EC4000546306944F085
:10D26000020400222146043001F074FB0246A0B9FA
:10D27000F06E30B12146043001F06CFB08B140681B
:10D2800070BD00220748214601F064FB024620B928
:10D29000054906482A46FFF7D2FF5068F0E700BF6D
:10D2A000B4040020582D060834C00508A41A060846
:10D2B0000A4B10B50446D3E90303984207D0E100B6
:10D2C000002241F00201043001F044FB20B9204665
:10D2D000BDE81040FFF7BEBF406810BDB404002099
:10D2E000032837B505460C4607D1084601F09CFFD8
:10D2F00000B30E24204603B030BDCA072FD54B1013
:10D3000008282AD801A252F820F000BFF5D202085E
:10D310003DD302085BD302085BD3020831D3020875
:10D320005BD30208F5D2020839D30208F5D202080D
:10D33000002BDED01E24DDE7002BDBDAB3F1404FFB
:10D3400006D14FF0804003B0BDE8304005F01EB973
:10D350005B425B0043F00104CCE7DB43F9E70628BE
:10D3600025D101F00703022B10D08B071FD10B68CA
:10D370001A7BE2B103EB82031A69204B9A4216D161
:10D38000486840B98B68C86801930CE0CC08204617
:10D39000F3F77CFE18B1400040F00104AAE701A9B0
:10D3A0002046F3F796FE0199F3F758FDF3E7204680
:10D3B00001F000FDC37ABBB100EB83002146036995
:10D3C00028469847B0B9042DB4D0A5F10803022B24
:10D3D00012D90B4B20465D5D01F0F8FC094903466C
:10D3E0002A460948FFF72BFF062DECD1640044F0D4
:10D3F00001047FE704467DE700247BE749540308E6
:10D40000E22B060840C00508CC1906082DE9F041BA
:10D4100005460E461746984601F0CCFC847A54B176
:10D4200000EB8404434624693A4631462846A44624
:10D43000BDE8F0416047284601F0C8FC02490246B9
:10D440000248FFF7FCFE00BF49C00508CC190608DA
:10D4500000231A461946FFF7D9BF0000F0B515465C
:10D46000124A87B00C46116904910646D1680591AD
:10D4700002A80F49C2E90335F2F79AFE224637683F
:10D4800031466846F6F7F8FEB4FA84F25209394696
:10D490006846F9F7A1FF044615B1FFF7D9FF044626
:10D4A0000120F2F78DFE204607B0F0BDB404002045
:10D4B00069CF020807B50022019101AB0121FFF7F6
:10D4C000A5FF03B05DF804FB07B5CDE900126B467C
:10D4D00000220221FFF79AFF03B05DF804FB30B48D
:10D4E0005568003D144618BF0125C5F1020302EB43
:10D4F00083030A462918206830BCFFF787BF000065
:10D5000010B5044603F05AFE30B1002320461A46F7
:10D510001946FFF77BFF0446204603F069FE28B951
:10D52000BDE810400249034803F0A4BD204610BDE9
:10D530004FC00508CC1906087FB5114B0592C000F5
:10D5400040F002000190186902900620CDE9030125
:10D55000D86E78B1002241F65231043001F0FAF968
:10D5600040B1406801AB00220521FFF74FFF07B033
:10D570005DF804FB01A905200BF0FCFAF7E700BFFA
:10D58000B404002070B5164604460D46FFF7EAFDC8
:10D59000336893B9A30709D12268084B9A4205D191
:10D5A000E28807492B460748FFF749FE204601F06D
:10D5B0000DFC054902462B46F5E770BD8C2B06088D
:10D5C00070C00508A01B060879C0050807B56A46A3
:10D5D000FFF7D8FFDDE9000109B102F05BFC03B001
:10D5E0005DF804FB2DE9FF41174606460C461D4633
:10D5F00001F0E0FB374A904208D12B463A462146DB
:10D60000304604B0BDE8F04104F07EBB818811F4DF
:10D61000C07812D0062C2DD12F4F00233B62FFF78C
:10D62000ABFC0346304698472860D8B93B6A002BCC
:10D6300018BF1C462C60002015E0062C1AD101AA48
:10D6400019213046FFF78EFD019B7BB901AA8A2183
:10D650003046FFF797FF039401AA00210120FFF74E
:10D660003EFF2860012004B0BDE8F08101AA4146D8
:10D670004046F4E7002CE9D1384601F09BFB1749FE
:10D680000AF09CF901AA60B147213046FFF76AFD14
:10D69000019B73B101AA21462046FFF720FF2860B5
:10D6A000C9E79B213046FFF75DFD019B0BB1039756
:10D6B000D2E70B49384603F0AFFD30B109490A48BB
:10D6C00003F0D8FC28600220CDE73846FFF718FFAA
:10D6D000F8E700BF9C1E0608B4040020C01C060822
:10D6E000541C060881C005085C1A06087FB540F284
:10D6F000613102AA0546FFF735FD029CDCB12046E8
:10D7000001AA694601F0F4FC0024009BA34201D861
:10D7100004B070BD019B53F8240007F0EDFD02AA90
:10D72000014606462846FFF72DFF02993046FFF7CF
:10D73000B1FC0134E9E7284602AA40F26731FFF75D
:10D7400021FF029DAB68A342E2D9EB6853F8340095
:10D75000E60080B104280ED007F0E6FD03785F2BC9
:10D7600009D0EB6853F8340007F0C6FDEB6833448A
:10D770005968FFF78FFC0134E4E7000073B50546F4
:10D780000C46164601F016FB437B5BB10422CDE943
:10D79000002600EB83022146136928466A46984713
:10D7A000009B43B1284601F011FB04490246234681
:10D7B0000348FFF744FD02B070BD00BF79C0050803
:10D7C000A01B060873B50C46064601F0F3FA8388E1
:10D7D0001906054632D4C37BB3B14CB900EB8303C1
:10D7E0001A69174B9A4203D01020F2F743FD044602
:10D7F000EB7BAA8805EB8303D2051B69214648BF52
:10D800001B683046984778B96A460F213046FFF7C3
:10D81000A9FC009B53B11CB91020F2F72BFD044664
:10D820002146684604F060FB02B070BD304601F04E
:10D83000CDFA044902460448FFF701FD3046F3E7FC
:10D840004D6E030898C00508CC19060837B5044684
:10D8500001F0B0FA818811F4C0750AD0104B002293
:10D860001A62FFF789FB0346204603B0BDE830404B
:10D8700018476A4619212046FFF774FC009B3BB904
:10D88000204601F0A3FA074902460748FFF7D7FCF4
:10D890006A4629462846FFF722FE03B030BD00BF86
:10D8A000B4040020A5C00508CC19060830B505460B
:10D8B00095B000F051FF284601F07CFA848814F4FA
:10D8C000C0740AD01B4B00221A62FFF755FB0346B7
:10D8D000284615B0BDE8304018476A461921284649
:10D8E000FFF740FC009BE3B102A8F2F783FC01467E
:10D8F00040B96A46FFF7F3FD0446F2F751FC2046B3
:10D9000015B030BD039B0C4918680AF057F8034660
:10D91000039823B103F07AFB064B1862EFE7F2F7A6
:10D9200081FC284601F052FA044902460448FFF7F8
:10D9300086FC00BFB4040020541C0608A5C00508DE
:10D94000CC1906082DE9F04F8DB0136802930446F8
:10D95000002857D102F10408C1F307294FEA49030F
:10D96000CFB253FA81F14FEA810B58F8216076105B
:10D970005ED13546BB00039308EB8703009308EBA9
:10D980000B03019308EB870A4FF0000B019B9A45AC
:10D9900052D1D9444FEA490B07F1010A002E5FD159
:10D9A0000BEB0A05A800F2F765FC814614B1046090
:10D9B00057460126039A414609EB86001CF062FE99
:10D9C0003C46A344AB4506D948464FEA8B01F2F7E3
:10D9D0006CFC5D468146DFF804A22646DDE9003294
:10D9E000934240F08A80321B21464B4652080298EF
:10D9F000FFF70CFD04464846F2F764FC20460DB0E4
:10DA0000BDE8F08F546802F10808A5E726FA0AF38A
:10DA1000D80708D558F82A0001F0E8FB18B101F042
:10DA2000BFFA013805440AF1010A5745EED1A1E7D2
:10DA30004FF0000A5546F8E7DAF800206AB9DAF83C
:10DA4000040050B1810708D1026864498A4204D1B8
:10DA500003F023F90BF1FF3B83440AF1080A95E731
:10DA600055445D44A800F2F705FC81460CB1046002
:10DA700001244FF0000A5745A3D026FA0AF3DA072B
:10DA800058F82A0035D5830716D10368544A9342C3
:10DA900002D0544A93420FD108AA07A901F028FBEB
:10DAA000079A089909EB840092001CF0EBFD079B94
:10DAB0001C440AF1010ADEE708A9FFF783FEA7EB81
:10DAC0000A03039004930398FFF7F0FE034600282F
:10DAD000EFD0049A2244954207D8E90048460593BE
:10DAE000F2F7E3FB059B81466D0049F824300134D1
:10DAF000E9E749F824000134DBE7009BD3E9002B78
:10DB0000002A62D11BF0030726D1DBF80030534511
:10DB100022D1DBF808309F4203D3009B08330093E7
:10DB20005CE7DBF80C3053F837004FEAC70888B1E0
:10DB300004280FD000F00703022B01D008F0EEFB01
:10DB400049F82600DBF80C30B20043444A445B68D5
:10DB5000536002360137DCE708AA6A215846FFF70E
:10DB600011FD002108AA0846FFF7B9FC0021FFF7C4
:10DB700029FE03900398FFF799FE07460028CCD0B2
:10DB8000731CAB4207D3E9004846F2F78EFB4FEA1D
:10DB900045088146454607F00703022B03D0384667
:10DBA00008F0BCFB074608AA0F215846FFF7EAFC1D
:10DBB00008AA002101200A97FFF791FCB3004B440B
:10DBC00049F8267002365860D4E7B3004B4449F850
:10DBD00026200236C3F804B09FE700BFC01806082D
:10DBE000F82A0608D820060870B5830786B00C46C8
:10DBF00015461BD103681D4A934202D01C4A93422A
:10DC000014D102AA01A901F073FA019BA34227D300
:10DC100019D8029B043D03EB84049C4201D106B059
:10DC200070BD54F8042D45F8042FF6E702A9FFF75C
:10DC3000C9FD002306469C420193304606D8FFF7F3
:10DC400035FE0028EBD00B4922460BE0FFF72EFEF5
:10DC5000019B28B1E21A013A013345F82200EAE7B4
:10DC6000019A05490548FFF7EAFA00BFF82A0608B5
:10DC7000D8200608C8C00508B3C0050884190608DE
:10DC80002DE9FF4183071546CFB2C1F3072436D1F2
:10DC90000368384A934202D0374A93422FD1029008
:10DCA000029803AA01A901F023FA01983B198342C3
:10DCB0005AD80399002601EB8003A64214D1C01B59
:10DCC00001EB8701801B05F043F9039945F8260015
:10DCD000BC0005EB86080B1942468B420AD1002393
:10DCE000029304B0BDE8F08153F8042D45F82620D6
:10DCF0000136E2E753F8040D42F8040FEDE7002186
:10DD0000FFF760FD002380469F42019317D8002152
:10DD1000084605F01DF906464046FFF7C7FD0146D7
:10DD2000C0B9B368A3421FD345F8246005EB840251
:10DD300005EB8301AA4211D11B1BB360D1E740461A
:10DD4000FFF7B4FD019B78B1FA1A2244013345F87C
:10DD50002200D9E7304604F070FEDDE7F768881A44
:10DD6000385842F8040DE5E7019A04490448FFF7E2
:10DD700066FA00BFF82A0608D8200608B3C00508CE
:10DD8000841906082DE9F04F85B000AF07F10802AD
:10DD900005460C46FFF7E6F9D7E9020129B102F082
:10DDA00079F81437BD46BDE8F08F0028F9D107F1A6
:10DDB000080240F26B312846FFF7D4F9BB6823B95B
:10DDC0001E491F482246FFF73AFA07F10802284683
:10DDD0001721FFF7C7F9391DB86807F013FB824612
:10DDE0002046F3F75FF9D7F8049009F10106851989
:10DDF000EB1D23F00703ADEB030D6B464A4651467E
:10DE00004FEAD30B68461CF03DFC2E2309F83B304B
:10DE10002046F3F752F981462046F3F743F96E4462
:10DE20000246494630461CF02DFC29466846F3F769
:10DE30007FF801221E21FFF77FFBB2E7E2C0050851
:10DE4000581B060808B50446F2F716FB18B104493A
:10DE50000448FFF7EBF9044902482246FFF7EFF9BF
:10DE6000E8C00508C81A06080FC10508014608B52C
:10DE70000148FFF7DBF900BF841906082DE9F043DC
:10DE8000831E87B0054688461746062B3BD8DFE839
:10DE900003F0093A3A093A040F00B94212D04FF0A0
:10DEA0000E09ECE03A4607B0BDE8F04301F0E4B9F2
:10DEB000384603F083F940B13946404603F0ACF9E7
:10DEC0000028ECD04FF01E09D9E017F0030440F011
:10DED00000813A68A14B9A4240F0FB8007F10409A7
:10DEE0007B68A342DBD959F8046F304603F066F92A
:10DEF000002800F05D813146404603F08DF900288E
:10DF0000E0D10134ECE711F0010F00F0FF804E107A
:10DF1000F90740F1CE807C10232800F2DA80DFE898
:10DF200000F0B2B6D8BABED8D8D8D8121D20233D3A
:10DF300046484AD850586A72121D20233D46484A26
:10DF4000D850586A729446EA040090EA40034FEAB7
:10DF5000400900F1A88049F0010990E086EA040038
:10DF6000F3E706EA0400F0E7002C02DA7C48FFF74A
:10DF70007DFF1F2C09DC6FF040432341B34204DBDB
:10DF80004FF040432341B34205DD3046F11704F022
:10DF9000EDFA8046C0E006FA04F0D6E7002CE5DB97
:10DFA0001F2C2046A8BF1F2046FA00F0CDE73019ED
:10DFB000CBE7301BC9E786FB0404B4EBE07FC4D099
:10DFC000E3E7002C00F0F680214630460DF09AFF82
:10DFD000BBE7002C00F0EE8007EE906AB8EEE70A8F
:10DFE00007EE904AF8EEE77A80EE270A07B0BDE820
:10DFF000F04303F015BA002C00F0DC8021463046D7
:10E000000DF072FFA1E7002C1CDA07EE906AB8EE63
:10E01000E70A394607B0BDE8F04303F06DBA33466E
:10E020000120E20706D580FB0302B2EBE07FACD112
:10E03000012C8AD083FB0332B2EBE37F4FEA640406
:10E04000EFD0A2E7EBD101207FE7002C00F0B280F7
:10E050000021022008F0D0FC2146814630460DF018
:10E0600051FF400040F00100C9F808002146304649
:10E070000DF03AFF400040F00100C9F80C0048469E
:10E0800007B0BDE8F083A642FFF61CAF07E7A64243
:10E090003FF718AF03E7A6427FF714AFFFE6A642AB
:10E0A000BFF610AFFBE6C11707B0BDE8F04304F0C0
:10E0B0005DBABB072AD13B682A4A934219D107EEC1
:10E0C000906A3946B8EEE70A03F016FA814600284E
:10E0D000D5D1254B40465D5D00F078FE04463846BC
:10E0E00000F074FE21490090234621482A46FFF79C
:10E0F000A6F8204A934209D107EE906ADFED1E0A86
:10E10000B8EEE70A394602F061F8DFE7062D03D1E1
:10E1100043462425B8461F46404600F04BFE037B8D
:10E1200033B9A5F109030C2B0DD80D35EDB2F3E78A
:10E1300000EB83003A4603694146284698478146EA
:10E140000028EED09BE7A5F116030C2B16D843460A
:10E150000F35B846EDB21F46DEE700BFF82A0608C5
:10E160003DC10508681D0608B02B060852C1050808
:10E17000CC190608D416060800000000242D04D986
:10E1800043460F3DB846EDB21F46242DA1D102A94A
:10E190004046FFF717FB04462046FFF787FB0028A1
:10E1A0003FF47DAE394601F0DFF80028F4D089E66F
:10E1B00037468EE701490248FFF738F865C1050880
:10E1C000E81B0608014608B50148FFF72FF800BF15
:10E1D000CC1906082DE9F041044617461E460D46A7
:10E1E00041B1186800F0E6FD6368834202D005483B
:10E1F000FFF7E8FFA06833463A462946BDE8F041FC
:10E20000FFF704B971C10508014608B50148FFF7D9
:10E210000DF800BF381A060807B50022019101ABBE
:10E22000012102F043FEF1F7FDFF0000014608B5B1
:10E23000024809B9FEF7FAFFFFF7EEFF541C060883
:10E2400008B500F0C3FD024902460248FEF7F7FF99
:10E2500077C10508CC190608410008B5024841F00D
:10E260000101FFF7D9FF00BF801A060808B5024870
:10E2700042F28231FFF7D0FF5C1A060830B593B046
:10E28000044668460D46F1F7B5FF48B920462946D1
:10E29000FFF710F90446F1F783FF204613B030BDB5
:10E2A0000199024800F0C0FD0024F6E7C8080608FE
:10E2B000054BD861B3F81C2212B2012A04BF002218
:10E2C000A3F81C22704700BFB4040020EFF31081B4
:10E2D00072B6084AB2F81C321B0443BFB2F81C32B3
:10E2E00003F1FF331BB24FF6FF73A2F81C3281F328
:10E2F00010887047B4040020EFF3108172B60C4B05
:10E30000B3F81C22013212B2A3F81C2252B9DA6906
:10E310002AB9D3F8202212B993F828222AB1002270
:10E32000A3F81C2281F3108870470122F8E700BF90
:10E33000B404002070B5EFF3108572B60F4B93F85C
:10E340002822082A18D0B3F81C4224B2012C04BF9A
:10E350000024A3F81C4293F82942561C224402F0E0
:10E360000702283283F8286203EBC203C3E90201E3
:10E37000012085F3108870BD0020FAE7B404002066
:10E380000228F8B52C4C034610D0E26972B1EFF3C5
:10E39000108272B6E06938B10021012BE16103D12E
:10E3A00082F31088F1F73EFF82F31088B4F81C3234
:10E3B0001BB243B9EFF3108272B6B4F81C6236B2E6
:10E3C00016B182F31088F8BDD4F824724FF6FF73AB
:10E3D000A4F81C3297B1D4F820526B68C4F82032EC
:10E3E0000BB9C4F824322B682E6082F310882846BB
:10E3F0009847EFF3108272B6AF42ECD194F82852EE
:10E40000BDB194F8293203F12801013304EBC101B5
:10E4100003F00703013DD1E9020184F8293284F8B1
:10E42000285282F31088FFF729FFBDE8F840FFF774
:10E4300063BF82F31088F8E7B40400200120FFF7DF
:10E440009FBF08B5FFF7FAFF30BF08BD08B5FFF75B
:10E45000F5FF30BF08BD000038B1044A1369984287
:10E4600002D010611846704700207047B4040020A5
:10E4700001F00F0108290DD8DFE801F011050A0CA1
:10E480000C0C0C0C0E0000280CBF0E201E20704738
:10E4900004F07CB804F095B8C00040F0020070476A
:10E4A00008B500F0D3FD10EE100A2AF0B1FB41ECE4
:10E4B000100B08BD00F0CABD08B551EC100B2AF0D6
:10E4C000FFFBBDE8084000EE100A02F0A9BF02F011
:10E4D000A7BF0000F0B593B00546684616680F4622
:10E4E0001446F1F787FE78B9002E0CBF394600219B
:10E4F000234632462846FFF775F80546F1F750FEE9
:10E50000012D0CD1284612E0019B236010492068A0
:10E5100002F082FE034620685BB9F1F783FE2368B0
:10E52000002DF3D10BB90623236036B9002013B0B8
:10E53000F0BD02F06BFD2060F7E70649304602F0BF
:10E540006BFE0028F2D03046FEF7DAFFE5E700BFA9
:10E55000541C0608C01C0608036803B94068FFF78E
:10E56000A5B91346C1F30722C9B2FEF74FBF1FB5C5
:10E5700001F00F03012B04460CD011F00E0F0BD04D
:10E58000023B012B0AD9012201A900F035FF50B14D
:10E59000019801E000F048FE04B010BD04B0BDE8F1
:10E5A000104000F009BD204600F006FDF4E708B574
:10E5B00028B1062803D0FEF7A3FFF1F733FE08BD0C
:10E5C00010B50C4619B9BDE81040FFF7FBB8FFF7CE
:10E5D000F9F884421CBF0023C4E90030002010BDBC
:10E5E00040F2C143984217D840F2BD43984209D83F
:10E5F0005E281DD075281DD03E2814BF4FF0FF3077
:10E6000001207047A0F2BF40022815D8DFE800F0D3
:10E610000C0E02000520704740F25353984214BF7D
:10E620004FF0FF30032070470620704707207047E7
:10E6300002207047002070470420704738B5034619
:10E6400014460D4661B152B111462846984760B153
:10E650006B683BB96C6045F00103AC60E3602C462D
:10E66000204638BDAB68DC60F5E76368EB60656049
:10E67000002BF5D144F00103A560EB60F0E7F8B59D
:10E68000064631B1002511F0010304D00023EB60F0
:10E6900029460846F8BDCC68CB6014F0010307D1C9
:10E6A000E768E36022463046FFF7C8FF3C46014674
:10E6B0000A4630462946FFF7C1FF21460546E2E7F4
:10E6C0008A422DE9F04184460F4606D10023516865
:10E6D0005360BDE8F041FFF7D2BFD66896B114464B
:10E6E000E468E307FCD524F00104516863689342B1
:10E6F00006F0010816D1002339B9984518BF1E4607
:10E700006660D1603846BDE8F0815360D3606046F2
:10E71000FFF7B5FF05466060EE60B8F1000FF1D07D
:10E72000A560EFE71D46DB689342FBD100225A60EB
:10E73000DA606046FFF7A3FF0028EDD0E8600546E9
:10E74000EAE70000034B82B0186801ABC01A02B0C0
:10E75000704700BFB404002007B5064A136852682A
:10E7600001A95B1A9A4201D8FFF780FD03B05DF85A
:10E7700004FB00BFB404002010B503461446500C3F
:10E78000C2F34F0221B1E10702D40C48FFF71AFD92
:10E79000904206D198420FD0094902460948FEF737
:10E7A0004EFD984204D9C21A07490648FEF747FDB4
:10E7B0009A4201D20549F1E710BD00BF7EC10508AC
:10E7C00088C10508CC1906089AC10508A2C1050828
:10E7D0002DE9F74FDDE90CA7002406468B461546C8
:10E7E0000193A046A146019B9C4204D1B1453CD275
:10E7F0002248FFF7E7FCB44210D2BAF80220920593
:10E80000F6D45BF8240009F101099AF80220012AE4
:10E8100024D100F009FD07F8240017E0BAF8001031
:10E82000C900002241F00201284600F093F888B99F
:10E83000BAF80220D30505D5BAF8002010491148CE
:10E84000FEF7FDFCDAF8042047F8242001340AF131
:10E85000080AC8E7406808F10108D6E7022A01D192
:10E8600000F09EFB47F82400F0E72B68B8EBD30FCD
:10E8700001D20548BDE703B0BDE8F08FBDC1050872
:10E88000B8C10508CC190608C7C1050870B586B01F
:10E890000446154602EB800203A81E4600F031F83C
:10E8A0000B9B01930A9B009303AA334629462046FB
:10E8B000FFF78EFF06B070BD08B50148FFF7A4FC56
:10E8C000D1C1050807490346002231F8020B9842DE
:10E8D00006D20132222AF8D103EB530343F00100A0
:10E8E000704700BFD014060810B50446416019B93E
:10E8F0000123A160236010BDC800F1F7D4FC0146DC
:10E90000F6E74160C90041F007010160826070478D
:10E9100003789B0710B5044602D48068F1F7D2FC57
:10E920002368002262F3DF036260236010BD037876
:10E930009B0710B5044602D48068F1F7C3FC236836
:10E9400003F0040343F0010323600023C4E901330F
:10E9500010BD00002DE9F04F022A85B004460E4696
:10E96000904612D0426882B1904BC1F386010B44AD
:10E9700093F82A32B3FBF2F102FB1133826802EB07
:10E98000C30552F83330B34213D0237813F0010299
:10E99000019213D006F00702022A0FD016F00302EC
:10E9A00003D130688249884207D0B8F1010F05D001
:10E9B0000025284605B0BDE8F08F01925B076AD5B7
:10E9C0002768A56827F007072F44BD4232D3B8F166
:10E9D000010FEDD1D4E90032B2EBD30FC3F3DC0168
:10E9E00011D104316160A068C900F1F75EFCD4E97F
:10E9F0000032A2EBD30223F00703A060D200002173
:10EA000018441BF083FE2368A168C3F3DC02501C8A
:10EA100001EBC20560F3DF03236041F8326000229E
:10EA200006F007066A60022EC3D0237862F3000363
:10EA30002370BEE72868B04224D1B8F1020F17D185
:10EA40002368D5F80480083B7A1B05F10801236090
:10EA5000083A28461BF046FE2568A368C5F3DC0289
:10EA600025F007051D44002143F83210C5F8048045
:10EA70004E4BC6F386061E44A368EB1ADB1086F8DD
:10EA80002A3296E7019B23B9314600F06DFC00283D
:10EA9000D3D1083599E763682BB9B8F1010F87D155
:10EAA000204600F087F806F0070BBBF1020F2BD1D0
:10EAB000F008F2F7EBFA81466368B9FBF3F203FB67
:10EAC000129A57460025A26852F83700FB000293BD
:10EAD00002EBC703F8B9B8F1010F7FF469AF226800
:10EAE000C2F3DC010131002D18BF2B4661F3DF02B8
:10EAF000BBF1020F2260C3E9006003D0227860F30B
:10EB0000000222701D4654E731460620FEF7E8FB5E
:10EB10004FEA6009D0E7042819D1002D08BF1D462F
:10EB200063680137B7FBF3F203FB1277BA45CAD12A
:10EB3000B8F1010F7FF43CAF002D32D023680022E2
:10EB400008332360BBF1020F2E606A606CE7B042AD
:10EB500018D1B8F1020F0ED1216860680839216020
:10EB6000791CB1FBF0F500FB1511A06850F83110CD
:10EB7000A9B9F80011500D4AC6F38606164486F866
:10EB80002A72BFE701990029CAD13146CDE9023284
:10EB900000F0EAFBDDE902320028C1D0D9E7042108
:10EBA000E7E7204600F006F886E700BFB40400203F
:10EBB000B02906082DE9F04146680446701CFFF7AD
:10EBC00081FE0546C000A768F1F76DFB236865600C
:10EBD00003F0060343F001032360A0603D1D4FF0E6
:10EBE0000008B04504D13846BDE8F041F1F76ABBF2
:10EBF00055F8041C39B1042905D001222046FFF73D
:10EC0000A9FE2B68436008F101080835E9E710B553
:10EC100000230446016043608800F1F744FBA060D4
:10EC200010BD03682DE9F74F04460F46934623B9FC
:10EC300012F0010F65D000F067F839460620FEF7A4
:10EC40004FFB4FEA600A2368BAFBF3F603FB16A6F4
:10EC500035464FF00008A16851F82590AA0001EB55
:10EC60008503B9F1000F0CD11BF0010F49D0626888
:10EC7000B8F1000F18BF4346013262601F60B94609
:10EC800033E0B9F1040F17D1B8F1000F08BF98466F
:10EC900023680135B5FBF3F203FB1255AE42DAD11E
:10ECA0001BF0010F2DD0B8F1000F26D0636801339F
:10ECB0006360C8F80070E2E739464846019200F008
:10ECC00053FB019A0028E3D01BF0020F0DD06368BC
:10ECD0002068A168013B63606B1CB3FBF0F400FB90
:10ECE000143351F8233023B98B50484603B0BDE8A4
:10ECF000F08F042341F82530F7E7204600F004F8B0
:10ED0000A1E74FF00009F0E7F8B507688668044608
:10ED1000781CFFF7D7FD0025206065608000F1F7C3
:10ED2000C2FAA060BD4204D13046BDE8F840F1F718
:10ED3000C9BA56F8251029B1042903D0012220466A
:10ED4000FFF76FFF0135EDE770B50168024600235C
:10ED5000994201D1002015E0946854F823009E00E8
:10ED600001330028F4D00428F2D05568013D5560E5
:10ED7000B3FBF1F201FB123354F82330002B18BF20
:10ED80000423A35170BD10B504468068F1F79AFAC8
:10ED90000023C4E90033A36010BD704710B50C46D2
:10EDA000F1F768FA046010BD10B50C46F1F770FA7F
:10EDB000046010BD83070FBF0068034B00F00F0015
:10EDC00053F82000704700BF1415060808B5FFF778
:10EDD000F1FFBDE80840C088F2F76FB970B50D4685
:10EDE00004461646FFF7B8FC2846FFF7E3FF437AD0
:10EDF00043B100EB83033246294620461B69BDE838
:10EE000070401847C28803492046BDE87040F2F7B9
:10EE1000EFBE00BFF6C105080A4601460148FFF7EC
:10EE2000DDBF00BF18390608F7B5044608460E4690
:10EE300002F0DEF970B101AA6946304602F03AFAF2
:10EE4000009B3BB116492046F2F719FB009D033D9C
:10EE5000002D0BDA314620460222FFF7BFFF114991
:10EE6000204603B0BDE8F040F2F709BB019A0E4915
:10EE700002EB850320465B6852F82520F2F7B8FEC6
:10EE8000019BAF003B449A6822B906492046F2F73D
:10EE9000F6FADCE705492046F2F7AAFED7E700BFFD
:10EEA000FBC1050875D805081FC2050834C205084E
:10EEB00008B50246FFF77EFF837A53B100EB830368
:10EEC00006491B698B4204D1BDE80840104608F092
:10EED00049BD181E18BF012008BD00BF897703086F
:10EEE000830710B5044603D10268084B9A4208D044
:10EEF00021460820FEF7F4F910B92046FFF7A0F9E3
:10EF000004462046BDE8104003F0CEBCC01F0608F2
:10EF1000830713B5044603D102680D4B9A4208D00B
:10EF200021460820FEF7DCF910B92046FFF788F9E2
:10EF3000044614F0010103D06010E11702B010BDC7
:10EF40006B460822204603F049FADDE90001F5E7A7
:10EF5000C01F06080E2838B503460C4604D100230E
:10EF600023600125284638BD1E2801D10123F7E77B
:10EF700010F0010501D04310F2E7820707D10168C4
:10EF8000064A914203D103F045FB2060E9E71946A8
:10EF90000820FEF7A5F90028F5D1E3E7C01F060811
:10EFA00013B501A90446FFF7D5FF10B92046FFF7B6
:10EFB00047F9019802B010BDC20705D4830705D1F7
:10EFC0000268034B9A4201D103F01DBBFFF7E8BF73
:10EFD000C01F06080E2838B503460C4629D01E2847
:10EFE0002AD010F0010508D0431000EE103AB8EE18
:10EFF000C00A84ED000A012519E081070CD10268DE
:10F000000F498A4202D103F067FCF2E70D498A42B8
:10F0100002D102F06DFAECE719460920FEF760F91B
:10F0200028B1820703D10268064B9A42F1D02846E4
:10F0300038BD9FED050ADCE7B7EE000AD9E700BF4F
:10F04000C01F0608681D06080000000013B501A9CE
:10F050000446FFF7BFFF38B92046FFF7B7FE044963
:10F0600002460448FEF7EBF89DED010A02B010BD20
:10F070003DC20508CC190608F8B504460F461646E9
:10F08000FFF7A8FF054620B100233360012528467D
:10F09000F8BDA10709D122680B4B9A4205D132462F
:10F0A0003946204601F08CF8F0E721460A20FEF7A9
:10F0B00017F90028EBD08207E9D10268024B9A4287
:10F0C000E5D132463946EDE7D416060810B50446B8
:10F0D000FFF7D2FF38B92046FFF778FE0249024613
:10F0E0000248FEF7ACF810BD48C20508CC19060866
:10F0F000830710B50FD103680A4CA34204D14368BB
:10F100000B600830106010BD074CA34203D1836828
:10F110000B60C068F6E7FFF759FE04490246044851
:10F12000FEF78DF8F82A0608D82006084FC2050811
:10F13000CC19060813B50C4601A9FFF7D9FF019BAE
:10F14000A34204D0034904482246FEF778F802B0EF
:10F1500010BD00BF58C2050884190608F7B51F4640
:10F16000D30706460D4614460DD554100194019858
:10F17000002823DA2844B7B100281DDBA84228BFA5
:10F18000284603B0F0BD01A91046FFF7E3FE0028B2
:10F19000EDD12046F588FFF719FE0A4903462A46B5
:10F1A0000948FEF74CF8002801DBA842E9D3F288B1
:10F1B00006490748FEF743F80020E2E7002FDDD1BB
:10F1C000F3E700BF6AC20508CC19060881C205082A
:10F1D000101B0608820701D003F0D8B9002801DA15
:10F1E00003F0EFB9400040F001007047830710B50D
:10F1F000014608D102680B4B9A4204D18068400056
:10F2000040F0010010BD0846FFF7D4FDC37A33B1CA
:10F2100000EB8300BDE8104003690520184718463D
:10F22000F0E700BF802906080E2810B5044620D05C
:10F230001E281CD006281CD0C20703D5013818BFD1
:10F2400001200EE0FFF7B6FDC37A5BB100EB83004F
:10F25000214603690420984720B1A0F11E035842BB
:10F26000584110BD2046FFF7C1FF0138E7E70120F4
:10F27000F7E70020F5E7000005282DE9F04707BF74
:10F280004FF00E084FF01E094FF01E084FF00E0908
:10F29000914207460C46154607D1C8075FD4084679
:10F2A000FFF788FD8388590759D504F00703022B1F
:10F2B00005D0A20717D122682A4B9A4213D105F034
:10F2C0000703022B05D0AB0712D12A68254B9A42BF
:10F2D0000ED12946204605F0C8FF00283FD14B46F5
:10F2E0001846BDE8F08714F0010623D0EE07F6D4E7
:10F2F00001262846FFF75EFD027B82465AB38188CD
:10F30000080704D42046FFF755FD824523D1052F79
:10F3100014D09AF80C300AEB830322461B69294665
:10F32000022098470346B0B1022FD9D0FFF77CFFE7
:10F33000D3E701262B4625461C46DAE7CB06E8D55F
:10F340000AEB82022946136938462246984703464B
:10F350000028DED0C4E7002EEBD0AC42BFD143463C
:10F36000BEE700BFB029060808B50A4601460220DC
:10F37000FFF782FFBDE80840FFF756BF10B504460F
:10F38000FFF734FF38B92046FFF720FD0249024657
:10F390000248FDF754FF10BD88C20508CC190608C5
:10F3A00038B50446FFF706FD837B15462BB100EB0D
:10F3B0008300036920469847A0B9204635B9FFF776
:10F3C00005FD094902460948FDF739FF042D04D11E
:10F3D000FFF7FCFC06490246F5E7FFF7F7FC054995
:10F3E0000246F0E738BD00BF95C20508CC190608F3
:10F3F000A8C20508BAC2050838B50546FFF7DAFC09
:10F40000037C14461BB914F004000BD138BD00EB8B
:10F41000830302F003021B69284698470028F2D1B3
:10F420000120F3E70148FEF7CDFE00BFC5C2050885
:10F43000042803D0052807D0002070478B68002BD4
:10F440000CBF0E201E2070478868400040F001006D
:10F4500070470000084A0346C1E900230022C1E9C1
:10F4600002220846054A1968914202BF5B68C3F34D
:10F4700017238360704700BF5C150608A8150608AF
:10F48000F8B50D460179044601F07F01164640208B
:10F49000002208F049FFA268E36827682B60424316
:10F4A0006A60227902F07F01A96009498F4201D088
:10F4B0000020F8BD110601D4B20706D46268C2F379
:10F4C000172200FB02332B60F2E70120F1E700BFB7
:10F4D000A8150608F8B5002205460E46014640204C
:10F4E00008F022FF07461020F0F7C4FE094A0A4B35
:10F4F0000571012D08BF13460360436803F0FF0345
:10F500000446C0E9013606FB07F0F0F7B3FEE06001
:10F510002046F8BDE8150608741506084268C36859
:10F5200091688B4230B40AD21479D16882685D1C2C
:10F53000C5601A4404F07F0030BC08F069BF0020A9
:10F5400030BC70474368FF2B70B504460E461AD88E
:10F5500001790022402008F0E7FEA1680831054645
:10F560004143E068F0F7A1FE6368E060082262F3BF
:10F570001F236360A36803FB0553C5EBC50200218D
:10F5800018441BF0C3F820793346D4E9022109F06E
:10F590007BF9A3680133A3606368A3F5807363609C
:10F5A000062070BD70B50E79012E05460C460ED1B1
:10F5B0001949F1F764FFD4E902213346284605F0E2
:10F5C000EFF828461549BDE87040F1F758BF1449D7
:10F5D0003246F2F70DFBA368002BF2D01149284602
:10F5E000F1F74DFF0026A368B34204D80E49284620
:10F5F000F1F745FFE5E71EB10C492846F1F73FFF5B
:10F600003246E168207908F003FF012201462846CE
:10F61000FFF7E4FB0136E6E7D3C2050803E005087F
:10F62000DFC20508EAC2050881D70508EEC2050851
:10F630002DE9F04F044689B00D4616460AB900255B
:10F64000DDE011F003078068DFF844A240F0EC80B1
:10F650000B68874A934240F0E78002AA08F0F8FA64
:10F6600010B98448FEF7D0FD2179042E01F07F0106
:10F670003A464FF0400000F0A38008F055FE16F027
:10F680000302054662D131688B7B002B4FD001EB22
:10F6900083031869784B984249D13179402001F0B1
:10F6A0007F0108F041FEA84202D07448FEF7DEFB5D
:10F6B00033685345D6E9029B45D17368C3F31728D5
:10F6C00005FB08F8DDE902032268E7681B1A5245CA
:10F6D000A9EB03063CD194F90420002AAFDA002EEE
:10F6E000E3D16268C2F3172205FB027705FB09F23A
:10F6F0000BEB080105FB007001931AF0F3FF03996F
:10F70000A2680298521A48446A4305FB017105FB3E
:10F7100000701AF0E7FF019BA068A3EB09023044D8
:10F720006A43002105FB00701AF0F0FF3BE0544BE8
:10F7300099420BD1012DB8D1052205A93046FFF71A
:10F740005BFEDDE905B94FF00008BBE74D4889E7EE
:10F75000002ECBDD6368B6EB132F2FD9A16831449F
:10F7600069433846F0F7A1FD6368E06066F31F2344
:10F7700082466360BB4508BF83460298A26803992E
:10F7800048443244121A6A4301FB05A105FB00A05C
:10F790001AF0A8FF029805FB09F20BEB080100FB29
:10F7A00005A01AF09FFF6368C6EB132262F31F23C4
:10F7B0006360A3683344A360062520E0BA46DCE713
:10F7C00008F0B2FD2268029B524506461BD1B3F1F8
:10F7D000807F03DB2C492D48FDF728FD1020F0F732
:10F7E00049FD054694E80F0085E80F00029A02EBF8
:10F7F000112363F31F216960039B9B1AAB602846AA
:10F8000009B0BDE8F08F03992079C91AFFF762FEAD
:10F81000DDE90232E168D21A0546724306FB0311A4
:10F82000C0681AF02FFFEAE700232A460146206845
:10F83000FFF794FC23685345024620790ED1636894
:10F84000042E02EB13220BD003067FF5F8AEE1681D
:10F85000334600F07F0009F017F8ADE7042EF6D12B
:10F86000E16800F07F0009B0BDE8F04F08F0D0BDBE
:10F87000A8260608F1C2050831F6020815C30508D6
:10F880008029060830C305084BC305080C1C060870
:10F89000A81506082DE9F043012885B007460E4655
:10F8A00008D08B0724D10B68254A934202D0254A01
:10F8B00093421DD1012201A93046FFF79DFDB8B149
:10F8C00000223946402008F02FFD029EB6FBF0F6DC
:10F8D000054631463846FFF7FDFD0199044606FB13
:10F8E00005F2C0681AF0CEFE204605B0BDE8F083F0
:10F8F0003046FFF77BFC054600B1451029463846E7
:10F90000FFF7E8FD002104463046FDF75BFF4FF0AE
:10F91000000806463046FDF7C9FF03460028E3D03D
:10F9200025B919462046FFF70DFEF3E74246E16888
:10F9300008F10109384608F0A7FFC846EAE700BF0A
:10F9400080290608E815060838B50C4620461146F9
:10F9500006221D46FEF710FF2CB92146BDE83840AF
:10F960000120FFF7B7BD2968CA0705D48B0708D166
:10F970000B680C4A93420DD10846FFF711FB014674
:10F98000ECE701F00703022B07D1012C05D1064853
:10F99000FEF718FC054A9342F6E7BDE8384001201F
:10F9A000FFF778BFC01F060860C30508B029060826
:10F9B00038B50D461C4611462846094AFEF7DCFEBE
:10F9C000206805F0B1FC012D007804D1BDE8384075
:10F9D0000021FFF77FBD6168BDE83840FFF75ABFDF
:10F9E00004000200F0B50F4685B001A904460122CB
:10F9F0003846FFF701FD014678B93846FDF7E2FECB
:10FA000005462846FDF752FF014610B9062005B00D
:10FA1000F0BD2046FFF796FDF3E700222179402054
:10FA200008F082FC6368029DB5FBF0F5B5EB132F7F
:10FA30000646C3F317221ED9A16829444143E06852
:10FA4000F0F733FC6368E06003F0FF03BC426360DF
:10FA500004D1052201A92046FFF7CEFCD4E9020318
:10FA6000019900FB063005FB06F21AF00BFEA368B5
:10FA70002B44A360CAE7521B62F31F236360EDE7C8
:10FA8000F0B51B288DB006460C46154626D005D885
:10FA900004286BD90E2850D000244BE02428FBD139
:10FAA000012203A92846FFF7A7FC00284ED0A10792
:10FAB0005AD12268474B9A4256D1012209A92046C1
:10FAC000FFF7DEFC01230093DDE90901DDE90323F3
:10FAD00004F02CFF002847D01E242BE00A683E4B80
:10FAE0009A42D9D0012206A92046FFF7C9FC052277
:10FAF00009A92846FFF780FC9DF8207000223946AE
:10FB0000402008F011FCA1680A9EB6FBF0F60546FD
:10FB100031443846FFF7DEFC079F069904463A4613
:10FB2000C0681AF0AFFDE068099906FB05F2384499
:10FB30001AF0A8FD20460DB0F0BD0A68264B9A4287
:10FB4000AAD029462046FFF74DFFF3E7EA0702D582
:10FB50000020FEF759FBAB0706D12B681F4A9342E2
:10FB6000F6D01F4A9342F3D00E24E3E7012206A900
:10FB70002046FFF785FC012209A92846FFF73CFC37
:10FB80000028F1D0089A012A1DD05A2A1DDC203203
:10FB900001460B9B012B1AD05A2B01DC2033014666
:10FBA0009342D5D123F00203642BD1D0022E01D091
:10FBB0000029CDD00A9B0093DDE90612099B30464F
:10FBC00008F085F886E74222E1E70021E1E74223D9
:10FBD000E4E700BFE8150608A8150608C01F0608D8
:10FBE000681D060870B50646102014460D46F0F74D
:10FBF00041FB054A067102604268C46002F0FF02E0
:10FC0000C0E9012570BD00BFA81506087FB51D46D7
:10FC1000084611464FF00212FEF7AEFD052201A97B
:10FC20002868FFF7E9FB9DF80C40029E2146002260
:10FC3000402008F079FB019AB6FBF0F12046FFF76F
:10FC4000D1FF04462868FFF7B5F80D4B834209D170
:10FC50002A6861685368C3F3172363F31F21616047
:10FC6000D368E3602868032201A9FFF7C5FB18B138
:10FC7000237963F07F032371204604B070BD00BF79
:10FC8000A815060870B505460E4601460120FFF787
:10FC900021FC2A4604463146C0681AF0F3FC20468F
:10FCA00070BD000038B505460C4610200349FFF72B
:10FCB00075F80122C0E90125C46038BDE8150608C1
:10FCC000136870B56BB94468A51C50F825509C4268
:10FCD00007D055F82360B14204D1023350F82330E5
:10FCE000136070BD0133F2E72DE9F0410F46124970
:10FCF00016460446F1F7C3FB06F1040800257368B5
:10FD0000AB4205D820460D49BDE8F041F1F7B7BB3D
:10FD10001DB10B492046F1F7B2FB57F825200949E0
:10FD20002046F1F765FF58F8041F01222046FFF72F
:10FD300055F80135E3E700BF78C5050803E005087D
:10FD4000EEC2050874C305084B6802330A4651F831
:10FD50002310FFF7C9BF0E3918BF0121490041F038
:10FD60000101FEF78BB8052807D00E3918BF012115
:10FD7000490041F00101FDF7B3BA002070470000CF
:10FD8000032A05D10E2914BF04490549F1F777BBB1
:10FD90000E2914BF03490449F8E700BFA8BA0508B3
:10FDA000ADBA0508C2A50508ED9A050838B50C4698
:10FDB0002046114602221D46FEF7DEFC1CB12868D3
:10FDC000FFF732FA08B90E2038BD1E20FCE70628DE
:10FDD00001BFD1E901305840400040F0010018BF98
:10FDE0000020704702280AD188689368984208D199
:10FDF0004868536898420CBF1E200E2070470020B0
:10FE000070470E207047136813B94068FDF7AAB910
:10FE100070472DE9F84F984602EB43035D1C042B15
:10FE200000AF82468B4616464FEA85051FD8EB1D6C
:10FE300023F00703ADEB030D6C464FF0000920469D
:10FE4000B96A40F804BB2A1F1AF01CFC234642463C
:10FE5000711C5046FDF7DAFA0446B9F1000F02D0E2
:10FE60004846F0F72FFA2046BD46BDE8F88F2846F1
:10FE7000F0F70BFA04460028D9D08146DFE707B532
:10FE8000009313460A46D0E90101FFF7C2FF03B011
:10FE90005DF804FB38B505460C460C200249FEF718
:10FEA0007DFFC0E9015438BD6C16060810B5034942
:10FEB00004460820FEF772FF446010BD9016060845
:10FEC0002DE9F04F866806EB010A04460AEB420072
:10FED00001EB4209052887B00F46154698464FEAC0
:10FEE000890904F10C0B16D801AFB6003246594609
:10FEF00038461AF0C7FB4A464146B8191AF0C2FB09
:10FF000060683B462A465146FDF780FA0446204683
:10FF100007B0BDE8F08F8000F0F7ACF9A268594651
:10FF2000920006461AF0AEFBA0684A46414606EB30
:10FF300080001AF0A7FBA168606833462A4639445E
:10FF4000FDF764FA04463046F0F7BCF9DFE7406895
:10FF5000FDF708B92DE9F041CD1CAD0080460E46F5
:10FF6000284608491746FEF719FFA5F10C02C0E91B
:10FF70000186044639460C301AF084FB2046BDE861
:10FF8000F08100BFA4160608D1ED017AF5EE407AA3
:10FF9000F1EE10FA73B504460D4624D01349144E01
:10FFA000F1F76DFA4FF0FF336320CDE90030002305
:10FFB0001A4695ED010A67212046F1F7F7FB022268
:10FFC0004FF0FF336321CDE90031204695ED020A61
:10FFD00000236721F1F7EAFB3146204602B0BDE875
:10FFE0007040F1F74CBA034E0022E9E778C50508E6
:10FFF00078C305087BC30508136810B5144643B9D8
:020000040803EF
:1000000040F2E543994205D190ED010A01F008FA6A
:10001000206010BDB1F5876FFBD190ED020AF5E7C6
:1000200008B508492DED028B0C20F0EE408AB0EEA9
:10003000608AFEF7B3FEC0ED018A80ED028ABDEC56
:10004000028B08BDD416060808B5072841D8DFE89A
:1000500000F01326404004401532D1ED017AF5EE50
:10006000407AF1EE10FA36D1D1ED027AF5EE407A0F
:10007000F1EE10FA2FD10E21084608BDD1ED027A1B
:10008000FDEEE77A17EE903AD1ED017AFDEEE77AD0
:1000900017EE902A53405B0043F00101ECE7D1EDED
:1000A000020A91ED010ABDE80840F1EE600AB1EEE6
:1000B000400AFFF7B5BF91ED020AD1ED017A20EEBB
:1000C000000AA7EEA70A1AF0D9FABDE8084001F025
:1000D000A7B90021D0E71E21CEE7000030B52DEDF5
:1000E000028B0C4685B01146204604221D46FEF7C1
:1000F00043FBF4B1012C286826D082074DD1026859
:100100002C4B9A4249D190ED018AD0ED028A686861
:10011000830749D10268274B9A4245D1D0ED027A34
:1001200038EE678AD0ED017A78EEA70AB0EE480A79
:1001300003E0DFED210AB0EE600A05B0BDEC028BF2
:10014000BDE83040FFF76CBF00F00702022A03460B
:1001500005D0810716D1026818498A420FD103A938
:1001600005F050F900230093012303991A46FCF788
:1001700023FB0346184605B0BDEC028B30BD0D498C
:100180008A42F7D003AA02A9FEF7A0FFDDED030A19
:100190009DED020AFFF744FFEBE7FEF757FFDFEDA7
:1001A000068AB0EE408AB2E7FEF750FF70EE280AEA
:1001B000BCE700BFD416060800000000B0290608FE
:1001C00043680B60836813607047000010B52DED25
:1001D000048B82B0044601AA08466946B0EE409AF4
:1001E000B0EE608AFEF748FF002800F0CC80A01E29
:1001F000202800F2CC80DFE800F0B6CACACACACA1A
:10020000CACACACACACA11205BCA292CCA68CACAC1
:10021000CACACA11205BCA292CCA6800DDED008A4F
:10022000DDED017A79EE288A38EE278AF0EE480A69
:10023000B0EE680AFFF7F4FEA5E0DDED008ADDED23
:10024000017A79EE688A38EE678AEFE75248FDF75F
:10025000B9FFDDED017A9DED007AF5EE407AF1EE21
:1002600010FAB5EE407A0BD1F1EE10FA03D14B49FA
:100270004B48FCF7DBFFC9EE078A88EE078AD5E713
:10028000F1EE10FA06D1B1EE499AC8EE278A89EE4E
:10029000278ACBE767EEA76AF1EE677AE7EE076A8F
:1002A00087EE266A87EEA67A8DED006A8DED017ADB
:1002B0009DED007ADDED017A68EE678A27EE088A07
:1002C000E7EE098AA7EE898AB0E728EE080AA9EEC8
:1002D000090A1AF0D3F9B5EE400AF1EE10FADDED95
:1002E000019A19D1F5EE409AF1EE10FA12D1DDED36
:1002F000007AF5EEC07AF1EE10FA0BDBF5EE407AFB
:10030000DFED287AF1EE10FAF7EE008A18BFF0EE72
:10031000678A8BE72449ABE719F016FBF0EE490A30
:10032000F0EE408AB0EE480A17F0B6FBDDED007A39
:10033000B0EE408A27EE888A29EEC00AA8EEA98A84
:10034000A7EEA80A19F030F9B0EE409AB0EE480ACC
:1003500019F0B8FC60EE098AB0EE480A1AF000F90C
:1003600020EE098A62E7DDED007AF4EE497AF1EEDB
:1003700010FA0ED1DDED017AF4EE487AF1EE10FAC2
:100380000CBF1E200E2002B0BDEC048B10BD00205F
:10039000F9E70E20F7E700BF7DC3050892C3050803
:1003A000E81B0608000000009FC305080B46D3EDBC
:1003B000020A93ED010A1146FFF708BFD0E90212C5
:1003C0000346C86882420AD00869496850F822008A
:1003D00001328A42DA6003D10022DA6070470020DD
:1003E000704700000346084603499A6801600349C4
:1003F000C260C0E90113704710230608BD0303085B
:1004000070B5C5684268466984686B1C9A4208BF2B
:100410000023F60705D5A34203D108490848FCF795
:1004200005FF0669A34246F82510C36004D10133D5
:100430009A4208BF00238360062070BD74CA050875
:10044000101B0608836810B55BB14469C268E407F5
:1004500003F1FF3307D5934205D109490948FCF759
:10046000E5FE4368F1E704698360934244F8231092
:1004700003D103B94368013BC360062010BD00BF30
:1004800074CA0508101B060830B585B00546084635
:100490006946FDF797F904462046FDF707FA01463D
:1004A00010B9062005B030BD2846FFF7A9FFF3E7D5
:1004B00070B504460E461546CAB1D4E90223991A0E
:1004C00048BF6368006848BFC91832460023FEF77A
:1004D00045FEA36818446368834298BFC01A236925
:1004E000042D0EBF53F8205043F82050062528460F
:1004F00070BD0000F8B51E460F460446114638464A
:10050000124AFEF739F97068FEF74AFD051E02DA55
:100510000020FDF7ABFC21461820FEF73FFC044607
:100520000023681C6060C4E902338000EFF7BBFE63
:10053000022F206103D9B068FEF732FD6061316897
:100540002046FFF7A1FF2046F8BD00BF06000400CB
:1005500008B5D0E902239A4203D107490748FCF7BE
:1005600065FE03B943680269013B0021C36052F88C
:10057000230042F8231008BDACC30508101B060871
:10058000042803D0052808D000207047D1E90203D1
:1005900098420CBF0E201E207047D1E90230C01ACD
:1005A00044BF4B68C018400040F001007047000095
:1005B000D0E902318B4210B5024603D108490948FF
:1005C000FCF734FE0169002451F8230041F8234070
:1005D000516801338B4208BF2346936010BD00BFB2
:1005E000ACC30508101B0608042803D0052807D053
:1005F000002070474B68082B34BF0E201E20704728
:100600004868C0F3DC00400040F001007047000083
:100610000346054A0A601A7A0A715B688B600023F8
:100620000846CB60704700BF28180608062802D18C
:100630000B7A022B02D04968FFF7D6BF490041F080
:1006400001007047044B0B6001230B71002388608D
:10065000CB600846704700BF2818060810B504494B
:1006600004460C20FEF79AFB02220272446010BD81
:100670004018060808B503799B0702D50020FDF74E
:10068000A1FD08BDF8B50F6806460D46144612B127
:100690003846FFF7EFFF69682246381DFEF75AF922
:1006A000034608B1406870B9022E05D1022C08D16A
:1006B00069680748FDF7B0FDA868012C00D15860B3
:1006C000F8BD0620F9E7022C04BF00225A60F7E7C4
:1006D000EC1A06080122FFF7D5BF0222FFF7D2BFAE
:1006E0000022FFF7CFBF10B50446FFF7C3FF201D60
:1006F000FEF71DF9062010BD30B50B68856802466F
:10070000AB4201D300200AE0D46804EBC30054F8E4
:1007100033400133002CF3D0042CF1D00B6030BDFA
:1007200013B5044600F10C018068FFF7E5FF60B1E6
:100730002379012B0BD0022B43680AD0026869464B
:100740000220CDE9002306F057F902B010BD006881
:10075000FBE71846F9E700007FB5174B0A7A0D460C
:10076000044653F82210F0F78AFE14492046F0F7A9
:1007700086FE134B00932B7A8DF804306B6802933E
:100780000023039301266846FFF7CAFF054630B9E8
:100790000C49204604B0BDE87040F0F770BE1EB9A9
:1007A00009492046F0F76BFE012229462046FEF754
:1007B00015FB0026E7E700BF1C180608AFC30508B5
:1007C00028180608B2C30508EEC205081FB504467E
:1007D000FFF750FF6368072B03D812491248FCF754
:1007E00025FD002201922279510744BFC3F3DC03A7
:1007F00003F1FF3301A9204648BF0193FFF77CFFB7
:100800006368083B636003680293436803930422B0
:100810000023C0E9002302A9022006F0EDF804B08D
:1008200010BD00BFB5C30508EC1A06082DE9F74F47
:100830000B68DFF8F090032A0EBFD0E902ABDFF8B7
:10084000E8B0DFF8E8A0154618BF01254B4504467F
:10085000884605D0032D03D0DA882C49F1F7C8F972
:100860002B492046F0F70BFE00230193012701A935
:100870004046FFF741FF064680B926492046F0F77B
:10088000FEFDD8F800304B453CD0032D3AD022492C
:10089000204603B0BDE8F04FF0F7F1BD1FB9514657
:1008A0002046F0F7ECFD032D2AD1336803F0070250
:1008B000022A25D013F0030708D11B681A7B2AB13E
:1008C00003EB82031A69154B9A4204D0144920465F
:1008D000F0F7D5FD012731682A462046FEF77EFA5B
:1008E0001FB10F492046F0F7CAFD59462046F0F7E0
:1008F000C6FD71682A462046FEF770FA0027B6E763
:100900000027E8E703B0BDE8F08F00BFCEC30508BD
:10091000D2C3050877BF050803E00508495403085A
:10092000D4C30508C01806081DD70508EEC205087F
:1009300010B5044904460C20FEF730FA002202727A
:10094000446010BD4018060810B5044904460C2048
:10095000FEF724FA01220272446010BD4018060816
:1009600010F003030CD10268117A31B102EB81025D
:100970001369044A9A1A5342534103F00100704725
:100980000023FAE7B50A03082DE9F3470C68164679
:10099000074620460D46FFF76DFE3168314AC9080B
:1009A0003846FDF7E9FE022F12D16F683846FFF78F
:1009B000D7FF0146E8B12B689F4209D0002301937D
:1009C00004F10408686801A9FFF796FE074640B9DC
:1009D000002504347368AB4233D8062002B0BDE86A
:1009E000F087396801224046FDF7B4FF7B68436019
:1009F000E8E73846FCF7E6FE04F1040A814648467B
:100A0000FCF754FF0028E3D00021FCF7DBFE804612
:100A1000FCF74CFF07464046FCF748FF05464046BA
:100A2000FCF744FF17B91048FDF720FA002DFAD063
:100A30000028F8D1012239465046FDF78BFF45606A
:100A4000DDE7B36853F8351003EBC50739B1042966
:100A500005D001222046FDF77DFF7B68436001350C
:100A6000B8E700BF05000200D6C3050810B5002294
:100A700004300C46FDF76EFF18B903482146FDF718
:100A8000CBFB406810BD00BFEC1A0608024B40F8D3
:100A9000043BFDF729BF00BFC018060838B505465E
:100AA0001020EFF7E7FB29460446FFF7EFFF20464B
:100AB00038BD00002DE9F041804686B000200D468B
:100AC00016461F46FFF7EAFF0F4BC0F80080984517
:100AD00002BF037943F00403037155EA0603044699
:100AE0000DD03B68019007EB8502314603A80293C5
:100AF000FDF707FF03AA01A9681CFFF745FF204681
:100B000006B0BDE8F08100BFF0180608F8B50C4645
:100B1000064600216068FCF755FE022E0546606817
:100B20008CBFA6680626FEF761FB50B9FFF7B6FF3B
:100B30000446071D2846FCF7B9FE014618B92046B1
:100B4000F8BD4010F2E701223846FDF703FF46608A
:100B5000F0E738B504468068FFF7A0FF23686268B5
:100B60000360237922F0070203F005031343436077
:100B7000A268E1680546D200C06819F083FD2846E6
:100B800038BD0000F0B5162885B00C46154663D078
:100B900005D8022810D0092862D0002409E02428B2
:100BA000FBD100222946201DFDF7D4FE00282ED1BE
:100BB0000E24204605B0F0BD02F003038A0728D1B9
:100BC0000A682B498A4224D1002BF1D1296891422D
:100BD00021D1CDE9013301A92046FFF78DFD02A9FE
:100BE00007462846FFF788FD064677B10028DFD084
:100BF00031683868FEF7B8FB0028D9D0716878688A
:100C0000FEF7B2FB0028E6D1D2E70028D0D11E249F
:100C1000CFE7002BCCD12A68164B9A42C8D1636823
:100C20006A685340072BC3D800230293043502A9F6
:100C30002046FFF761FD06460028E8D03168002213
:100C40002846FDF787FE0028B2D041687068FEF79D
:100C50008BFB0028EBD1ABE70846FFF77AFF044691
:100C6000054A02A90220CDE90245FFF78DFEA0E763
:100C7000F0180608C01806082819060810B40C7ADF
:100C8000012C06D1242804D149685DF8044BFFF7F4
:100C900079BF00205DF8044B70474068C00870477A
:100CA00070B504460E461546FFF7E4FC01223146B6
:100CB000201DFDF74FFE4560204670BD13B5022292
:100CC000CDE90001044669461046FFF7DBFC2046EB
:100CD00002B010BD38B50C461AB9FFF7EFFF062079
:100CE0000BE0042A0AD100220430FDF733FE18B9C4
:100CF00004482146FDF790FA406838BDFFF7D0FF61
:100D0000EDE700BFEC1A060813B504464068FCF78F
:100D1000CDFD58B1A3685A1C5B0043F00103CDE937
:100D20000030A2606946022005F066FE02B010BDE8
:100D30001FB50446084611461A4602AB01930A4BFA
:100D400000930223FDF7A2FD21460C20FEF726F8B2
:100D5000002104460298FCF735FD039B60602046A5
:100D6000A36004B010BD00BF34190608C3685A68F8
:100D7000012A70B506462AD19D68AB0727D12A689B
:100D8000154B9A4223D1EC682378FF2B20D14A20BF
:100D9000EFF77BFA044638B9104AD2F81832343BE0
:100DA000492B12D9946B3434E9682046F0F7FAF9EC
:100DB000EC60204619F0E8FC0023A8606B60A9688D
:100DC0002046F0F74BF8686001E0054BF36070BD1A
:100DD0006B68002BFBD1F2E7B0290608B4040020B1
:100DE000BC2A0608F8B5164602F07F07320605460B
:100DF0000C460AD47B1E012B0DD80B68D888F0F75F
:100E00005CF901462846F0F73AFB022F03D123494B
:100E10002846F0F734FB2046FFF7A8FF16F07D07C1
:100E200034D1E3680BB15A682AB928461C49BDE899
:100E3000F840F0F724BB20681A4988421FD1022AE3
:100E40001DD89868C3071AD509F088FB0346B0B1CE
:100E5000E2681549926828465210F0F7C9FEE36827
:100E60005B68012B19D90D492846F0F708FBE368A8
:100E7000D9683A462846BDE8F840FDF7AFBFE368B9
:100E80005A68012A02D199680022F3E7E1683246E4
:100E90002846BDE8F84005F035BDF8BD1DD705086A
:100EA0002CD80508801A060808C405082DE9F8435F
:100EB0000D46044611462846194A1A4F9846FDF732
:100EC0005BFC1020EFF7E1F9002814BF8146B9461A
:100ED0000023C9F80040C9F808302DB9124CC9F8F0
:100EE0000C404846BDE8F883AE1CB6003046EFF72C
:100EF000CCF9044648B9D7F8F02106F118039A4214
:100F0000A7F12807EADBBC6B1834084BA6F10802EE
:100F1000C4E90035414604F1080019F0B3FBDEE7EF
:100F2000FEFF0100DC040020BC2A0608F82A06089F
:100F3000F8B51546D0E901320F46511999420446D9
:100F40000FD30178D9B105F110061E44C068012203
:100F50003146EFF7B5F978B96568A3682070013DAF
:100F6000ED1AD4E902302A461844394619F08AFBB2
:100F7000A3682B44A360F8BD6660E060F1E7013B25
:100F80009D1AEEE7024B0022C3F818229A637047BD
:100F9000B404002010B5FEF703F8041E11DDEFF7CE
:100FA00069F90346084A906BEFF3108172B6C2F8F4
:100FB0001842936381F3108808B1EFF783F9062094
:100FC00010BD0023EEE700BFB404002038B505468D
:100FD000FDF7F0FE007A70B12846FDF7EBFE0446FF
:100FE0002846FDF7E7FE037A04EB8304024B2069F1
:100FF000C31A5842584138BDAD0E030810B5044617
:10100000FFF7E4FF00B92469204610BD10B5FFF7D3
:10101000F5FFC3685B68044623B1FFF7A7FEE368EA
:10102000986810BD0620FCE738B5136805461446DD
:101030004BB1B1F55C7F05D15368062B02D100237B
:10104000C380236038BD3D2903D1FFF78FFEEB68D5
:10105000F7E7A22903D040F2FA339942F2D12846A9
:10106000FFF7D4FF2060EDE700231A461946FFF78B
:101070001DBF000073B5054610200E46EFF705F9B9
:10108000044630B9104BD3F81822332A12DD9C6B7A
:1010900024340E4B2360304619F076FB0022C4E95D
:1010A0000206626001AB012128460194FFF7FEFEB3
:1010B00002B070BD034602460146284602B0BDE8B4
:1010C0007040FFF7F3BE00BFB4040020B02906084B
:1010D0002DE9F04306469BB010200D461746EFF76A
:1010E000D4F80446284619F04FFB00F10109804668
:1010F0004846EFF7CAF80CB1002848D12549D1F885
:101100001822432A29DD886BA2F1340900F1240456
:101110000121343003AB01931F4B02932B78CDF8A0
:10112000109081F001010022FF2BCDE905208DF800
:101130000C1004D1294607A8F0F734F807AD3A4659
:10114000294601A8F0F7A4FBDDE905320021D154BE
:10115000059BA360069BE3600CE044B9234622464E
:10116000214630461BB0BDE8F043FFF79FBE70B983
:10117000C4E902850022094B2360626007AB0121AC
:1011800030460794FFF792FE1BB0BDE8F0830021C4
:10119000C0E700BFB4040020310F0308B0290608DF
:1011A0000EB403B503AA52F8041B0192FFF790FF97
:1011B00002B05DF804EB03B07047000083070BD169
:1011C0000268084B9A4207D1037A2BB100EB8303E4
:1011D0001A69054B9A4202D0044906F0EFBB012080
:1011E000704700BF8C2B0608AD0E03082C1D0608A7
:1011F00010B50446FFF7EAFE50B92046FDF7DAFDC8
:10120000FFF7DCFF20B12069024BC01A18BF012094
:1012100010BD00BFF02B060838B504460D46FFF799
:10122000E7FF18B12046FDF7C5FD044629462046D4
:10123000BDE8384006F0C2BB2DE9F04188461746AC
:101240001E46FFF7DBFE04468068E0B90C20EFF78E
:101250001CF8A060A8B9164BD3F81822172A0EDD87
:10126000986BA0600623A3800023E380E38800EB53
:101270008302D91CE18040F82380C2E90176BDE8F1
:10128000F0810323EFE7E388A5880233AB42EDDB6F
:10129000074B9B6B9842F2D003350122A900EFF770
:1012A0000FF80028EBD0A388A0600333A380DDE70C
:1012B000B404002038B50D461446FFF79FFE83683E
:1012C0001BB1C2882A60236038BD1A46FAE737B5D9
:1012D0000446A068FCF7EAFA019068B16568062D3B
:1012E00005D001AB002201212846FCF78FF8FDF75D
:1012F0009BFF0028EDD0019803B030BD38B50446FF
:10130000084611464FF004121D46FDF735FA2146F6
:101310000C20FDF743FD2B684360044600216868FC
:10132000FCF750FAA060204638BD13B54FF0FF33EC
:101330006322CDE900320C4694ED010A00234FF4FC
:1013400080726721F0F732FA02B010BD38B52DED8A
:10135000048BD0ED009A91ED009AB0EE690AF0EEA0
:10136000490A05460C4617F043F979EEC07AB5EE06
:10137000400AF1EE10FAC7EE898AB0EE408A21D118
:1013800019EE103A9FED248ADFED247A002BB8BFC6
:10139000B0EE678AF5EE408AF1EE10FA29D1C9EE77
:1013A000897A9FED1D0A17EE903ADFED1C7A002B2B
:1013B000B8BFB0EE670A85ED000A84ED008ABDEC87
:1013C000048B38BDB5EEC00AF1EE10FAB5EEC09A46
:1013D0004CBF01220022F1EE10FA4CBF0123002382
:1013E0009A421EBFF7EE007A30EE098A78EEE78A5D
:1013F000D0E7B0EE680A18F0E9FB78EEC08AF6EEA6
:10140000007AF4EEE78AF1EE10FAC4BFF7EE007A44
:1014100030EE270ACFE700BF000000000000008088
:1014200008B508202DED028BB0EE408AEEF722FFC2
:1014300080ED018ABDEC028B014A026008BD00BF4D
:10144000681D060830B50D4687B0114628460222B1
:101450001C46FDF791F935B99FED100A07B0BDE8BC
:101460003040FFF7DDBF2068012203A9FDF7C4FF6C
:1014700040B10023DDE9030100931A46FBF79CF914
:1014800007B030BD2068830703D10268044B9A423D
:10149000F6D0FDF7DBFDFFF7C3FFF1E7000000002A
:1014A000681D060891ED010A07281DD8DFE800F045
:1014B0000A181C1C041C0C14B5EE400AF1EE10FABC
:1014C00014D01E2108467047BDEEC00A10EE103A37
:1014D000590041F00101F5E710EE103A002BF1DA66
:1014E000B1EE400AFFF79CBF0021EBE70E21E9E7D0
:1014F00090ED010A7047000030B52DED028B0C46CF
:1015000087B0054603A920468DED010AFDF762FD6F
:10151000002800F0C680232D00F22781DFE815F0B7
:10152000E900F50001010D01190125012501250141
:1015300025012501250125012501250124002D0076
:10154000340025013B004F005D008F00250125017F
:1015500025012501250124002D00340025013B0033
:101560004F005D008F00CE00DDED017A9DED037A26
:1015700077EE877ACDED017A1CE0DDED017A9DED05
:10158000037A77EEC77AF5E7DDED017A9DED037A10
:1015900067EE877AEEE7DDED037AF5EE407AF1EE5D
:1015A00010FA03D172497348FBF740FE03A901A862
:1015B000FFF7CCFE9DED010AFFF732FF71E0DDED94
:1015C000037AF5EE407AF1EE10FAEBD0DDED016A28
:1015D00086EEA77A8DED017AECE79DED038AB5EEF4
:1015E000408AF1EE10FADDD09DED010AF0EE480AD6
:1015F00016F0FEFFB5EE400AF1EE10FA0AD118EE31
:10160000103ADFED5D7A9FED5D7A002BB8BFF0EE0A
:10161000477AAFE7B5EEC00AF1EE10FAB5EEC08A30
:101620004CBF01220022F1EE10FA4CBF012300232F
:101630009A4240D038EE008A8DED018ABAE7DDED9E
:10164000018A9DED038AF5EE408AF1EE10FA0DD184
:10165000B5EEC08AF1EE10FA08D59FED497AF0EEAA
:10166000C87AF4EE477AF1EE10FA9BDDF5EEC08A07
:10167000F1EE10FA19D5B0EE480A18F0A7FAB4EE58
:10168000480AF1EE10FA10D0B4EE488AF1EE10FAE2
:101690000BD6DFED390A2146B0EE680A2220FEF7AC
:1016A00095FD07B0BDEC028B30BDF0EE480AB0EE00
:1016B000680A17F0C7FC8DED010A7BE7DDED037AC0
:1016C000F5EE407AF1EE10FA3FF46CAF03A901A8F1
:1016D000FFF73CFE9DED010AFFF7A2FE9DED030A18
:1016E0000490FFF79DFE04A90590022005F084F9FF
:1016F000D7E79DED017ADDED037AB4EEE77AF1EEFE
:1017000010FA4CBF1E200E20CBE79DED017ADDEDD7
:10171000037AB4EEE77AF1EE10FACCBF1E200E2069
:10172000BFE79DED017ADDED037AB4EE677AF1EE65
:1017300010FA0CBF1E200E20B3E79DED017ADDEDFF
:10174000037AB4EEE77AF1EE10FA94BF1E200E2071
:10175000A7E79DED017ADDED037AB4EEE77AF1EECD
:1017600010FAACBF1E200E209BE7002099E700BFB7
:1017700065C10508E81B06080000000000000080A5
